:1000000000400020F96B0000396C00003B6C0000E0
:1000100000000000000000000000000000000000E0
:100020000000000000000000000000003D6C000027
:1000300000000000000000003F6C0000416C000068
:10004000436C0000454E000075700000436C0000DA
:10005000436C000000000000436C0000436C000093
:10006000436C0000457300004D2D0000436C000000
:10007000436C0000436C0000436C0000436C0000C4
:10008000436C0000DD740000436C0000436C000012
:10009000436C0000436C0000436C0000436C0000A4
:1000A000436C0000436C00000000000000000000F2
:1000B0000000000000000000000000000000000040
:1000C00010B5064C2378002B07D1054B002B02D02E
:1000D000044800E000BF0123237010BD640200202B
:1000E0000000000030DE0000044B10B5002B03D0F0
:1000F0000349044800E000BF10BDC04600000000F6
:100100006802002030DE0000164B002B00D1144B9B
:100110009D46402292029A1A924600218B460F4633
:100120001348144A121A0AF081FF0F4B002B00D01B
:1001300098470E4B002B00D0984700200021040068
:100140000D000D48002802D00C4800E000BF0AF066
:100150002DFF2000290006F0ABFF0AF001FFC0468A
:100160000000080000400020000000000000000027
:10017000640200209C2F002000000000000000000E
:100180000123034010D104280CD90268120909D0B8
:10019000531E9B001A1DC1180979002902D0013392
:1001A0009342F8D1180070470023FBE70378002B37
:1001B00003D05AB2002A01DB013070473F2293433B
:1001C000C03B59424B41C01803789343802BF4D174
:1001D0000130F9E710B500240378002B01D120008D
:1001E00010BDFFF7E3FF0134F6E770B5002204000D
:1001F0000D00411C092003F0B9F8002806D00123A6
:100200006200134343600023A34200DB70BD9A00E9
:10021000A958821891600133F6E770B5012803DC14
:100220001C2000F0A1FE70BD01230D6811201D42AD
:10023000F7D04868184206D1042804D90F23026871
:100240001340042B01D00E20EBE702F0F9FE6D10F5
:100250000400002D03DDFFF7BDFFA84206DA1220DF
:10026000DFE72000FFF7A2FF0400013D012DF8D1D8
:1002700020787F2809DDDF280BDCF8233F22DB0014
:10028000800118406378134018430123400018434D
:10029000C9E7EF280BDCFC22637812019B011340B5
:1002A0003F220007000C0343A0781040ECE7F7283A
:1002B00012DCFC22637892021B031340E0228004CC
:1002C000520310403F221843E3781340FC220343BB
:1002D000A07812018001E8E701204042D5E7F0B59F
:1002E000070085B00D001C20012F06DD4C6801239E
:1002F00022001A40019203D10D2000F035FE54E097
:10030000022F02D08A681A42F6D001232E681E42BC
:1003100000D07EE0042E00D87BE01C41002C00DCE5
:100320001C000F2332681340092B29D173685B101E
:100330000193022F05D0AB68019A5B109A4200DD51
:100340000193019B01221F1B0137FB43DB171F4059
:10035000791C092003F00AF8061E09D001237F004A
:100360001F4303002A68083347600199A14202DA5B
:10037000300005B0F0BD0134A100515802C3F4E7CC
:10038000042B46D1300002F05BFEFFF723FF029002
:10039000022F04D0AB685B10984200DD0293029BF1
:1003A0009C4204DD002003F04DF80600E0E7300039
:1003B00002F046FE0700019B9C4222DC30000197C0
:1003C00002F03EFE03903800FFF7F0FE029B01347E
:1003D0000700A342F7DA019BC71A380003F032F88E
:1003E000061EC5D002F02CFE0400286802F028FE8C
:1003F000039A019B991A41183A0020000AF0FAFD6D
:10040000B6E73800FFF7D2FE019B070001330193E6
:10041000D1E7212071E7F8B54D680F00EB0706D44E
:10042000042D04D90F232E683340092B03D00B2051
:1004300000F09AFDF8BD6B6836095C10731EA3428C
:100440000FD80321200008F0ADFC6421642803DCF0
:100450000100032800DA03212800891902F0B6FF01
:1004600005002B6800201B09013B9C42E2D23A6840
:10047000A31C9B005A510123013464001C436C608F
:10048000D8E7F0B585B0012803DC1C2000F06CFD36
:100490002AE001244D682200022806D08B682342FE
:1004A00003D05C10002C00DC140001231D4200D09E
:1004B00073E0042D00D870E00F272B680E683B40D6
:1004C000042B27D1033B1E4205D1042E03D93368E8
:1004D0001F40042F01D00E20D8E72800FFF750FE60
:1004E000A04203DA0120404205B0F0BD280002F02E
:1004F000A7FD0700300002F0A3FD013C0100381900
:100500000BF04AF90028EDD00123C01B0130400058
:100510001843E9E7092B40D16B685B1000939C42BC
:10052000E0DC01231E4230D1042E2ED933683B403B
:10053000042B2AD1300002F083FD012302900193A5
:100540000397671CBB00E858864203D101986400FA
:100550002043C9E7019B18420ED104280CD9036837
:10056000039A1340042B07D102F06AFD01000298A0
:100570000BF0DCF80028E9D0009B3C009F42E0DD56
:10058000B0E71C00009B9C42ACDC631C9A00AA589C
:10059000B242F6D164000120DAE7212076E710B5F7
:1005A00002F032FD43000120184310BD10B57F2931
:1005B00002DC0170013010BD1A4B99420CDC402363
:1005C0008A115B42134303703F230B408021494251
:1005D000194341700230EEE7134B994210DC20239F
:1005E0000A135B4213433F24802203708B11524253
:1005F0002340214013430A43437082700330DAE7FB
:100600000A4B9942D7DCF0230370603B4370113BE7
:100610008A11FF3B1A4382703F2211401943C17077
:100620000430C8E7FF070000FFFF0000FF0F0100D4
:10063000F0B50D0085B0002803DC1C2000F094FC10
:100640000DE009680122080010400AD002AC1141F7
:100650002000FFF7ABFF011B200002F0FFFE0400AB
:100660001AE004293FD90F230C682340092B3AD103
:100670004B685B10019303239C46019B9A420EDD5D
:1006800002F0E0FE041E07D02E68012502F0D8FC1F
:100690002F00019B9D421DDD200005B0F0BD013201
:1006A0009300CC580123234001D10D20C6E76410EC
:1006B0007F2C0DDD0D4E0223B44209DD0C4E634646
:1006C000B44205DD00270B4EE30FA6427B419B00A1
:1006D000C018D2E70135AB00F1583942E5D04910D6
:1006E000FFF764FFD5E72120A8E7C046FF07000019
:1006F000FFFF0000FF0F010010B5040001200840BB
:1007000010D104290DD90F230A681340042B08D1F6
:10071000080002F095FC010020000BF007F84342AE
:10072000584110BD0020FCE7F7B50F00012803DC9D
:100730001C2000F019FCFEBD01264D682E4006D19C
:10074000042D04D90F222B681A40092A01D00B204E
:10075000EFE76A681B095410A34200D85C1E396891
:100760001E48FFF7C9FF01230190002813D1396803
:100770001B48FFF7C1FF002811D0002C0DD001232A
:10078000621C013C9C409200535123436B6004E087
:100790000136B200AB50B442FADA0020CBE73B6836
:1007A0000D20DA07C5D55B10002B11DD9C420FDB55
:1007B0009B00A200291DEB1889180433994209D126
:1007C0000123013C9C40AA181C4353606C60E4E781
:1007D0001220AEE758681860EFE7C046B7C60000C1
:1007E000BBC60000002310B50C000B70C30705D575
:1007F0000D49421020000AF05DFF08E00B49002877
:1008000002D0042804D10A4920000AF073FF10BD69
:100810000428FCD90F2302681340042BF7D102F0FF
:100820000FFC04490200E5E7F4CF0000C0C6000059
:10083000C6C60000CBC60000F0B593B0039003001D
:1008400002911C20012B1DDD029B01251B681C0051
:100850002C4000D0A8E0042B00D8A5E01A680F2394
:100860001A40092A48D10194019A029992008A58A3
:1008700016002E4005D1042A03D910681840092813
:1008800004D0222000F070FB07002CE052685210C8
:10089000A418019A013201920199039A8A42E3D184
:1008A000611C012202F062FD071E01D100271AE03F
:1008B00064002543456005000835029AB300D1580D
:1008C0004B680A685B1012099A4200D8531E002236
:1008D00093420BDCDA43D21713409B00ED18019BC7
:1008E00001369E42E9DB380013B0F0BD90000C18D1
:1008F000A46801322C50EBE7042A55D12F002600C2
:100900001D00029AB300D058384237D1042835D997
:1009100003682B40042BB4D1FFF732FC039B013654
:100920002418B342EDD1200002F08CFD071EBDD08B
:10093000039B029D9B00EB18041D029301232E686C
:100940001E4222D1042E20D90F2233681340042BDB
:100950000DD13000FFF714FC0190300002F070FB65
:10096000019A010020000AF045FB019BE418029B5C
:100970000435AB42E2D100232370B4E705A9FFF7A9
:1009800031FF05A80AF0DCFEC8E705A93000FFF733
:1009900029FF05A80AF0D4FE0600020005A92000E0
:1009A0000AF028FBA419E2E7212000F0DDFA7DE738
:1009B000F0B50D0095B0002806DC1C2000F0D4FA3C
:1009C0000400200015B0F0BD0C68012123000B408D
:1009D000009306D1042C04D922680F331A40092A47
:1009E00001D00B20EAE7626852100392002A03DC70
:1009F000009802F027FDE3E73F4A019201280BD05F
:100A00006868084208D1042806D902681340042BFC
:100A100002D102F015FB019001980AF091FE060048
:100A20000F27039B0834013B04935E43039B029012
:100A30009B001B19059301232068184251D10428FB
:100A40004FD903683B40042B52D1FFF799FB059B1C
:100A500004343618A342EED1300002F0F3FC041E39
:100A6000AFD02B680593029B002B03D0686802F07F
:100A7000E7FA0190200002F0E3FA0500009B059AD6
:100A80009B00D3189F68380002F0DAFA01230600B1
:100A90001F4201D1042F04D807A93800FFF7A2FE96
:100AA00007AE30000AF04CFE0700020031002800BB
:100AB0000AF0A0FA029BED19002B0AD0049B009AC1
:100AC000934206DD2800029A01990AF093FA029BEC
:100AD000ED18009B01330093009A039B9342CDD104
:100AE0006FE707A9FFF77EFE07A80AF029FEAEE729
:100AF00002F0A6FAF9E7C04633CA000010B5002498
:100B0000A04207DD0B6801341C4003D05C10E343B6
:100B1000DB171C40611C0122092002F027FC002881
:100B200003D0012364001C43446010BD0B6870B502
:100B300018000125284032D1042B30D90F241A681F
:100B400049681440092C16D15C6812092C41A24254
:100B500000D8541E844205DC02200132904206DB9C
:100B600000200FE085005D19A9600130F2E78400E4
:100B700019510130F2E7032C11D1294203D113207E
:100B800000F0F2F970BD4910FF29F8D812090433BA
:100B900092009A189A42E3D919700133FAE70B20B0
:100BA00000F0E2F9DCE700000123F7B500264D680C
:100BB0000F002B400093B3420DD11E00042D0AD923
:100BC0000F222B681A40092A0FD16A681B09561098
:100BD000B34200D85E1E3968CB0713D54C10002CE9
:100BE00001DDA64219DA12202EE0042A04D12800E1
:100BF000FFF7C6FA0600EEE7009E032AEBD11E09B6
:100C0000B600E8E72E48FFF777FD002814D00AF079
:100C1000EDFC310008F0ACF94C1C009B002B4CD1D2
:100C2000042D4AD92A680F331340092B10D10134FF
:100C3000A40064592000FEBD39682248FFF75CFD1E
:100C400034000028E9D1113000F08EF90400F1E7FA
:100C5000042B2AD1280002F0F3F90600FFF7BAFAB4
:100C6000A042C0DB012C1ADC280002F0E9F9009058
:100C70003000FFF79BFA851B280002F0E3FB041EFF
:100C8000D8D002F0DDF90190786802F0D9F9009B24
:100C90002A00F11A411801980AF0ACF9CAE73000AD
:100CA000FFF784FA013C0600DCE7032B05D12C1981
:100CB000E478023B64001C43BCE70B20C4E7C04659
:100CC000B0C60000BBC60000F7B54C680F0001209D
:100CD000210001402AD1042C28D90F222368BE68A4
:100CE0001A40092A13D162681B0955100191AB42C1
:100CF00000D85D1E39682848FFF7FEFC002829D07F
:100D00000F2322681340092B19D1012313E0032A72
:100D10000CD1064203D1132000F026F9FEBD72105B
:100D20000192FF2AF7D81D09AD00E3E70B20F3E796
:100D300001339A00A6509D42FADA0020EEE7032B19
:100D4000FBD1230001331A1BAA42F6DC6A46127952
:100D5000DA70F7E73968CB0706D54910002901DDBD
:100D60008D4209DA1220D7E70C48FFF7C5FC2900AD
:100D7000002801D11130CFE70F2322681340092B3F
:100D800003D1013189000E51D7E7032BD5D16B4632
:100D90001B796418E370D0E7B7C60000BBC600003B
:100DA00010B501240868204216D1042814D90F2256
:100DB00003681A40092A01D1406810BD032A03D1F3
:100DC0001809C0002043F8E7042A05D102F038F9D9
:100DD000FFF700FA4000F5E70B2000F0C5F8ECE75C
:100DE00010B5034A0A21034804F024F910BDC04697
:100DF00060C6000058C6000010B50124044002D0AF
:100E00004410200010BD04280CD90F2302681340A1
:100E1000042B07D102F014F921000A220AF058FD30
:100E20000400EEE70D22014B1A70EAE7A40200204D
:100E30000123020010B51A4015D1042801D9026817
:100E400012090B4011D1042901D90B681B09002498
:100E5000934206D104309B000431C318984206D354
:100E60000124200010BD0022EBE70023EFE7047807
:100E70000A78002C01D1002AF2D0013001319442CD
:100E8000ECD00024EDE70000F0B585B003930190AD
:100E900002912C4E2C4B002A02D002223270013AD1
:100EA00000251A601B68F554019B9D4201DB05B0CB
:100EB000F0BD029AAB00D058234B1C68C8239B009E
:100EC00037191C1B0123184206D0204A4310210069
:100ED00038000AF0BDFB09E01D4A002802D00428B2
:100EE0001BD11C4A210038000AF0B2FB30000AF086
:100EF00027FC154A039B1060002B0CD0019B013B83
:100F0000AB4208DD144B984205D8431C13602022E5
:100F100032540022F2540135C6E704280FD90F23BA
:100F200002681340042B04D102F08AF80B4A030034
:100F3000CDE7092B04D14368094A5B10C7E70123B9
:100F4000084AC4E7A5020020C8050020F4CF00002D
:100F5000C0C60000C6C600001F03000003D6000084
:100F600030C900003FC90000014B187000207047D5
:100F7000A402002070B501F0D7FD094C0100251D29
:100F80001F2228000AF0F4FB28000AF0D9FB0423F2
:100F900004308008000118432060200070BDC04666
:100FA00080020020C368F0B59D00836889B05D1998
:100FB0000300183306930369069A9F00069B02906C
:100FC000DF19436901939B00D3180393CD4B1B7822
:100FD000002B26D17F222B68CB491C1213409B008B
:100FE0005B58043501929F46029B587804F000FC40
:100FF0000023029A137027E0C24B1B78002B10D1FC
:101000002B68019A1C121340BF4A9B009B58043561
:10101000E9E7069B3A1DD11ABA4BD82928DD1A22D6
:101020001A70029BB74C9B6821780193EA1A029BC5
:1010300092109B7812021A43029B587804F0E0FB4E
:101040000023029A23701370029B069A9B680193F7
:10105000ED1A029BAD10DD60069BFE1A029BB610D6
:101060001E61039B9B1A029A9B10536109B0F0BD4D
:101070001B783C60002B01D01700D2E72B68019948
:101080001C120B40A0499B005B5817000435AAE7CF
:10109000069B3A1DD11A9B4BD82902DD1A221A70E1
:1010A000BFE728681B78291D3860002B02D0170085
:1010B0000D00B6E76B6801991C120B4092499B002A
:1010C0005B58170008358EE7069B3A1DD11A8D4BE9
:1010D000D82902DD1A221A70A3E7A4001B782C1964
:1010E0003C60002B01D017009BE72B6801991C1274
:1010F0000B4085499B005B581700043573E7069B3E
:101100003A1DD11A7F4BD82902DD1A221A7088E7BE
:101110007E49A40061581B783960002B01D017006C
:101120007FE72B6801991C120B4077499B005B58A5
:101130001700043557E7043F744B3A68A400E250A7
:10114000704B1B78002B00D06BE72B68019A1C12A8
:1011500013406D4A9B009B58043544E76B4BA40039
:10116000E058FFF749FE043F06003868FFF744FEE9
:1011700036180120654B76000643E650614B1B781C
:10118000002B00D04DE72B68019A1C1213405E4AD9
:101190009B009B58043526E7069B3A1DD11A594BF4
:1011A000D82902DD1A221A703BE70698039C012118
:1011B000A04202D221000C3909681B783960002B4B
:1011C00001D017002DE72B6801991C120B404E49E6
:1011D0009B005B581700043505E7069B3A1DD11AA2
:1011E000484BD82902DD1A221A701AE7069903988B
:1011F00081420FD203000C3B1B6845495B10641809
:10120000E41AA40023583B603E4B1B78002B05D00A
:10121000170006E7182119700023F4E72B680199DD
:101220001C120B4038499B005B5817000435DAE666
:10123000069B039A934219D213000C3B1B68344A55
:10124000043FA4185B10E31A039A39689B00995075
:101250002C4B1B78002B00D0E3E62B68019A1C1264
:101260001340294A9B009B580435BCE61822254BA5
:101270001A70EDE7069B039A93422DD2244B3E1F32
:10128000E31814000C3C04932368049A5B10D31AEF
:10129000039A9B009858FFF7AFFD07903068FFF75F
:1012A000ABFD2468049B64101C1B079BA4001F1843
:1012B00001207F00039B0743E7503700114B1B7849
:1012C000002B00D0ADE62B68019A1C1213400E4A89
:1012D0009B009B58043586E618220A4B1A70EDE7EE
:1012E000069B3A1DD11A074BD82902DD1A221A7023
:1012F00097E60399A40061581B783960002B09D048
:1013000017008EE6A402002030C70000802D0020C8
:10131000FDFFFF3F2B6801991C120B40D7499B0032
:101320005B58170004355EE6043F039B3A68A4004F
:10133000E250D34B1B78002B00D072E62B68019A49
:101340001C121340CD4A9B009B5804354BE6039B6F
:10135000A4001C192368043F38685E10FFF74CFD99
:1013600036180120C64B76001B7806432660002BFA
:1013700000D056E62B68019A1C121340BF4A9B000E
:101380009B5804352FE6069BA4003F1BBC4CBB4278
:101390000CD82378002B00D043E62B68019A1C124E
:1013A0001340B64A9B009B5804351CE6B54801F033
:1013B00037FE2378002B00D033E62B68019A1C12ED
:1013C0001340AE4A9B009B5804350CE6A300ED1871
:1013D000002C00DA38E6AA4B1B78002B00D020E660
:1013E0002B68019A1C121340A44A9B009B58043599
:1013F000F9E5043F3B68042B04D1A300ED18002C51
:1014000000DA21E69E4B1B78002B00D009E62B6802
:10141000019A1C121340994A9B009B580435E2E53F
:10142000043F3B68042B06D0A200AD18002C02DA62
:10143000002B00D108E6924B1B78002B00D0F0E582
:101440002B68019A1C1213408C4A9B009B58043550
:10145000C9E53A1F13685B10013B002B06DD012133
:101460005B00A4000B432D191360EDE5844B1700BE
:101470001B78002B00D0D4E52B68019A1C12134076
:101480007E4A9B009B580435ADE53A00069B0C3222
:10149000D31AD82B03DD1A22794B1A70C1E5FF232A
:1014A00061005B001940FE3BFF3B19433960029924
:1014B00006988968241204916D1A0299AD108978F2
:1014C0002D020D4303999D40091A891099401D432F
:1014D0000B43BB60029B7D609C70E4B26A4BE400EE
:1014E0000392E358029A9360654A1278002A03D067
:1014F00008331D00039F94E51D00019A9B680C357D
:101500001C1213405D4A9B009B58039F6BE53B1FD9
:101510001C68039A069B93422DD10A20E3070CD442
:10152000042C13D90F2322681340042B11D120005F
:1015300001F086FD0AF004F90630643003F00CFE79
:1015400000280FD1043D069B03937DE50720042C62
:10155000F3D02000431E9841FA234042FF33184045
:101560000730EAE7029B2100587804F05BF900237A
:10157000029A1370E7E7039B039A0C3B1B680299DE
:101580005B109B00D31A0C3B1C601F1D1300083B13
:101590001B685A108A70D2B23B49D2005B00555882
:1015A0009B0A029A9B009560ED18039B069A043BE8
:1015B0001B685B109B00D3180393314B1B78002BE7
:1015C00000D02EE52B68019A1C1213402B4A9B0079
:1015D0009B58043507E53B1F1868FFF70DFCA40076
:1015E00006003F1B1E2827DC00280DDC244B1B783F
:1015F000002B00D015E52B68019A1C1213401F4ADE
:101600009B009B580435EEE401F07CFA033E36184B
:1016100001F078FA1D4B801B9842F9D8184B1B78C3
:10162000002B00D0FDE42B68019A1C121340134AD2
:101630009B009B580435D6E40123029A137001F0F5
:1016400061FA029B0A3886195E60FDE43B1F186848
:10165000FFF7D2FBA40006003F1B002818DC084B54
:101660001B78002B00D0DCE42B68019A1C1213407D
:10167000024A9B009B580435B5E4C04630C70000C1
:10168000A402002051C90000882500203F420F001D
:10169000C84B984203DD1D22C74B1A70C1E40123D9
:1016A000029A137001F02EFAFA239B005E43029B0C
:1016B0000A3E30185860C7E4A300FF1A0023200038
:1016C0001A003900FFF7E0FBBC4EBD4C316820002A
:1016D00001F0C4FEBB4B31681860200003F056FFD8
:1016E0003168200004F0A5F8B34B1B78002B00D024
:1016F00097E42B68019A1C121340B34A9B009B5835
:10170000043570E4AC4BA4001B783F1B002B00D0C9
:1017100087E42B68019A1C121340AB4A9B009B582C
:10172000043560E4029803F07BFDA34B1B78002B8B
:1017300000D076E42B68019A1C121340A24A9B0049
:101740009B5804354FE43B1F1B68002B3ED13B00E8
:101750000C3B1B68DA072CD5390001225B105800BE
:10176000083902430A60002B44DD0122590011436D
:10177000381F01603900083909681141CB1A390056
:101780000C390968114224D09B189340A4001343DC
:10179000039AA350884B1B78002B00D041E42B68A0
:1017A000019A1C121340884A9B009B580435FFF78E
:1017B0001AFC042B06D90F211A680A40092A01D104
:1017C0005B68C9E719227C4B1A702AE45B10013B65
:1017D000C9E7042909D90F200A680240092A04D15F
:1017E00002339B005B58A400D2E71922724B1A7097
:1017F000FFF717FC0435CDE7A300069AFB189B1AE8
:10180000D82B13DC0122631E002C14DC6A4B1B78DE
:10181000002B01D0FFF705FC2B68019A1C12134026
:10182000694A9B009B580435FFF7DDFB1A22624B87
:101830001A70FFF7F6FB3A601C000437E3E7069ADC
:101840003B1D9B1A5C4ED82B03DD1A233370FFF728
:10185000E8FB069B039AA40093422AD23B1F186818
:10186000FFF7CAFA011E21DD039B0C3B1A685210D8
:1018700082421BDB9007801A544B4018C018039B10
:101880008000C2583B1B1A604B4B3F1B1B78043730
:10189000002B01D0FFF7C5FB2B68019A1C121340E7
:1018A000494A9B009B580435FFF79DFB202333706A
:1018B000EAE71823FBE7434BA4001A683B1B1F0011
:1018C0001A603D4B04371B78002B01D0FFF7A9FBB2
:1018D0002B68019A1C1213403B4A9B009B5804350D
:1018E000FFF781FBA3009C46FE1A002C17DC1C228C
:1018F000314B1A70002333606346FF1A2E4B0437B6
:101900001B78002B01D0FFF78CFB2B68019A1C126F
:1019100013402D4A9B009B580435FFF764FB0020C1
:1019200033685A108300F15801230B4003D10D2175
:10193000214A1170DFE749108A4200DD0A000130B8
:101940008442EFDC012352001343D4E7A3009C46FA
:10195000FE1A002C17DC1C22174B1A700023336070
:101960006346FF1A144B04371B78002B01D0FFF796
:1019700058FB2B68019A1C121340134A9B009B587A
:101980000435FFF730FB002033685A108300F1580C
:1019900001230B4003D10D21074A1170DFE74910E5
:1019A0008A4200DA0A0001308442EFDC012352004F
:1019B0001343D4E780EE3600A4020020C8050020BF
:1019C000A50200200800002030C70000FCFFFF3FF8
:1019D0003B00083B1868FFF70FFA3B1F060018682A
:1019E000FFF70AFA0023864200DA0433A4003A1B08
:1019F00017001360E54B04371B78002B01D0FFF76D
:101A000010FB2B68019A1C121340E14A9B009B5863
:101A10000435FFF7E8FA3B00083B1868FFF7ECF9DC
:101A20003B1F06001868FFF7E7F9F30FC217B04233
:101A30005341A4003A1B17009B001360D34B04379B
:101A40001B78002B01D0FFF7ECFA2B68019A1C12CF
:101A50001340CF4A9B009B580435FFF7C4FA3B0064
:101A6000083B18683B1F1968A600BE1B042381426F
:101A700002D0042802D80023336018E001239C46DA
:101A80001842F8D10F2302681A40042AF3D16346A2
:101A90001942F0D10429EED90B680B321340042B04
:101AA000E9D1FFF7C5F9431E984180003060B74B7C
:101AB000A4001B783F1B0437002B01D0FFF7B1FABD
:101AC0002B68019A1C121340B14A9B009B580435A5
:101AD000FFF789FA3B00083B18683B1F1968A6000E
:101AE000BE1B0023814202D0042802D804233360A5
:101AF00018E001239C461842F8D10F2302681A40CF
:101B0000042AF3D163461942F0D10429EED90B68B7
:101B10000B321340042BE9D1FFF78AF943425841B5
:101B200080003060994BA4001B783F1B0437002BCA
:101B300001D0FFF776FA2B68019A1C121340944AE1
:101B40009B009B580435FFF74EFA3B00083B186892
:101B5000FFF752F93B1F06001868FFF74DF9F3171E
:101B6000C20F86425341A4003A1B17009B0013602A
:101B7000864B04371B78002B01D0FFF752FA2B68F5
:101B8000019A1C121340824A9B009B580435FFF7B0
:101B90002AFA3B00083B1868FFF72EF93B1F0600A6
:101BA0001868FFF729F90023864200DD0433A400FA
:101BB0003A1B17001360754B04371B78002B01D0BC
:101BC000FFF72FFA2B68019A1C121340704A9B00F2
:101BD0009B580435FFF707FA3B1F1B68A400043B22
:101BE0005A1E93413A1B17009B001360674B043742
:101BF0001B78002B01D0FFF714FA2B68019A1C12F6
:101C00001340634A9B009B580435FFF7ECF93B00F7
:101C1000083B1868FFF7F0F83B1F06001868FFF74D
:101C2000EBF832180120A4003B1B1F0052000243B6
:101C30001A60564B04371B78002B01D0FFF7F1F9DF
:101C40002B68019A1C121340514A9B009B58043583
:101C5000FFF7C9F93B00083B1868FFF7CDF83B1FB9
:101C600006001868FFF7C8F8321A0120A4003B1BD1
:101C70001F00520002431A60444B04371B78002BAC
:101C800001D0FFF7CEF92B68019A1C121340404A8D
:101C90009B009B580435FFF7A6F93B00083B1868EA
:101CA000FFF7AAF83B1F06001868FFF7A5F8020027
:101CB0000120A4003B1B1F007243520002431A6024
:101CC000324B04371B78002B01D0FFF7AAF92B68A1
:101CD000019A1C1213402E4A9B009B580435FFF7B3
:101CE00082F93B1F1868FFF787F8061E17D11F23DC
:101CF000264A1370A4003B1B1F001E60234B0437B1
:101D00001B78002B01D0FFF78CF92B68019A1C126D
:101D100013401F4A9B009B580435FFF764F93B00B2
:101D2000083B1868FFF768F8310007F03BF8012618
:101D300040000643DEE73B1F1868FFF75DF8061E0C
:101D400017D11F23114A1370A4003B1B1F001E60F4
:101D50000E4B04371B78002B01D0FFF762F92B687C
:101D6000019A1C1213400A4A9B009B580435FFF746
:101D70003AF93B00083B1868FFF73EF8310007F0DE
:101D8000F7F8012649000E43DEE7C046A402002012
:101D900030C700003B1F1868FFF72EF8C2178018E5
:101DA00050400122A4003B1B1F004000104318605C
:101DB000F14B04371B78002B01D0FFF732F92B6869
:101DC000019A1C121340ED4A9B009B580435FFF703
:101DD0000AF9A300FE1A3068012C24D1FFF70CF891
:101DE0000494079009F002FC0799002900DC012106
:101DF00007F0BEF8049BA400C91801234900194349
:101E0000DD4B3F1B1B7831600437002B01D0FFF7FF
:101E100008F92B68019A1C121340D84A9B009B5862
:101E20000435FFF7E0F8FEF7E7FF04907068FEF76F
:101E3000E3FF049B0130C31A0793D3E7A300FE1A04
:101E400031002000049301F0B3FC049B3060FF1AC2
:101E5000C94B04371B78002B01D0FFF7E2F82B6841
:101E6000019A1C121340C54A9B009B580435FFF78A
:101E7000BAF83B00083B1868FEF7BEFF3B1F0600A0
:101E80001868FEF7B9FF02000120A4003B1B1F00E9
:101E90003240520002431A60B74B04371B78002BC4
:101EA00001D0FFF7BEF82B68019A1C121340B34A09
:101EB0009B009B580435FFF796F83B00083B1868D9
:101EC000FEF79AFF06003B1F1868FEF795FF3200E9
:101ED00002430120A4003B1B1F00520002431A6072
:101EE000A54B04371B78002B01D0FFF79AF82B681D
:101EF000019A1C121340A14A9B009B580435FFF71E
:101F000072F83B00083B1868FEF776FF06003B1F9F
:101F10001868FEF771FF320042400120A4003B1B0D
:101F20001F00520002431A60934B04371B78002BAA
:101F300001D0FFF776F82B68019A1C1213408F4AE4
:101F40009B009B580435FFF74EF83B1F1868FEF7BF
:101F500053FFC0430122A4003B1B1F00400010435D
:101F60001860854B04371B78002B01D0FFF759F818
:101F70002B68019A1C121340804A9B009B58043521
:101F8000FFF731F83B00083B1868FEF735FF060005
:101F90003B1F1868FEF730FF3200824051000122DB
:101FA000A4003B1B1F000A431A60734B04371B78C5
:101FB000002B01D0FFF735F82B68019A1C12134053
:101FC0006E4A9B009B580435FFF70DF83B00083B19
:101FD0001868FEF711FF06003B1F1868FEF70CFF9C
:101FE0003200024151000122A4003B1B1F000A43A2
:101FF0001A60614B04371B78002B01D0FFF711F8F2
:102000002B68019A1C1213405C4A9B009B580435B4
:10201000FEF7E9FF3B000C3B1868FEF7EDFE3B00C6
:10202000083B06001868FEF7E7FEF1170200C31729
:10203000300006F0EFFF3B1F049005911868FEF793
:10204000DBFE02000498059906F098FF430001208A
:10205000A4003E1B37001843474B30601B78043701
:10206000002B01D0FEF7DDFF2B68019A1C121340F4
:10207000424A9B009B580435FEF7B5FFA300FE1AA9
:10208000310020000493FEF739FD049B3060FF1AF5
:10209000394B04371B78002B01D0FEF7C2FF2B68A9
:1020A000019A1C121340354A9B009B580435FEF7D9
:1020B0009AFFA300FF1A39002000FEF737FD2E4BD0
:1020C0001B78002B01D0FEF7ACFF2B68019A1C1285
:1020D00013402A4A9B009B580435FEF784FFA30057
:1020E000FE1A310020000493FEF75EFD049B306071
:1020F000FF1A214B04371B78002B01D0FEF791FF0C
:102100002B68019A1C1213401C4A9B009B580435F3
:10211000FEF769FFA300FF1A39002000FEF7D4FD87
:10212000154B1B78002B01D0FEF77BFF2B68019A23
:102130001C121340114A9B009B580435FEF753FFB5
:10214000A300FE1A310020000493FEF729FE049B31
:102150003060FF1A084B04371B78002B01D0FEF7C4
:1021600060FF2B68019A1C121340044A9B009B5885
:102170000435FEF738FFC046A402002030C7000037
:102180003B1F186800F05CFF3A00083A1268030031
:10219000A400D10729D4042A0CD910680F221040BA
:1021A000013808280FD806F05FFD05200E220E0E1C
:1021B0000E0E2400F049180009F0B8FA43425841C5
:1021C0003B1B80001860ED4B3F1B1B780437002B36
:1021D00001D0FEF726FF2B68019A1C121340E84A33
:1021E0009B009B580435FEF7FEFEE649E3E7E6490F
:1021F000E1E7E649DFE7069B3E1DF31ADF4CD82BEB
:1022000003DD1A232370FEF70CFF00F085FC43006A
:102210000120184323783860002B02D03700FEF7E6
:1022200000FF2B68019A1C121340D54A9B009B5853
:1022300037000435FEF7D7FE069B3E1DF31ACF4C40
:10224000D82B03DD1A232370FEF7EBFE00F05AFCB7
:10225000CF4B400018400123184323783860002BEF
:1022600002D03700FEF7DDFE2B68019A1C121340E6
:10227000C34A9B009B5837000435FEF7B4FE012388
:10228000A600BE1B20001A003100FEF7FDFDC14C68
:102290002068643002F060FF002802D1043DFEF7A0
:1022A000D3FE029B21685A78BB4803F0D0FA012381
:1022B000029A3700137000F025FCB84B22681B68A7
:1022C000063253431818029B5860FEF7BDFEA60065
:1022D000BE1B2000012300223100FEF7D5FDAD4CCE
:1022E0002068643002F038FF0028D7D0AA4803F0F5
:1022F000A5F8DCE7A4003E1BFEF73CFE37009F4B31
:1023000030601B780437002B01D0FEF78AFE2B6863
:10231000019A1C1213409A4A9B009B580435FEF701
:1023200062FEA4003E1B300000F025FC3700934BFA
:1023300030601B780437002B01D0FEF772FE2B684B
:10234000019A1C1213408E4A9B009B580435FEF7DD
:102350004AFEA4003E1B300000F00FFC3700874B04
:1023600030601B780437002B01D0FEF75AFE2B6833
:10237000019A1C121340824A9B009B580435FEF7B9
:1023800032FEA300FE1A31002000049300F0F8FB97
:10239000049B3060FF1A794B04371B78002B01D067
:1023A000FEF73FFE2B68019A1C121340744A9B00F3
:1023B0009B580435FEF717FEA4003F1B380000F0C1
:1023C00011FC6E4B1B78002B01D0FEF72AFE2B6808
:1023D000019A1C1213406A4A9B009B580435FEF771
:1023E00002FEA300FE1A31002000049300F022FC3C
:1023F000049B3060FF1A614B04371B78002B01D01F
:10240000FEF70FFE2B68019A1C1213405C4A9B00DA
:102410009B580435FEF7E7FDA4003F1B380000F091
:102420004BFC564B1B78002B01D0FEF7FAFD2B68B6
:10243000019A1C121340524A9B009B580435FEF728
:10244000D2FD0121200000F01FFC4C4B1B78002B1B
:1024500001D0FEF7E6FD2B68019A1C121340484A92
:102460009B009B580435FEF7BEFD0021200000F0C4
:102470000BFC424B1B78002B01D0FEF7D2FD2B68E2
:10248000019A1C1213403E4A9B009B580435FEF7EC
:10249000AAFDA4003E1B300000F030FC3700374B93
:1024A00030601B780437002B01D0FEF7BAFD2B6893
:1024B000019A1C121340324A9B009B580435FEF7C8
:1024C00092FDA4003E1B300000F02CFC37002B4B8B
:1024D00030601B780437002B01D0FEF7A2FD2B687B
:1024E000019A1C121340264A9B009B580435FEF7A4
:1024F0007AFDA4003F1B380000F0EEFB1F4B1B7859
:10250000002B01D0FEF78DFD2B68019A1C121340A1
:102510001B4A9B009B580435FEF765FDA4003F1B3A
:10252000380003F0AFFC154B1B78002B01D0FEF7F1
:1025300078FD2B68019A1C121340114A9B009B588E
:102540000435FEF750FDA4003E1B300003F032FDC1
:1025500037000A4B30601B780437002B01D0FEF7A0
:1025600060FD2B68019A1C121340054A9B009B5882
:102570000435FEF738FDC04661C90000A402002002
:1025800030C7000069C9000070C9000077C90000A9
:10259000FEFFFF7FC8050020A502002004000020E8
:1025A000A4003F1B380003F01DFCC24B1B78002B1E
:1025B00001D0FEF736FD2B68019A1C121340BE4A6B
:1025C0009B009B580435FEF70EFDA4003E1B300017
:1025D00003F01EFC3700B74B30601B780437002B2C
:1025E00001D0FEF71EFD2B68019A1C121340B24A5F
:1025F0009B009B580435FEF7F6FCA300FF1A390038
:10260000200001F015FCAB4B1B78002B01D0FEF72E
:1026100008FD2B68019A1C121340A74A9B009B5887
:102620000435FEF7E0FCA300FF1A3900200001F09A
:102630003BFAA04B1B78002B01D0FEF7F2FC2B6875
:10264000019A1C1213409C4A9B009B580435FEF7CC
:10265000CAFCA300FF1A3900200001F021FB954BB2
:102660001B78002B01D0FEF7DCFC2B68019A1C12B2
:102670001340914A9B009B580435FEF7B4FCA3001D
:10268000FF1A3900200001F033FB8A4B1B78002B26
:1026900001D0FEF7C6FC2B68019A1C121340864A33
:1026A0009B009B580435FEF79EFCA300FE1A3100E8
:1026B0002000049303F023FD049B3060FF1A7D4B40
:1026C00004371B78002B01D0FEF7ABFC2B68019A76
:1026D0001C121340784A9B009B580435FEF783FC7C
:1026E000A300FE1A31002000049303F010FD049BA8
:1026F0003060FF1A6F4B04371B78002B01D0FEF7B8
:1027000090FC2B68019A1C1213406B4A9B009B584B
:102710000435FEF768FCA300FE1A31002000049384
:1027200003F0FDFC049B3060FF1A624B04371B78FA
:10273000002B01D0FEF775FC2B68019A1C12134088
:102740005D4A9B009B580435FEF74DFCA300FE1A22
:1027500031002000049303F0FDFA049B3060FF1A5F
:10276000544B04371B78002B01D0FEF75AFC2B6822
:10277000019A1C121340504A9B009B580435FEF7E7
:1027800032FCA300FF1A3900200001F0C5F9494BC3
:102790001B78002B01D0FEF744FC2B68019A1C1219
:1027A0001340454A9B009B580435FEF71CFCA300D0
:1027B000FF1A3900200001F0C3FA3E4B1B78002BB2
:1027C00001D0FEF72EFC2B68019A1C1213403A4AE6
:1027D0009B009B580435FEF706FCA300FE1A31004F
:1027E0002000049301F02AFA049B3060FF1A314B59
:1027F00004371B78002B01D0FEF713FC2B68019ADD
:102800001C1213402C4A9B009B580435FEF7EBFB2F
:10281000A300FF1A3900200001F0DCF9254B1B78DA
:10282000002B01D0FEF7FDFB2B68019A1C12134010
:10283000214A9B009B580435FEF7D5FB069B029A64
:10284000FB1A9B101361A300FF1A3900200002F04D
:1028500005FC184B1B78002B01D0FEF7E2FB2B6820
:10286000019A1C121340144A9B009B580435FEF732
:10287000BAFB069B029AFB1A9B101361A300FE1A77
:1028800031002000049302F0E9FB049B3060FF1A42
:10289000084B04371B78002B01D0FEF7C2FB2B68D6
:1028A000019A1C121340044A9B009B580435FEF702
:1028B0009AFBC046A402002030C700000023F7B5F1
:1028C0005A1E0192002B07DA01F0C8FA02F0BCFE92
:1028D00003F01CF81923019300263000194B1968E6
:1028E000B14212DD184B1A6801328A420FDAF02425
:1028F0001A601D68154F6C43E35D002B1FD0E4196F
:10290000022B06D12000FEF74DFB019BD8E70022E9
:10291000EDE7012B0DD1002801D100F0F3F8F022F2
:102920006A43BB185B680A49C31A8B4201D8022369
:10293000BB54F0235D43054BEB5C022BE2D0013628
:10294000CCE7C046CC05002000000020281C002059
:102950003F420F00012200210A4B0B481A61195017
:1029600004301950A2210420C9005850C121C020B0
:102970008900800258501A60044BFC311960044BE6
:102980001A70704700A000400405000000E100E05C
:10299000F305002004207047F8B550C90123220038
:1029A0001A40101E2DD03340181E2AD0641000206B
:1029B0001C2C26D81D4B761035009E4200DD1D00D4
:1029C0001B4F3B5D012B05D00121200004F006FDCB
:1029D00001233B55174B1B78002B01D1FFF7BAFFA2
:1029E0000023154A9E420DDCFF2514491448D65C8D
:1029F000B44202D15E007052D5540133042BF6D19B
:102A00000420F8BDD15C8C4203D10C4A5B009D527E
:102A1000F6E70133042BF5D10023D15CFF2901D166
:102A2000D454F2E70133042BF7D1E9E7881300000F
:102A3000D4050020F30500201C0000200E0000201B
:102A4000DC050000F8B530C9012623003340181E0C
:102A50001BD02B003340181E17D0344100201C2CF3
:102A600013D8174F3B5DB34204D03100200004F06F
:102A7000B5FC3E5569100800124A1038124B9042BE
:102A800004D9012252421A600420F8BD1C600F488C
:102A900006F088F90E4B18800E4B1B78002B02D1E4
:102AA000FFF758FFF0E701220B4B9A64A922D200EE
:102AB0009A588018A82280B2D2009850E4E7C04605
:102AC000D4050020908601001800002020A10700F6
:102AD0000C000020F305002000A0004004207047F7
:102AE00001220020054B06491A6158500431033079
:102AF00058500831801858501A60704700800040C4
:102B0000040500000122034B1A64A822D200985841
:102B10007047C0460080004010B5FFF7F3FFFA2170
:102B2000890006F0B5F810BD00487047BCC9000028
:102B30001D20704770B5054E0400335C0D008B42BC
:102B400002D004F04BFC355570BDC046D4050020C2
:102B500070B50024064D635D012B05D100212000D6
:102B600004F03CFC0023635501341D2CF2D170BDF0
:102B7000D405002070470D2070473B2070470000AF
:102B8000F8B501240B6806000D00234204D10D2086
:102B9000FEF7EAF92000F8BD5B102000052BFAD8FB
:102BA0000E4A9B009C580E4F3B5D002B05D0002128
:102BB000200004F013FC00233B55012E06DD6B685A
:102BC000042B03D10221200004F008FC200004F0B3
:102BD000B3FA012440002043DDE7C046A4C9000049
:102BE000D4050020F8B501260568354202D04468B6
:102BF000344203D10D20FEF7B7F9F8BD6D101C2D3E
:102C0000FBD80A4F7B5D012B04D03100280004F073
:102C1000E5FB7E55064964108C4202DCE143C9178E
:102C20002140280004F00EFBE7E7C046D405002051
:102C3000FF03000070B501240D68254204D10D206A
:102C4000FEF792F9200070BD6D101C2D17D80024DE
:102C5000012804DD4C68043C63425C416400094E79
:102C6000735DA34204D02100280004F0B7FB745523
:102C7000280004F0E7FB03000420012BE3D0002030
:102C8000E1E7C046D405002070B504000D001C2803
:102C90000ED8084E335C012B04D0012104F09EFBBA
:102CA00001233355290020004D1EA94104F0B4FB37
:102CB00070BDC046D4050020036810B5DA0703D400
:102CC0000D20FEF751F910BD4168581004394A42F1
:102CD0005141FFF7D9FFF6E737B569460A00064BC1
:102CE00030CB30C203680220042B02D100F0D8FFA1
:102CF00037BD00F0FDFFFBE77CC9000010B5084CB4
:102D00006379002B05D00021052004F067FB002328
:102D10006371052004F096FB43425841800010BDCA
:102D2000D405002010B5084CE37A002B05D0002113
:102D30000B2004F053FB0023E3720B2004F082FB12
:102D400043425841800010BDD4050020F7B5304DF6
:102D5000304E6B6C002B15D0A8240023E4003759AB
:102D60006B642D4B186800280CDB2C4B19784A42F9
:102D70005141C9B2197004F04FFB294B1B88DF1970
:102D8000BFB23751AB6C002B39D00021254B264FF9
:102D9000F458A9643A780C340193244D8A4206D041
:102DA0002B68032B03D8224AD05C04F035FB2B6838
:102DB000204A0133134004D50422013B52421343FD
:102DC00001331B4900228C462B60042B18D060462F
:102DD000C05C591CFF2802D10B000122F5E7002A34
:102DE00000D02B60012104F017FB01233B702B68FE
:102DF000114A5B009B5AE418019BA4B2F450F7BD42
:102E000001235B422B6000233B700C4BF3E7C04671
:102E1000FCA0004000A0004018000020F2050020A7
:102E20000C00002044050000F1050020D005002022
:102E30001C000020030000800E000020504600000F
:102E4000084B094AFF201A805A809A80DA800023B2
:102E5000064A07491370074A087048708870C8709E
:102E6000136070470E000020DC050000F105002013
:102E70001C000020D00500200122024B52421A60A3
:102E80007047C0461800002010B5034A04210348CB
:102E900002F0D0F810BDC04684C9000026D1000061
:102EA000E12170B54902144803F03EFFFFF718FE18
:102EB0000A2004F03BF90023FF21104A9954013302
:102EC0001D2BFBD1012200200D4B01001A600423B1
:102ED0000C4A0D4D1468002CFCD02C680002013BFC
:102EE00020431160002BF5D10122084B1A6004F039
:102EF000D7F801F0FFF870BDB01B0020D40500200A
:102F000000D0004000D1004008D5004004D000406F
:102F1000F8B50B4E070030000D0003F04DFF040024
:102F2000A84200DD2C003D00EB1B9C4205DD30007B
:102F300003F04CFF28700135F6E72000F8BDC046CD
:102F4000B01B002010B50100014803F0F5FE10BDD4
:102F5000B01B002010B5054C200003F0FBFEE12162
:102F60002000490203F0E0FE10BDC046B01B002067
:102F7000C3070CD4064B1B68834208D8054B1B685B
:102F8000984204D8031F1B68002B00D0180070471C
:102F9000FC050020F80500200023012210B50A4896
:102FA000990001334250642BFAD1084C084B0021A0
:102FB0001A602000074A08F039F8074B074A636097
:102FC000074B1A6010BDC046802D0020000600206F
:102FD00008000020D409000030270000040600206B
:102FE000F405002010B5044B044A1A60044B054A4E
:102FF0001A60FFF7D1FF10BDFC050020000600207D
:10300000F8050020D40F0020044B1B681868000945
:103010000238C343DB1718407047C046F405002050
:1030200000B59BB00200054901A808F043FB01A8C8
:1030300002F020FA02F06AFCFCE7C04623CA000056
:103040000A4BC20704D4042804D8094B00D0094B0A
:10305000180070470F2203681A40031D042AF7D096
:10306000054B092AF4D0054BF2E7C04609CA000017
:10307000C6C60000C0C600001CCA000013CA00007B
:103080000020064A0649131F186013681B09023303
:103090009B00D2188A42F6D37047C046040600202F
:1030A000D40F0020F7B50F240126304B304A1968A1
:1030B000304B314D186813681F002740072F25D863
:1030C00013681B0902339B00D218AA42F3D30024D1
:1030D0002A4EA500AD192868FFF74AFF0134286081
:1030E000642CF6D1264C2068FFF742FF2060254C67
:1030F0002068002802D0FFF73BFF20600025224B0C
:103100001B680093009B9D4213DBF7BD1B099B00CE
:10311000D3189A42D4D01F68374208D1B94206D298
:10312000B84204D3043F3F68002F00D01F60043B27
:10313000EFE7F0236B43154A9B181A78002A01D158
:103140000135DFE71F693C2300266B43DB199B0039
:1031500001930136BB1BF3D4019BB4001C1B0B4B2A
:103160001C19A069FFF704FFA061F2E7FC0500202D
:1031700004060020F8050020D40F0020802D002038
:1031800008000020D40F0020CC050020281C0020BF
:10319000F7B50124204244D1224B1B689C4698423B
:1031A0003FD3214B1B68019398423AD8031F1B68F9
:1031B000002B36D10200036800941B09002B0FD1AD
:1031C0000099131F196090422BD015682B1F1B68A4
:1031D000990069180C68013B14600A602A00EDE749
:1031E0009D0055192968009C214218D18C4516D89C
:1031F000019C8C4213D30E1F3468002C0FD10F6832
:103200000F343C40072C07D92F60151F2B600B682B
:103210000A601B090A00D1E700993160CEE7013B43
:10322000CCE7F7BDFC050020F80500200D49F0B5FE
:103230000B000F260C4D18681C1F2768020902326C
:10324000002F0BD000208B4200D00800206090009F
:10325000091892009B18AB42EDD3F0BDB043186043
:10326000F7E7C04604060020D40F0020F8B5114C43
:1032700026000F2233681F0913420DD07D1CAD00BC
:10328000A64204D02A003100200007F0BCFE002234
:103290006319043564191A600237BF00064BF6192A
:1032A0009E42E6D31B1B9B10013B1B012360034B7B
:1032B0001C60F8BD04060020D40F0020F405002097
:1032C000F0B59BB0FFF71EFC00240700204AA300C6
:1032D000D0580134FFF75CFF642CF7D11D4B186800
:1032E000FFF756FF1C4B1868002801D0FFF750FF6E
:1032F00000261A4B1B689E4216DBFFF797FFFFF76D
:10330000D1FEFFF7B3FFFFF7FDFB154BC21B1B6898
:1033100014491B6801A81B09023B08F0CBF901A85E
:1033200002F0A8F81BB0F0BDF02575430E4BED1868
:103330002B78002B01D10136DBE72B695C1E002CBA
:10334000F9DBA300EB189869FFF722FF013CF6E7D1
:10335000802D002008000020D40F0020CC05002084
:10336000F4050020E9C90000281C0020F7B5164D1F
:103370004F1C2B6806001B680C0001921B099F4222
:103380000ADBFFF79DFF2B681B681B099F4203DBCD
:103390000A20FDF7E9FDFEBD2868A71CBA00DB1B6B
:1033A00081181B010B6029600021031F19600F2386
:1033B0001E4003002401264340C3083A9A189A424B
:1033C000E9D9019902C3FAE7F4050020F7B5030033
:1033D0000122134004000D000193002B2AD1164B4B
:1033E0001B68834226D8154B1B68834222D90F23C2
:1033F000134F386000681840FFF7B8FF019B3C6826
:10340000061E3B6016D0236804301B099D4200DD78
:103410001D00AA00211D251F07F0ECFDFFF730FE5F
:103420002E60FFF73FFE00232B6022680F339A4384
:10343000226034002000FEBDFC050020F8050020BD
:10344000D40F00200323043010B5C1171940091808
:10345000891000220420FFF789FF10BD70B5050018
:1034600008000C00FFF7EEFF0023002804D170BD18
:10347000E95CC21811710133A342F9DBE343DB17A6
:103480001C40002304192371F1E7F0B50C009BB038
:10349000022804DC1C20FDF767FD1BB0F0BD0123F2
:1034A0000868184206D1042804D90F260168314063
:1034B000042901D00E20EEE761680D001D40F9D10E
:1034C0000429F7D90A683240042AF3D1A2681A42C3
:1034D00001D10D20DFE7FFF7B3FD06006068FFF7BD
:1034E000AFFDA768010001AC7F103000257002F02D
:1034F000C6FF39006423220003F026F8200008F0FC
:103500001FF901002000FFF7A9FFC6E710B51C4C0A
:10351000A544041E02D1FFF795FF0BE002F0C8FEA0
:103520000138062828D805F09FFB0909111829043D
:10353000240000208023DB009D4410BD200002F009
:1035400033FF011B2000FFF789FFF3E7200002F0A3
:10355000D9FE430001201843ECE780226946D200DF
:10356000200002F0E6FE684608F0EAF8010068462E
:10357000E9E704210348E6E70020CCE70420D9E787
:1035800000FCFFFF7CCA000070B50C00022803DCC1
:103590001C20FDF7E9FC70BD01230868184206D124
:1035A000042804D90F2501682940042901D00E20E0
:1035B000EFE761681942FAD10429F8D90A682A406C
:1035C000042AF4D1A2681A4201D10D20E1E7FFF7E5
:1035D00037FD05006068FFF733FDA4680100641043
:1035E000280002F04CFF210002F089FFFFF78EFF58
:1035F000D1E770B50D00012803DC1C20FDF7B4FCF9
:1036000070BD01240868204206D1042804D90F2186
:1036100002680A40042A01D00E20EFE76A682242BD
:10362000FAD1042AF8D913680B40042BF4D1FFF720
:1036300007FD06006868FFF703FD0100300002F097
:103640001EFF02F0A0FF40002043D9E7F8B50700B5
:103650000C001C20012F0BDD01250868284206D133
:10366000042804D90F2102680A40042A03D00E203E
:10367000FDF77AFCF8BD62682A42F8D1042AF6D92F
:1036800013680B40042BF2D1FFF7DAFC06006068E8
:10369000FFF7D6FC0100022F14D0A4682C4211D0F1
:1036A0006410300002F0EBFE050002F001FE01287C
:1036B00011D1002C02DD0135012C06D12800FFF7C5
:1036C00025FFD7E701246442EBE7280002F078FEEB
:1036D000013C0500F0E70228F0D1002CEEDD0135B9
:1036E000012CEBD000222800110002F09BFE02F01A
:1036F00067FE013C0500F3E710B5012408680440AB
:1037000016D04410200005F0E1FD134905F0ACFC93
:1037100007F092FB03F0DAFF0022104B06F046FDA3
:1037200003F07CFF07F018FB43000120184310BD95
:1037300004280CD90F2302681340042B07D1FFF78C
:103740007FFC21000A2208F0C3F80400DAE70D200C
:10375000FDF70AFCD6E7C046D30237390000D04057
:1037600010B5012803DC1C20FDF7FEFB10BD012075
:103770000A68024201D10C30F6E74B68034206D1D9
:10378000042B04D90F2419680C40042C01D00E20FE
:10379000EAE7090989005210002A01DD914201DAA5
:1037A0001220E1E79B18DB785B001843DEE700009E
:1037B000086870B501240500254006D1042804D905
:1037C0000F2302681340042B03D00E20FDF7CCFB1F
:1037D00070BDFFF735FC03782900233B5A42534163
:1037E0001022C01808F074F880239B05C218044BFF
:1037F0009A4201D91420E9E740002043E8E7C04697
:10380000FFFFFF3F10B5002803DC1C20FDF7ACFBD9
:1038100010BD01200B68034206D1042B04D90F22EE
:103820001B681A40042A01D00E20EFE71B09DB00B9
:103830001843EDE710B5034A0821034801F0FAFBED
:1038400010BDC0463CCA000034CA000000207047CA
:1038500010B51E20FDF788FB10BD10B51E20FDF72A
:1038600083FB10BD10B51E20FDF77EFB10BD10B50B
:103870001E20FDF779FB10BD10B51E20FDF774FB6F
:1038800010BD10B51E20FDF76FFB10BD10B51E203A
:10389000FDF76AFB10BD10B51E20FDF765FB10BDDE
:1038A00010B51E20FDF760FB10BD10B51E20FDF702
:1038B0005BFB10BD10B51E20FDF756FB10BD10B50B
:1038C0001E20FDF751FB10BD10B51E20FDF74CFB6F
:1038D00010BD000010B5034A0E21034801F0AAFBF9
:1038E00010BDC046C8CA000038CB00000120034B01
:1038F0001860034B1B68834018437047F80F002083
:10390000D80F0020F0B5EFF310810123194083F3A5
:103910001088134C134AA4461268134E013A934080
:10392000124F134A002B17D0146803420FD03D6882
:103930002C60C046C046C046C046C046C046C046D1
:10394000C0460C4C1568246825605B08EAE76546AC
:103950002C6014683460F8E781F31088F0BDC0462D
:1039600008050050200000200C050050E40F002046
:10397000EC0F0020E00F002030B585B001AD0C2227
:103980000649280007F036FB0024285D0121013498
:10399000FFF7D0F80C2CF8D105B030BDF7CB000004
:1039A000F7B56A46394B01AD13801C239370384B31
:1039B0002B800A23AB70FFF7A5F8364B364CC018A6
:1039C0002368984201D2002323602668002E3DD14F
:1039D0006B469F5D01213800FFF7ACF801360021EE
:1039E000380003F019FD032EF2D10026AF5D01214E
:1039F0003800FFF79FF801360121380003F00CFD75
:103A0000032EF3D1C8200138C046C046C046C04688
:103A1000C046C046C046C046C046C046C046C04676
:103A2000F1D100212878FFF785F868780021FFF7A9
:103A300081F8A8780021FFF77DF8FFF763F8FA23F3
:103A400000251B01C01820602800FEBDFFF75AF8B2
:103A5000236800259842F7D3032003F06DFB06008E
:103A6000042003F069FB36180A2003F065FB0B4BBA
:103A70009B1B181A0A4BA84206DB18600023094A50
:103A8000236013600125DFE71D60F7E71A1B0000C4
:103A90000304000010270000F00F0020E3030000E3
:103AA000D80F0020F80F00200022054B10B51A6037
:103AB000044B1B68934201D002F09AFB002010BD1A
:103AC000F40F0020D41A002010B5041E10DA0024D0
:103AD0000A4BA400E25801239340094A09491360A4
:103AE000094A1160094A0A4911600A4A136010BD67
:103AF000FFF71EF8A042EADDEAE7C046E8D800007A
:103B0000EC0F002008050050E40F0020E00F00201B
:103B10000C050050180500502B4BF7B51B680C0026
:103B2000002B03D101204042FFF7CEFF246801267D
:103B3000250035401AD0FF22631012026012104097
:103B4000DAB21043FF221B021204134018431F4B2A
:103B50001B68202B06D1B4401D4BA40EA400E358D3
:103B600000021843FFF7CEFE0020FEBD042CFBD957
:103B70000F2322681340092BF6D1FF2763683F0209
:103B80005B100193019B9D42EEDAAB00E3189B684A
:103B9000334216D05A105812D1B238400843FF2190
:103BA000120209040A401043084A1268202A06D16A
:103BB0005B009B0E06499B00020258581043FFF71A
:103BC000A1FE0135DEE7C046EC0F002020000020FA
:103BD000E0CD00000200086810B5C3070FD5401003
:103BE0001823012A03DD4A68042A00D10833054A54
:103BF0001360FEF7BFFFFFF767FF002010BD012035
:103C00004042EDE72000002010B50124044002D01E
:103C10004410200010BD04280CD90F230268134063
:103C2000042B07D1FFF70CFA21000A2207F050FEFF
:103C30000400EEE70D20FDF797F9EAE70868F8B50C
:103C4000C3071AD5FFF7E0FF0300203B5E2B23D804
:103C50000520012258430023104E451DA84217D0CD
:103C600005211024375C3C4200D09B1801395200DA
:103C700064100029F7D10130F0E704280CD90F2295
:103C800003681A40042A07D11B0905D00079DBE735
:103C900001205B001843F8BD0120FCE703CC0000C5
:103CA00070B508680D00FFF7AFFF04006868FFF704
:103CB000ABFF621E0100042A14D8451E042D11D842
:103CC00005236B439B18012215009D402B000648DD
:103CD00005682B430360054B1B68002B02D02000B6
:103CE00002F087FA002070BDF40F0020D41A0020E3
:103CF00070B508680D00FFF787FF04006868FFF7DC
:103D000083FF621E0100042A13D8451E042D10D81B
:103D100005236B439B1801229A400748036893438D
:103D20000360064B1B68002B03D00022200002F02A
:103D300060FA002070BDC046F40F0020D41A0020A5
:103D4000F0B5050089B008680C00FFF75DFF06902C
:103D5000022D36DD6068FFF757FF0190A068FFF77E
:103D600053FF04000127231D661E0793731C029353
:103D7000079B9E4235D0052373430593019B019D0C
:103D800005330493049BAB421ED0042E16D86B1E41
:103D9000042B13D80122059B2349013B5B199A4050
:103DA0009446224A0B681068069A3A4003920DD056
:103DB00062461A430A60012200280DD17F000135B6
:103DC000E0E701240194CDE7029ECFE762469343EA
:103DD0000B600028F2D0039A0299280002F009FA39
:103DE000ECE7019B1E1D042E1AD8012C18D10025CA
:103DF00005273B0021006B439B1999400B000A4AA1
:103E0000013511689943094B11601B68002B05D0DF
:103E1000019B0022581D290002F0EBF9052DE8D185
:103E2000002009B0F0BDC046F40F0020D41A0020D5
:103E3000086810B5C30703D5FFF7E6FE054B186009
:103E4000054B1B68002B03D0024B186802F0D2F917
:103E5000002010BDF40F0020D41A00207FB5A04C24
:103E60002368002B0AD19F4A1268002A06D19E4B74
:103E70001B68002B01D0FFF793FD7FBD9B4D2A6887
:103E8000002A26D1984A1268002A1BD0FFF788FD25
:103E90000028F2D0FFF770FD924B24681A681C606E
:103EA000002A16D0002C14D101AD0C229049280014
:103EB00007F0A0F8285D00210134FEF73BFE0C2C32
:103EC000F8D1DAE7874A1268002AE5D1002BE3D05F
:103ED000E0E700211A2003F09FFA00211B2003F0E5
:103EE0009BFA00211C2003F097FA2E68012E5CD06B
:103EF000022E00D1A2E0002E50D101363100794CC3
:103F000003202368994303F087FA042021680140C5
:103F10004B42594103F080FA102123680A201940CE
:103F20004B42594103F078FA802123680901194076
:103F30004B425941062003F06FFA802123680902A1
:103F400019404B425941072003F066FA802123684B
:103F5000490219404B425941092003F05DFA802182
:103F60002368890219404B425941192003F054FA41
:103F700080212368C90219404B425941182003F09F
:103F80004BFA802321681B0319404B4259411720EB
:103F900003F042FA31001A2003F03EFA2B680321A5
:103FA000581C04F0E5FF296067E702214D4C1720FB
:103FB000236819404B42594103F02EFA0821236827
:103FC000182019404B42594103F026FA80212368FA
:103FD000C90019404B425941042003F01DFA8021C9
:103FE0002368490119404B4259410A2003F014FA51
:103FF00080212368C90119404B425941032003F035
:104000000BFA80212368890319404B42594109204A
:1040100003F002FA802321681B0419404B425941E6
:10402000192003F0F9F93100062003F0F5F9310009
:10403000072003F0F1F931001B20ADE72021294CC6
:104040001720236819404B42594103F0E5F94021FC
:104050002368182019404B42594103F0DDF98021B3
:104060002368192019404B42594103F0D5F98021AA
:104070002368490019404B425941092003F0CCF90B
:1040800080212368890019404B425941072003F0E1
:10409000C3F980212368890119404B425941062008
:1040A00003F0BAF980212368490319404B42594172
:1040B0000A2003F0B1F980212368C90319404B425B
:1040C0005941032003F0A8F9802321685B041940BB
:1040D0004B425941042003F09FF901211C205BE76A
:1040E000F40F0020E80F0020F80F0020DC0F002064
:1040F000F7CB0000012010B54042FFF7E5FC10BDF2
:1041000010B5034A0921034800F094FF10BDC046D2
:10411000E0CE000028CF000030B502248025094BF6
:10412000094AED009C505C59002CFCD0A124E4000D
:10413000884202D30021995030BD8025ED001851EE
:104140004019F5E700E001400405000010B5002823
:1041500006D1C020B02140028902FFF7DDFF10BD6B
:10416000B02080218002C902F7E700004342584195
:10417000064B40421840B0239B02C0180368002041
:104180001A0E532A01D11B02180A704700C0FEFF05
:1041900030B501248025054B054AED009C505C5943
:1041A000002CFCD001600021995030BD00E001409E
:1041B0000405000043425841074B40421840B023D9
:1041C0009B02C018A62310B50902DB05090A194392
:1041D000FFF7DEFF10BDC04600C0FEFF70B5012432
:1041E00080250D4B0D4EED009C515C59002CFCD0F0
:1041F000002902DC00229A5170BD557814782D02F6
:1042000025439478013924042543D47804322406C4
:104210002C4310C0ECE7C04600E00140040500005C
:1042200070B505004B680A009C1C2100A400FFF734
:10423000D5FF281970BD0000134B1B68002B0CD054
:104240008022B023D2029B0200280BD11A1D5B688A
:104250001B0E522B00D110007047B022C0239202D7
:104260005B02F1E782420DD903681B0E522B09D184
:10427000436802339B00C018824203D903681B0EB7
:10428000522BE9D00020E7E7FC100020F0B5002019
:10429000B7B00024FFF7D0FF270005002600002D4F
:1042A0002ED1284D2868FFF761FF32003B000190B6
:1042B0000094254904A807F0FDF904A801F0DAF8F4
:1042C000224B64201C682B68A0215A425341204A8B
:1042D0005B421340B02292029B18E41A60434902E9
:1042E00004F060FDA022520203000092194922004E
:1042F00004A807F0DFF904A801F0BCF837B0F0BD5E
:10430000FF226B6829689C460233FF180B120136A6
:1043100013409C4200DA1C00FF200A140240039262
:104320006246014001920091039A0B4904A807F0EC
:10433000C1F904A801F09EF82800FFF77DFF0500F1
:10434000ADE7C046FC10002032D000000011002074
:1043500000C0FEFFDCCF00001ED0000070B50020C2
:10436000FFF704FF04000120FFF700FF844200DA9A
:1043700004000A4B1D686A42554128001D60FFF782
:10438000E5FEA0226B4252021340054A28009B180A
:10439000044A611C1360FFF70DFF70BDFC10002084
:1043A0000480010000110020F8B50020FFF7DEFEB8
:1043B00007000120FFF7DAFE3E00204D0643204CA7
:1043C0000DD18021C020C9024002FFF7A5FE0121C6
:1043D0003000FFF7EFFE1B4B2E6023601DE087428D
:1043E00009DD0023B0212B60164B8902236023686E
:1043F0000020012517E0012380212B60124BC90208
:104400002360F4E7120E522A08D0002800D023605F
:104410000E4801F02FF8FFF7A1FFF8BD28005A68F9
:10442000023292009B188B4205D21A68561CE9D1C1
:104430000028F2D0D1E72160EFE7C046FC10002051
:10444000001100200480010004C00200F7CF00002A
:1044500070B50020FFF7F0FEFF260500002801D10F
:10446000280070BD03681C143440FFF7E5FEDA2C09
:10447000F4D10500F2E700008022F0B55200A1B0AF
:104480000021674806F0D2FD8022002152006548D5
:1044900006F0CCFD644BFF271B681A0004935342BF
:1044A0005A4110000592FFF751FE049C0020631E44
:1044B0009C415E4B64421C405D4BE418FFF7C8FF13
:1044C0000600002E2DD10498FFF750FE411C0598E0
:1044D000FFF770FE059A574D534B2C601A60FEF79C
:1044E00039FD514B64201B68A0215A4253414F4A69
:1044F0005B421340B0222C6892029B18E41A60437E
:10450000490204F04FFCA0225202030000924A49E3
:10451000220007A807F0CEF807A800F0ABFF21B0F3
:10452000F0BD3268131412123A403B4003921A0055
:104530000A3A092A49D83A4B039A995C002931D1A1
:1045400010223E4806F072FD35002B6803991A12BE
:104550003A40914209D11A143A400B2A27D0132A23
:104560002DD00A2A01D1354B1D602800FFF764FECB
:10457000051EEAD1314B196800290FD02000FFF742
:104580004FFE04002D4B5B195968002903D0200011
:10459000FFF746FE040004350C2DF3D1204B01211A
:1045A000039A99543000FFF747FE060089E73B4025
:1045B000022BDADC214A9B00D3185D60D5E710227C
:1045C00000211E4806F032FDCFE71A00153A082AEE
:1045D000E8D8144A0399525C002AE3D13500152B20
:1045E00000D01500300003681A143A40152A0FD085
:1045F0001D2A00D10025FFF71FFE0028F3D1002D52
:1046000004D020002900FFF70BFE0400054BC6E78D
:10461000039A1B123B409A42EDD10500EBE7C046DE
:10462000FC0F002004110020FC10002000C0FEFF41
:1046300004C0020000110020C1CF0000102F002094
:1046400010B5FFF719FF10BDF0B585B00392032236
:104650000333DC17294D1440E4182B68284F5A42C5
:10466000534180225B42D202A4103B409B18A21C03
:104670000291244E910000910190316800980A182F
:10468000934215D2FFF7F8FE2B685A42534180221D
:104690005B421F40D202BF183368009A9B189F42AA
:1046A00006D2194800F0E6FE0025280005B0F0BD4E
:1046B000029B356819066B461A7BA423DB0513435E
:1046C000FF222F00090C1943019B12041B04134005
:1046D00019432800FFF75CFD0837281D21003760CB
:1046E000FFF756FD002C04D00A9A21003800FFF78E
:1046F00075FD009B083BFF183760D6E7FC100020D3
:1047000000C0FEFF001100209BCF000070B59AB0E2
:10471000FFF74AFEFF221E4CD2000021200006F0C7
:1047200085FCFF25FFF794FE0026002814D1020027
:10473000C300E3580130591E8B41D218FF28F7D12E
:10474000144901A806F0B6FF01A800F093FE124834
:1047500000F090FE1AB070BD03681A142A400A2AAD
:104760000AD11A122A40FF2A03D0D200A1180B71D5
:10477000A050FFF761FDD8E7132AFAD11B122B4096
:10478000FF2BF6D0DB00E2181671E650F1E7C046C9
:104790008825002067D000007BD000000021094B55
:1047A000094A59600131516059680029FCD0002143
:1047B0001961012393600222044B8131FF315A5069
:1047C0001A607047FC1000400010004000E100E05B
:1047D0000222064B0121DA670022054B5A61054A85
:1047E00011615A69002AFCD07047C04604E100E01C
:1047F000FC1000400010004010B5044C2378002B42
:1048000001D0FFF7E5FF0020207010BD0512002049
:10481000802301205B055B6E5B001843704700003E
:104820000120024B1B685B00184370478812002070
:104830000120024B1B685B001843704724000020D6
:104840000120024B1B685B00184370478C1200204C
:1048500070B504000D001600FEF75EF980230121FB
:104860005B055A6E2670002653006170E17062721B
:10487000010A5A0A6071A171A272010C5A0C000E51
:104880005B0EA6702571E1712072E272237370BD18
:1048900010B5044C200006F053FF01002000FEF785
:1048A000DDFD10BD911200200E4B10B51B680E4CA3
:1048B0005A1C0FD00D4C002B0CD00D4C012B09D0E5
:1048C0000C4C022B06D0094C042B03D00A4C052BB0
:1048D00000D1074C200006F033FF01002000FEF756
:1048E000BDFD10BD280000200CD1000069C90000EA
:1048F00017D1000070C9000011D1000070B5214C23
:104900002278002A3DD1204B01215A608022D20515
:1049100011605A68002AFCD0002207201B4B1C495A
:1049200001255A500439585008315A5019481A492B
:1049300058501A491A485A501A495A50A622D200B9
:104940009D50082218495A500431585002201749E6
:1049500058501749174858501748043958501820CC
:1049600016495850C12189005A500539FF39585805
:10497000921802435A501249124A9950FFF70EFFFB
:10498000257070BD05120020FC00004000100040A2
:104990000C050000746962751C0500002405000008
:1049A000200004022C05000014050000340500005E
:1049B0003C050000FFFF000021100100540500002D
:1049C000061200200405000070B50E4B06001B788F
:1049D000002B01D1FFF792FF00200B4D2C78844271
:1049E0000ED00A4B202219780323091B1940084BCB
:1049F0004901C918300006F0FDFA0120013C2C7075
:104A000070BDC04605120020901200200412002044
:104A100006120020002370B588B0984235DD0D687D
:104A200001262C0034409C422FD12300042D2CD988
:104A30000F222B681A402300092A26D16A683F2AD0
:104A400023DD6846FFF7C0FF230000281DD06B461A
:104A500019783300A14203DB6B461B5D5B003343D7
:104A6000A200AA1801349360202CF2D109216944D4
:104A70004A780B7812021A438B781B041A43CB78BE
:104A80001B061343024A13600423180008B070BDCC
:104A90008C12002070B5454B8AB01B78002B01D1D9
:104AA000FFF72CFF02AC2000FFF78EFF002802D199
:104AB00000200AB070BD23780B2BF9D96378012B45
:104AC000F6D1E378012BF3D100231120384E394D74
:104AD00033602B7068442379374A41781360027839
:104AE00009021143827812041143C27812060A4364
:104AF00032490A60002B0ED1152169444A780B789F
:104B000012021A438B781B041A43CB781B061343FB
:104B10003360002318E0012B1AD1152169444A782B
:104B20000B7812021A438B781B041A43CB781A2194
:104B30001B06134333600E23627C6944934200DDFD
:104B4000130000229A422CD100220420EA54B0E73C
:104B5000022B03D1627B10331621EEE7042B0DD11B
:104B6000152108226944684606F044FA0098019924
:104B700002F0C4FC06F0F0F83060CAE7052BC8D19B
:104B8000152108226944684606F034FA0098019914
:104B900002F0B4FC06F0E0F83060627D0A231E21CA
:104BA000CBE7885CA8540132CCE7C0460512002050
:104BB0008812002091120020280000208C12002072
:104BC00010B5134B04001B78002B01D1FFF796FEA4
:104BD000FFF7FEFD00200F4A0F49104B545058605C
:104BE0000130106058680028FCD0002018610130A6
:104BF000906018690028FCD0094B0A481B785B01BB
:104C00001B185350FFF7E4FDFFF7C8FD10BDC04669
:104C1000051200200010004004050000FC100040B8
:104C2000041200200612002010B588B000281DDDF7
:104C30000A68012113000B4018D1042A16D90F204D
:104C400014682040092811D150683F280EDD9800D3
:104C5000101880680024084201D04010C4B2684691
:104C6000C4540133202BF2D1FFF7AAFF002008B073
:104C700010BD000010B5002813DD0C68E30710D547
:104C80006410532C0DD8084B1B78002B01D1FFF773
:104C900035FEFFF79DFDA123044ADB00D450FFF74A
:104CA0007DFD002010BDC046051200200010004010
:104CB00010B500280EDD0C68E3070BD56410FF2C3F
:104CC00008D8054B1B78002B01D1FFF717FE034ACC
:104CD000034BD450002010BD0512002000100040EE
:104CE0002405000013B5002814DD0C68E30711D576
:104CF000094B64100093094B0193072C0AD8084B09
:104D00001B78002B01D1FFF7F9FD6B46054A1957B7
:104D1000054BD150002016BDE2ECF0F4F8FC000485
:104D200005120020001000400C05000070B588B08E
:104D3000002820DD0124086804401CD104281AD969
:104D40000F2302681340042B15D1FEF779F90600F2
:104D500006F0F6FC0500122800D912252A000221CF
:104D60000D326846FFF774FD6B465D73A54205DCA6
:104D70006846FFF725FF002008B070BD2300325DB4
:104D80006B449A730134F1E7F0B50D008BB0012844
:104D900032DD08680122040014402DD104282BD9EB
:104DA0000F2301680B40042B26D16B68134223D0DC
:104DB000FEF746F96E6807007310019306F0C0FC19
:104DC00005000E2800D90E252A000121113202A863
:104DD000FFF73EFD6A46127902AB5A7302AA7312BC
:104DE0009373019B76141B0ED67313745574A542EE
:104DF00005DC02A8FFF7E4FE00200BB0F0BD3A5D31
:104E000002A963189A740134F1E730B589B000281B
:104E100014DD0C68E30711D5102268460021FFF766
:104E200017FD6B466A4665105D73684663122D0E6A
:104E300064149373D4731574FFF7C2FE002009B095
:104E400030BD0000174B184A5968002903D00021D3
:104E5000596001319160196900291FD00020186143
:104E60008023DB00D3581149012B18D1A923DB0083
:104E7000D3585B420B600E490B78032B01D80133EA
:104E80000B7003200B490B78013303400B700A4968
:104E90005B015B1809495350012393607047086018
:104EA000FAE7C046FC10004000100040240000203B
:104EB00090120020041200200612002004050000B9
:104EC00010B5034A1021034800F0B4F810BDC046E5
:104ED0008CD0000083D00000044A05491368C854F0
:104EE00001339B059B0D13607047C046C016002020
:104EF000C012002070B5114C114A2368834202DCB5
:104F00000023236016E0155C411C2E00FA3E012EA2
:104F100005D899420FDA555C013D1F2D01D90800D3
:104F2000ECE70100151A565C6E5401318B42FADC35
:104F3000181A206070BD1570FAE7C046CC1A002020
:104F4000CC16002010B5FDF7DDFD064B1A68824235
:104F500001D900221A601B68C31A03489842804195
:104F6000404210BDBC120020204E000010B5094C7C
:104F7000094A23681268934200D110BD074AD05CE9
:104F8000FDF7E0FF0028F8D0236801339B059B0D57
:104F90002360ECE7C4160020C0160020C0120020D9
:104FA00010B50400064B074A1B6812689B1ADB43C6
:104FB0009B059B0DA34200DB10BDFFF7D7FFF1E778
:104FC000C0160020C4160020F7B5050056680191F0
:104FD000B000441C06301700FFF7E2FFFB20FFF78C
:104FE0007BFF1C20FFF778FFE8B2FFF775FFE0B208
:104FF0002412FFF771FFE0B2FFF76EFF6B461879DE
:10500000FFF76AFF0025AE4200DCF7BDAB00FB18DE
:105010009C680135E0B2FFF75FFF2012C0B2FFF7D6
:105020005BFF2014C0B2FFF757FF200EFFF754FFBD
:10503000E9E7000070B5074E3368092B08DC0C2542
:105040005D43054C0133285164196160A2603360EF
:1050500070BDC046C8160020202F0020F0B587B0D4
:1050600002900C00012803DC1B20FBF77DFF45E0CC
:10507000244B08680093C30709D4042807D90F23D9
:1050800002681340042B02D1FDF7DAFF00901D4B9C
:1050900060680193C30709D4042807D90F23026865
:1050A0001340042B02D1FDF7CBFF01900027164BD4
:1050B0001B680493049BBB42D6DD0C267E43134B36
:1050C0000099F618306806F031FB051E05D17368AB
:1050D000B6680593059B9D4201DB0137EAE730681E
:1050E0000199039606F022FB0836002808D121001A
:1050F0000298039B083102385B68984707B0F0BDFF
:105100000135E7E733CA0000C8160020202F002031
:1051100010B5FBF765FEFEF7F3FFFDF7B5FEFEF7F2
:1051200089FBFEF7D7FBFFF7CBFE00F07FFE01F017
:1051300063F801F0ADFA10BD962210B512010021FE
:10514000034805F073FF0022024B1A6010BDC046F1
:10515000281C0020CC050020064B074A1B6812685B
:105160009B1ADB439B059B0D0122834200DC00223E
:1051700010007047C0160020C4160020F8B50500C6
:105180000C0016001F1E0ED10320FFF7E5FF0028BC
:1051900008D0FA20FFF7A0FEE8B2FFF79DFEE0B2CC
:1051A000FFF79AFEF8BD501DFFF7D6FF0028F9D093
:1051B000FB20FFF791FEE8B2FFF78EFEE0B2FFF7AB
:1051C0008BFEF0B2FFF788FE3012C0B2FFF784FE0C
:1051D0003C00E31B9E42E5DD2078FFF77DFE0134B5
:1051E000F7E7000070B50024F0250B4B1B68A342C5
:1051F00002DCFFF7A1FF70BD2B006343074A9B1839
:105200001A78002A05D05978002311201A00FFF7D8
:10521000B5FF0134E9E7C046CC050020281C00207A
:10522000F8B507000024F0252B0063430C4A013435
:105230009E18B74211D0317800290BD00133D15CD0
:10524000002311201A00FFF799FF2A0000213000E7
:1052500005F0ECFE0A2CE7D1F8BD024B1C60F9E723
:10526000281C0020CC050020F0B5150001222F00DD
:105270005E4C1740A54401900291002F11D005AB60
:105280001A706A105A70120E1A71052269129970FA
:105290006D140299DD70FFF771FFCF239B009D44D1
:1052A000F0BD042D1ED90F232A681340042B25D1ED
:1052B000023B04AA28001371FDF7C2FE040006F0A9
:1052C0003FFA4B4B984200D91800B84204DC421C0C
:1052D00005AB02990198DEE701377B1EE35C05AA66
:1052E000D355F2E7042D7CD1032304AA043D1371A6
:1052F0006B425D4105AB55710222EAE7092BCCD127
:10530000042205AB1A706A68511000916946521266
:1053100009789A70009A59701F2A01DD20220092A4
:105320006A46127806ACDA70009BBB4202DC05AB21
:10533000E21ACEE70126BB00EB189868064006D1BA
:10534000042837D90F2302681340022B0CD1012304
:1053500023704310637042121B0E4014A270E07061
:10536000237105340137DFE7042B21D1023B237081
:10537000FDF766FE039006F0E3F9A31C0C2809D89C
:105380006070864201D19C19ECE7039A925D9A55B0
:105390000136F6E70C226270039A925D9A55013647
:1053A000092EF9D12E23E372237363730E34D9E7E8
:1053B000012B07D103230438237043425841607006
:1053C0000234CFE7092B09D1053B23704368E6700F
:1053D0005A105B126270A3700434C3E72670013464
:1053E000C0E7002D00D058E77EE7C046C4FCFFFFB1
:1053F0002303000070B502000024F0210D4E0800C8
:10540000604380194578954203D001340A2CF6D1C7
:1054100070BDF022002105F009FE074A1368013B28
:10542000A34200D11460002329001A001120FFF7C5
:10543000A5FEEDE7281C0020CC05002010B5B2B079
:1054400002236A460400137006F07AF9C72800D9CF
:10545000C7200023984207DC421C6B46FE21142023
:10546000FFF78CFE32B010BD694601335A1EA25CB4
:10547000CA54EFE730B5B3B002236A460500137093
:1054800006F05EF90400C72800D9C72400239C4217
:105490000BDC20003230FFF783FD621C6B46FF21DE
:1054A0001420FFF76BFE33B030BD694601335A1E3E
:1054B000AA5CCA54EBE70000F7B5234B06001B6853
:1054C000F02100930023009A9A4211DC0024F0237B
:1054D0001A006243019201991C4A55182F78002F37
:1054E00012D001340A2CF3D11948FFF7C3FF29E089
:1054F0000A005A43154882185078B04202D11278F7
:10550000002A1FD10133DEE7F0223900280005F020
:105510008DFD02230D4A0199EB6053540D4AF100B1
:105520008A58009B6E70AE70AA602F616F61A342B3
:1055300002DC054B01341C60002331001A001020EE
:10554000FFF71CFEF7BDC046CC050020281C00203C
:1055500015D600008825002010B5FFF743FEFF2474
:10556000084AE3005B429B18074AD35C043B012BCB
:1055700003D8E043C0B2FFF79FFF013C002CEFD1FE
:1055800010BDC046FC07000088250020F7B50F00BD
:10559000FF247F2501901E4AE300D31A1D4A9A1862
:1055A0001278062A01D0032A20D1FF22D2009B18AC
:1055B000186883682B401C2B18D1C3681A002A4036
:1055C000042A13D102692A40192A0FD11B0A013378
:1055D0009B000C30C018FDF733FD03780600002B4C
:1055E00010D006F0ADF80023B84209D0013C002CE1
:1055F000D1D1F7BD019AF15CD25C9142F6D1013371
:105600009F42F7DCE043C0B2FFF756FFEEE7C0462B
:1056100088250020FC07000070B50500FF24084A1B
:10562000E3005B429B18074AD35CAB4203D1E043E3
:10563000C0B2FFF741FF013C002CF0D170BDC04665
:10564000FC07000088250020F7B5FDF75BFA514BF9
:105650001A68824201D900221A601A684E49821AD9
:105660008A4200D883E01860FDF756FA071E00D181
:1056700001370020FDF742FB01900020FDF752FBAF
:10568000019B0090454C464D002B14D02368002B05
:1056900000D07AE02B682760002B00D171E0414BED
:1056A00001261B78002B63D10920FFF7B5FF3E4B85
:1056B0001E703C4B1E70009B002B12D02B68002BE1
:1056C0000FD123682F60002B1ED0374B01261B788B
:1056D000002B52D10920FFF79FFF334B1E70314B37
:1056E0001E702368002B0FD02F4E3278002A0BD16A
:1056F0009F4200D227602368FB1A312B04D9072070
:10570000FFF78AFF012333702B68002B0FD0254E43
:105710003278002A0BD1BB4200D92F602B68FF1AC8
:10572000312F04D90820FFF777FF01233370236856
:10573000002B0CD0019B002B09D11B4E3378002B82
:1057400002D10720FFF768FF0023236033702B6826
:10575000002B0CD0009B002B09D1124C2378002B7E
:1057600002D10820FFF758FF00232B602370F7BDFC
:105770000720FFF751FF0C4B9CE70820FFF74CFF79
:10578000ADE7009B002B9CD1ABE7009A002A95D196
:10579000AAE7C046B81200200F270000A812002078
:1057A000B0120020B4120020AC12002037B5002443
:1057B0000500FFF717FD01A80194FDF78DFA210000
:1057C0002000FEF771F9FEF749FBFDF739FBFDF705
:1057D00053FBFEF78FFCFDF7BBF9A54204D0FDF7A4
:1057E000DBFB0248FFF746FE37BDC04606D6000089
:1057F000002310B501001A001120FFF7BFFC10BDF7
:1058000007B56B46197069465A7013128B701314E2
:10581000120ECB700A716B46010005221320FFF7B0
:10582000ADFC07BD10B50A0001001220FFF71CFDFA
:1058300010BD70B5050008000C003230FFF7B0FB5A
:105840002B00220000211B20FFF798FC70BD10B533
:105850000C000300110014202200FFF78FFC10BD84
:10586000012370B5FF24084A41185B42884201D3E6
:10587000D84370BD06781D0A234073409B009B5897
:1058800001306B40F2E7C046E8D10000002313B5B9
:1058900001930B4BC2000400D058002805D0436888
:1058A00008309900FFF7DCFF01900920FFF778FB33
:1058B00001AB042221001720FFF760FC13BDC04696
:1058C00088250020F7B50190FEF7C2FD01250400F0
:1058D000FF276D42002C01D12800FEBD266833143D
:1058E0003B40152B0DD121000198083105F01EFF1A
:1058F000002801D135123D402000FEF79DFC040038
:10590000E8E71D2BF8D101256D42F5E7F0B58027BA
:105910009DB0FFF72BFBA54CA54D2068FF00391A61
:105920004019FDF7F5FA23680600C3182360002B21
:105930000ED11DB0F0BD2068391A2818FDF7E8FA1D
:10594000236806001B182360FDF7DCF8994B1860EC
:10595000002EF0DC2B78FA2B00D037E12368022BE5
:1059600007DCFFF7EFFA0028E3D00120FFF7C2FAC7
:10597000DFE76878AC78023818282BD803F07EF976
:1059800019002C0030003400370040002A004A0083
:105990007C0086008A00A000F10002012A002A0093
:1059A0002A002A002A002A002A002A002A002A00A7
:1059B0001001FF2C0ED02000FFF71CFD00227E4BB3
:1059C000E100CA505B181A712100009213001320E5
:1059D000FEF73AFE0320C9E72000FFF76DFDF9E767
:1059E0002000FFF707FDF5E7FFF7B6FDF2E7FFF749
:1059F000F9FB0020FFF7DAFE7048FFF73BFDE9E70F
:105A0000632CE7D86E4BA200D25821001520FFF777
:105A10002BFCDFE7FEF71CFDFF270400002CD9D08C
:105A200025682B143B40152B04D02000FEF704FC06
:105A30000400F3E72000083005F082FE0600053080
:105A4000FFF7AEFAFB20FFF747FA2D121D20FFF7F4
:105A500043FAE8B2FFF740FAF0B2FFF73DFA30122E
:105A6000C0B2FFF739FA25002B1B9E42DDDD287AF4
:105A7000FFF732FA0135F7E700211D2000910B00F6
:105A80000A00FEF7E1FDFDF787FAA3E72000FFF724
:105A9000FDFE9FE7FDF748F803AC4A4A64210090F9
:105AA000494B200005F0D4FD02232000237005F0AF
:105AB00047FE2300020000211620FFF75FFB89E765
:105AC00000243D4AE300D558002D27D06B689E0086
:105AD000701DFFF765FA2B00002532000833210006
:105AE0000120FFF74BFB2F00FEF7B2FC2E00002831
:105AF00018D1002F04D03A0001212000FFF764FAEA
:105B0000002D04D02A0002212000FFF75DFA002EAC
:105B100004D0320000212000FFF756FA0134FF2C98
:105B2000CFD157E7FF2103681A120A40A24209D1D8
:105B30001A140A400B2A08D10B400CD0012B0CD0B0
:105B4000022B0CD0FEF778FBD1E7132AFAD10025FF
:105B50002F002E00F6E70600F4E70700F2E7050045
:105B6000F0E70024FFF73EFB220021000094230011
:105B7000DA20FEF769FDFF222100D2000E4805F071
:105B800055FA80E7012C02D1FEF780FB22E7022CB8
:105B900002D1FEF755FD1DE70120FFF707FE19E7CB
:105BA000002321001A001A2087E7C046CC1A0020E3
:105BB000CC160020BC12002088250020E8D500006B
:105BC000802D0020FFD50000FAD50000FB2B00D06F
:105BD000CBE62268042A00DCC3E62E79E878574B2E
:105BE000360206439E4200DDBFE6331D9A4200DCCA
:105BF000B7E6EB5CFE2B00D0B7E66B78AC78771E8F
:105C00001B2B61D019D8072B47D0082B1CD0012B98
:105C100018D1FF2C16D02000FFF7ECFB6D79484A15
:105C2000B31E009221002A000A20FEF70DFD454B0D
:105C3000E400E0501B191D7104E01D2B56D048D321
:105C40001E2B6AD0701D91E6632CFBD86A79022A5C
:105C500013D0032A1BD0012AF4D1E979AB790902C8
:105C600019432B7AA4001B0419436B7A1B060B43C0
:105C70005B001343344AA350E4E7002FE2DDB11E7A
:105C80002F48FDF7EBFB304BA400E050DAE7AB798F
:105C9000A4005A1E93419B00ECE7632FD2DC03ADB6
:105CA0003A002A49280005F0A5F900232800EB5501
:105CB000FFF708FE0028C5DB234B8000C2582100F7
:105CC0001520FFF7D1FABDE739002048FFF75EFC49
:105CD000B8E7FF2CB6D06A79022AB3D818490B204E
:105CE00000912100B31EFEF7AFFCABE7632F00DD90
:105CF0006327002303A99F420ADCFB430022DB1732
:105D00003B40CB181A70152000917B1C2100EAE75C
:105D1000EA185279CA540133EDE7012C92D1002FD1
:105D200090DD6B79002B03D01C00322B00DD322478
:105D300064235C43064B1C6084E7C046F603000006
:105D4000D216002088250020802D0020D1160020AA
:105D5000040000200122094B1A60094A1368002B35
:105D6000FCD00322074B1B68D8171040C018012332
:105D700080100638400018437047C04600C00040FD
:105D800000C1004008C500400120704710B5064C16
:105D9000200000F0B3FD0549200000F0D7FD0122EE
:105DA000034B1A6010BDC046F81A0020801A060086
:105DB000D01A002010B501210D20FCF7BBFE0121F7
:105DC0000E20FCF7B7FE00210F20FCF7B3FE044CB9
:105DD000200000F0CFFC1021200000F0E7FC10BDF7
:105DE000D81A002010B504680D20E30703D564100D
:105DF000FF2C03D91720FBF7B7F810BDFFF7DAFF28
:105E0000E1B2024800F0F4FC0020F6E7D81A0020C6
:105E100010B5FFF7CFFF0021034800F0E9FC430075
:105E20000120184310BDC046D81A002010B5034AFF
:105E300008210348FFF7FEF810BDC0462CD600002D
:105E40006CD600000D4B70B51B6804000E001500E9
:105E5000002B01D1FFF79AFFE1B2094C200000F0BE
:105E60000CFEF1B2200000F00FFDE9B2200000F0BE
:105E70000BFD200000F06CFE70BDC046D01A002063
:105E8000F81A002010B501240368234205D04168A8
:105E9000214202D08268224203D10D20FBF764F830
:105EA00010BD5810802801D91520F7E74910FF29A7
:105EB00001D91620F2E75210FF2A01D91720EDE789
:105EC000FFF7C0FF0020EBE7F7B501221400904276
:105ED00022DD0D682A421FD01D4B15411B684C68FE
:105EE000002B01D1FFF752FFE9B201272500194E1F
:105EF0003D40300000F0C1FD002D0FD03C4130008E
:105F0000E1B200F0C1FC300000F022FE0024A0420B
:105F100002D02320FBF728F82000FEBD042CF2D984
:105F20000F2322681340092BEDD163685B100193A6
:105F3000019BAB42E7DDAB00E3189968394204D01E
:105F40004910C9B2300000F09FFC0135F0E7C046AF
:105F5000D01A0020F81A0020144B70B51B680500F9
:105F60000E00002B01D1FFF711FF114CEDB22900FB
:105F7000200000F082FDF1B2200000F085FC00213D
:105F8000200000F085FD002801D0404270BD0122B4
:105F90002900200000F06CFD200000F066FC0028C5
:105FA000FAD0200000F066FCF0E7C046D01A0020CE
:105FB000F81A002010B501240368234202D041687A
:105FC000214203D10D20FAF7CFFF10BD58108028D1
:105FD00001D91520F7E74910FF2901D91620F2E76A
:105FE000FFF7BAFF40002043EFE70000002370B541
:105FF000344D0400EB5601330BD10D211D20FFF76A
:10600000ABFF5A2814D101222A212A703D38FFF70C
:1060100019FF0023EB56022B2AD0032B49D0012B6A
:106020004CD121001D200124FFF796FF644225E09A
:106030000F211920FFF790FF332805D102235F229B
:106040002B7020211A38E2E70D211E20FFF784FF74
:10605000C7280AD1032300222A21A9382B70FFF771
:10606000F1FE1B222A211E20D1E700232B70D0E74E
:10607000012C13D129211920FFF76EFF7F2801DDA4
:106080000138FF3803007F3301DA7F204042642368
:106090007F21584302F086FE604370BD032C0BD174
:1060A0002B211920FFF758FF043CE7E72D21192089
:1060B000B9E721001E20B6E7052CF7D00124002007
:1060C0006442E4E72C00002070B50120FFF78EFF4A
:1060D00004000320FFF78AFF05000520FFF786FF75
:1060E0006D43644340436419201804F06BFE01F0D3
:1060F00035FB04F031FE43000120184370BD10B59C
:106100000120FFF773FF43000120184310BD10B5B5
:106110000320FFF76BFF43000120184310BD10B5AB
:106120000520FFF763FF43000120184310BD000066
:10613000F8B501231C00984229DD0F683B4226D0A8
:106140004E6835001D4022D1042E20D90F2231681F
:106150000A40092A1BD173685C10202C00DD202422
:10616000134B1B68002B01D1FFF710FE7F10F9B213
:10617000104F2200380000F07BFCA54214DA3800F2
:1061800000F073FB002804D101246D002C43200093
:10619000F8BD380000F06EFB0122AB004000F318A0
:1061A00010439860AD18E8E764000125EEE7C046AB
:1061B000D01A0020F81A00200020704701207047F4
:1061C0000020704700207047012070470020704772
:1061D0000020704700207047002070470020704763
:1061E0000020704700207047002070470020704753
:1061F000704770477047000010B5034A0E210348EE
:10620000FEF718FF10BDC046BCD600002CD700001A
:106210000378013B1F2B00D970470130F8E710B518
:10622000FFF7F6FF0378002B0BD00130222B11D1A2
:106230000378002B03D0421C222B03D11000FFF760
:10624000E7FF10BD5C2B03D14378002B00D0821CEC
:106250001000EDE73A2BF2D02C2BF0D07B2B0BD19A
:10626000FFF7D6FF0378002BE9D07D2B01D1013059
:10627000E5E7FFF7D4FFF5E720225B2B14D1FFF70A
:10628000C7FF0378002BDAD05D2BF0D0FFF7C7FFF4
:10629000F7E7202BD3DD2C2BD3D0190091435D29B8
:1062A000CFD0222BCDD001300378002BF1D1C6E71F
:1062B000002210B5904216D0FFF7AAFF03780422FF
:1062C000222B10D0023A7B2B0DD0013A5B2B0AD047
:1062D000190030390232092905D92D2B05D1417811
:1062E000303909290AD8100010BD0522742BFAD0C4
:1062F0000132662BF7D001326E2BF4D0581E834149
:106300005A42F0E770B5FFF783FF037801222D2B87
:1063100001D18018023A00230A2502E06B430130C4
:10632000CB1801783039CCB2092CF7D95A43100078
:1063300070BDF8B50C001500FFF76AFF0378222B3B
:1063400002D000232370F8BD0D236A1E210008250A
:106350000C260A279C4601300378222B02D1002309
:106360000B70F0E7002BFAD0441C5C2B0BD1437868
:10637000841C622B0ED0662B0ED06E2B0ED0722B8F
:106380000ED0742B0ED0002AE9DD0B70013A0131DA
:106390002000E1E72B00F6E73300F4E73B00F2E7EB
:1063A0006346F0E70923EEE710B50400FFF737FF77
:1063B000A04202D90378202B00D910BD0138F7E79D
:1063C00010B5002815D00378002B13D0FFF720FF5D
:1063D0002021037802008B4300205D2B09D01000A0
:1063E000FFF71DFF03782C3B5A425341C018FFF7BB
:1063F0000FFF10BD1800FCE70300002070B50C0073
:1064000081420EDD1A785B2A0BD1581CFFF700FF82
:106410000125AC4205D0FFF7D3FF002801D001359C
:10642000F7E770BD70B50C001500002901D00023FE
:106430000B70002820D00378002B1ED0FFF7E8FE59
:10644000037806002C2B03D10130FFF7E1FE060094
:10645000337800207D2B0FD0844204D02A00210005
:106460003000FFF766FF3000FFF7D9FE03783A2BC4
:1064700002D10130FFF7CCFE70BD1800FCE7F0B58B
:106480000D0004009DB02E78002E35D02E2128005E
:1064900005F03EF9071E14D0431B0193303E092E30
:1064A00014D82800FFF72EFF01002000FFF7A4FFFB
:1064B0000400002C20D0002F1ED0019B0133ED18CA
:1064C000E1E7280005F03CF90190E7E723787B2B12
:1064D00011D1601C642203A9FFF7A4FF041E0BD096
:1064E000019A290003A805F032F90028E1D0200024
:1064F000FFF795FEEEE7002420001DB0F0BD70B55B
:10650000050000200C0081421DDD2800FFF7D0FEB1
:106510000300681C012B14D00020022B13D1002291
:10652000681C1100FFF77EFF012C0CD0FFF748FF1D
:1065300000221100FFF776FF013CF5E7FFF740FF6F
:10654000013C012CFAD170BDF8B5050000200C000B
:1065500016001F0081420DDD2800FFF7A9FE030091
:106560000020022B06D1681C3A003100FFF75AFFC9
:10657000012C00D1F8BDFFF723FF3A003100FFF7EF
:1065800051FF013CF4E710B50024A04218D0FFF7FA
:106590003FFE03787B2B0AD1013000221100FFF768
:1065A00041FF00280CD0FFF73AFE0134F5E75B2BE2
:1065B00006D10130FFF704FF002801D00134F9E7CC
:1065C000200010BDF8B5002816DD0D68EB0713D5C7
:1065D0006D10013D0124FDF73BFF0026FF276442BB
:1065E00000280CD1002E21D0300005F0A9F80100C0
:1065F0003000FCF733FFF8BD01256D42EAE7036880
:106600001A143A40152A0BD11B123B409C4200DA67
:106610001C009D4201D106000836FDF70DFEDFE7A4
:106620001D2AFAD1012400266442F6E70120013434
:1066300064002043DFE7000010B508680C00FCF799
:10664000FFFCFFF73FF9002803DB6268024B800084
:10665000C250002010BDC046802D002010B5086833
:10666000FCF7EEFCFFF72EF90123002802DB024BBA
:106670008000C358180010BD802D002010B5086898
:10668000FCF7DEFCFFF71EF9C043C00F800010BD11
:1066900010B5034A04210348FEF7CCFC10BDC046E8
:1066A000BCD70000B5D7000010B5FCF7F9FBFCF72C
:1066B00099FCFEF72DFD0448FEF7DCFEFEF726F8F8
:1066C000FEF74AFF10BDC0460BD8000010B5FCF71E
:1066D000F5F810BD70B5002504AC24780573A94207
:1066E00005D10A4B0A4A23210A4804F015FC01602F
:1066F0000949920052589B0002715B58A4008371B3
:106700006358856043710223C37170BD23D80000B4
:1067100088D8000031D80000E8D80000037B002BA7
:1067200004D1437383730361013303737047000023
:106730001FB50191A02100240068C900D2B24450C5
:10674000012A10D0A24209D0032A0AD0074A835056
:10675000074B019AC250012343501FBD022213432D
:10676000F4E70422FBE70622F9E7C04654050000DF
:106770002405000010B50400FFF7D0FFA122236814
:10678000A179D20099506179064A20009950217967
:1067900004329950044B19685A689B68FFF7C8FF88
:1067A00010BDC0460C050000EC1A00204BB2002BB7
:1067B0000FDB80233F290FD81F290FD80F290FD8AF
:1067C00007290FD803290FD81B060168074A8B50E9
:1067D000704780239B04F8E7DB04F6E71B05F4E72A
:1067E0005B05F2E79B05F0E7DB05EEE7240500001B
:1067F0000368074A99501A00FC32D1680029FCD07E
:10680000A321C90058580023C0B2D3607047C046C6
:106810001C05000007B58022074BD2051A60002234
:106820009A6002321A710F230C3200930349023B23
:106830000348FFF74FFF07BDEC1A0020003000406F
:10684000D81A0020F8B505000E0017000024BC423D
:1068500008D02B68315D1B6828009847002801D0BC
:106860000134F4E72000F8BD704710B51C3000F08B
:10687000A9F910BD10B51C3000F096F910BD10B587
:106880001C3000F0A5F910BD70B5437E0D00002B43
:1068900001D1002070BD6430040000F0A2F900288E
:1068A000F7D12000290000F070F90120F2E7000084
:1068B000F7B50193FA23002504009B0083600D4B7C
:1068C0004560083303601C300F00160000F052F9D9
:1068D0002000643000F04EF9074A2761B600B35833
:1068E00020006375019B9B009B586576A576A37578
:1068F000FEBDC046C8D80000E8D800000123A02291
:10690000C375837D0E49C133FF33D2059B00995077
:10691000437DC133FF339B009950CC220169094B61
:106920005204CA5005220169243BCA50827D016984
:106930000833CA500269417D034BD1507047C046AD
:106940000C060000240500000C050000A022002316
:1069500010B50469D200A3500A4CA1420FD90A4CC9
:106960008C425B4109495B420B40CD21C9045B1855
:1069700004690749635005210369995010BDCC2370
:106980005B04F5E7A086010090D00300000098FDAD
:1069900024050000F7B5040000200D000193824299
:1069A00065D01600402A00D9402627001C37380041
:1069B00000F0F6F8B1232269DB00D55080220123D4
:1069C000216992008B50A27E002A03D122691362B2
:1069D000226913600025731EAB4207D1019B002B77
:1069E00004D0802202212369920099500122236958
:1069F0001A622369FC33DA68002A02D19A6A002AF3
:106A0000F9D09A6A002A0BD1DA60A3232269DB004D
:106A1000D1583800C9B2013500F0B7F8B542DAD321
:106A2000019B2269002B0FD11300FC339B6A002BC2
:106A30000AD10133A376D3612369FC33DA6C002ACF
:106A4000FCD00022DA640AE000230121A376516120
:106A50001A002369FC3399680029FCD09A602369E5
:106A6000FC339A6A002A01D000229A62E8B2FEBD85
:106A700010B50123FFF78EFF10BD0300AC3310B536
:106A800004001970643000F08BF80123637610BDA8
:106A90000023020070B5AC3243760D001178B122AC
:106AA00004000069D20081508022216992008B503D
:106AB0002269013313622269936026006436300034
:106AC00000F080F8002812D0300000F06DF81E4B66
:106AD0002269D0502369FC331A6A002A02D19A6ACB
:106AE000002AF9D09A6A002A01D11A62E5E72369DF
:106AF0000122002D0DD11900FC31896A002908D12D
:106B0000DA612369FC33DA6C002AFCD00022DA64F3
:106B100007E05A612369FC339A68002AFCD00022FE
:106B20009A6000202369FC339A6A82420BD09862F3
:106B30002169064A8B588B501800022B03D0181F6E
:106B4000431E9841033070BD1C050000C4040000C2
:106B500010B50121FFF79CFF10BD000010B51323F5
:106B6000142202490248FFF7A3FE10BD0040004076
:106B7000F81A002010B540220021040004F056FA53
:106B8000002320002364636410BD10B53F24026C11
:106B9000531C2340446C9C4201D08154036410BDBB
:106BA0000023036443647047436C026C934206D035
:106BB0003F21C25C01330B40436410007047012049
:106BC0004042FBE7036C406C181A00D54030704718
:106BD000436C026C934201D0C05C7047012040427C
:106BE000FBE73F22036C406C01331340181A434209
:106BF0005841C0B27047000003210A4802680A43A6
:106C00000260094802680A4302600849084A094BC1
:106C10009B1A03DD043BC858D050FBDC00F012F88F
:106C2000F9F772FA24050040540500403CDE0000EC
:106C30000000002064020020FEE7FEE7FEE7FEE71A
:106C4000FEE7FEE72D4B10B51A68D2B2012A0FD12C
:106C50002B4A126812070BD12A4AE0241168F0224D
:106C60000800104021422DD12749096811422CD03B
:106C70001A68D2B2012A12D12149096809070ED136
:106C8000F020204909680140402908D11E490968BF
:106C9000014204D18020C121C005C90042501B68B7
:106CA000DBB2012B0DD1164B1B681B0709D1154B0D
:106CB0001A68F0231A40A02A0FD1134A12681A4208
:106CC0000ED010BD3028CFD0D2E7104A1049116045
:106CD0008021104A09021160CAE7D02AF1D1ECE7FD
:106CE0000D4B1A68012A04D00C4A1A601A68012A4E
:106CF000FCD1C0220A4B1A60E3E7C046E00F00F067
:106D0000E40F00F0E80F00F0EC0F00F00405004085
:106D1000DFFF07C0186C004000EC064075930000D0
:106D200014EC06400120704710B503681322DB699C
:106D3000984710BD70470000054B0269D1500369A8
:106D4000FC331A6A002AFCD0002201201A62704724
:106D50001C050000030010B55C331A781F231A408D
:106D60001E3B19009140114AD167C22204210469D7
:106D70009200A150026953600269D360A0230022EF
:106D80000169DB00CA5001230169094A5B428B504B
:106D90000169084A8B5001690C3A8B50016908322D
:106DA0008B501430FFF7FCFE10BDC04604E100E03C
:106DB0000C0500001405000010B51430FFF702FFA9
:106DC00010BD10B51430FFF703FF10BD10B514301F
:106DD000FFF7EAFE10BD0000030070B55E331A78BD
:106DE0000469724BE25003005D331A780469704BFA
:106DF000E250030061331C7802696E4B012C00D015
:106E00009EE005005F352E78A225ED005651020068
:106E100060321578A1220669D200B5500269D450BB
:106E20009623DB00994200D88CE096231B019942FF
:106E300000D88AE096235B01994200D888E0962327
:106E40009B01994200D885E0E1239B01994200D83B
:106E500082E09623DB01994200D880E0E123DB0148
:106E6000994200D87DE096231B02994200D87AE02F
:106E7000E1231B02994200D877E096235B029942F6
:106E800000D874E0E1235B02994200D871E0E1236D
:106E90009B02994200D86EE0474B994200D86CE0C3
:106EA000E123DB02994200D86AE0E12200231203C9
:106EB0008A425B41414A5B421340802252059B1843
:106EC00001693F4A8B50A02304220169DB00CA50AC
:106ED00000210369FC33D9600369FC331962012383
:106EE00001690B6001698B60C121046989006250EE
:106EF0001F215C3002780A4093406231314AFF31F1
:106F000053500021415600293CDA0F230B40083B27
:106F10002D4C9B089B001B1903242140A140FC34ED
:106F20008C40DD69A5432C00C0258D4029002143FC
:106F3000D9611F23017819401E3B8B40136070BD3F
:106F400000246CE79E23DB02BAE79D231B03B7E70F
:106F50001E4BB5E71E4BB3E7EC239B03B0E71D4B7D
:106F6000AEE71D4BACE71D4BAAE71D4BA8E71D4B39
:106F7000A6E71D4BA4E71D4BA2E78023DB049FE798
:106F80001B4B9DE78C080F4BA400E41803230B4018
:106F9000FF21C025DB009940AD0066598E433100CA
:106FA000C0269E4033000B436351C2E70C0500002E
:106FB000140500006C05000090D0030000D0BEFE58
:106FC0002405000000E100E000ED00E000B0130047
:106FD0000050270000A04E0000F0750000509D00FA
:106FE00000F0EB0000903A0100E0D70100B0AF03E1
:106FF00000705F07F7B5009308AB1B78002501937D
:10700000FA2304009B0083600E4B45600833036045
:1070100014300F001600FFF7ADFD23005C3327612D
:107020001E70009B084A9B00995823005D3319701D
:10703000019B20009B009A5823005E33DD701A707C
:10704000FEBDC0466CD90000E8D80000036910B549
:107050001A00FC32D2680400002A0AD0A322D2000F
:1070600099581430C9B2FFF790FD00222369FC3310
:10707000DA6010BD10B50248FFF7E8FF10BDC0464A
:10708000B01B0020162307B5022200930249013BE2
:107090000248FFF7AFFF07BD00200040B01B0020F3
:1070A00010B5002801D004F07DFA10BD7047000033
:1070B00010B500F011F8FFF7F9FF012000F000FA19
:1070C000FFF7F2FAFFF702FB024B002BFAD000E0C9
:1070D00000BFF7E700000000C420114B80001A58E1
:1070E00010491140C02212020A431A50C0218022C6
:1070F000490092025A501A608023A3220021DB0526
:10710000D20099500122F9309A60074BFF30195094
:10711000C120023180001950403019501A60704768
:1071200000E100E0FF00FFFF00100140014B18608C
:107130007047C04678000020F7B5002320285AD8B1
:10714000384B8000C258042A5BD007D8022A54D09A
:1071500055D80423012A09D000234CE0062A54D034
:1071600051D31A2A53D002231B2AF5D12E4A116873
:1071700008294ED909294FD00A240226A02001252A
:107180002A4AC00015502A482A4D07681C20BF0013
:1071900007402948019700685759009027481B026B
:1071A00007401F43C02300989B020340FF20575114
:1071B0005759000207401F43019B1F43009B580182
:1071C0006023184007433E43565101251C4B156070
:1071D00058680028FCD000205860A1230125DB005E
:1071E000D3585560A025ED0050511BB2A14202D0EA
:1071F00015D2611ACB401800FEBD0823B6E7102354
:10720000B4E72023B2E74023B0E78023AEE70123B1
:10721000ACE708240026B1E70C000126AEE7091B05
:107220008B40E8E7E8D800007400002000700040C0
:10723000300000200405000034000020FF00FFFFA4
:10724000FC700040F0B520285BD8364B8000C25857
:10725000354B1E68002E30D1C227344BBF00D859A1
:10726000334C03250440C02000022043D851C024E1
:1072700080206400800018512E4F18602E4B803CF7
:10728000D859FF3CA043D8510437D859A8432043CC
:10729000D8510837D8590C35A8438446072065468D
:1072A0002843D851A820C0001E50C120802680004D
:1072B00076021E501C601C4B1C60142500202B0005
:1072C0001E4C2E0046433659771C1BD14343E250D7
:1072D000A0230325C132FF329200DB05D550184BA5
:1072E0001A68082A14D114234343E3189A681248F1
:1072F0005132FF32920059601150DA68C1239B006D
:10730000C250F0BD9642E1D001300328D9D1F8E750
:10731000082A02D9083AD140E5E708239A1A914091
:10732000E1E7C046E8D80000141C002000E100E0BE
:10733000FF00FFFF0405000000900040380000201F
:10734000780000202149F0B54A6C2148002A14D069
:10735000A025A12600230124ED05F600C258571CE4
:1073600006D0C7187F68002F02D027009740AF5182
:1073700014333C2BF2D100234B64A0230121DB0505
:1073800000260F009C4614234B43C3181A1F126893
:10739000104C0E4D920014195219526C002A10D044
:1073A0001A00143A1268551C09D0103B1B68FF2BB9
:1073B00005D03B00934065461A00074BEA50FC3469
:1073C000666401310429DED1F0BDC046FC90004066
:1073D00038000020009000400C05000000B5202877
:1073E00010D80C4A8000835803290BD8A02208002B
:1073F000C133FF33D2059B0001F036FC02090507BB
:107400000021D15000BD0C21FBE70421F9E7032145
:10741000F7E7C046E8D8000020280AD8074B8000CC
:10742000C25801239340A022D205002902D1044969
:1074300053507047A121C900FAE7C046E8D80000C0
:107440000C05000003000020202B0AD8A021A22256
:10745000C905D2008858034A9B009B58D840012395
:1074600018407047E8D80000F7B506000D000C0082
:107470008B180193019B671B9C4207D033682178CE
:107480001B683000984701340028F3D13800FEBD56
:107490000849094A094B10B51B688858FA22190A8D
:1074A0001B0618439200002301F0B4FD4904C00BF1
:1074B000084310BD0010014004050000181C002006
:1074C00070B5041E09D0FFF7E3FF050000F014F8C3
:1074D000FFF7DEFF401BA042F8D370BD0022044B33
:1074E0009A60044A13680133DBB213607047C046E8
:1074F000FC100140181C002070470000F0B5C64683
:1075000000B5CB0F9846404A4B005B0D9A1882B0ED
:107510000D000400132A2FDC002A49DB3B4F1741E2
:107520003E000E40064323D07F08390029400C431B
:107530000AD03749BD438C4663445C425C4180239A
:10754000DB021341E4071D434146CE0031492B00C5
:107550008E192200346875682000290001F000FFB0
:10756000009001910098019922002B0003F090F8FF
:1075700002B004BC9046F0BD332A08DD8023DB0056
:107580009A42F5D102000B0001F0EAFEF0E7224A30
:107590009446012263445242DA400242E8D0520843
:1075A0000242D1D094438022D2051A411443CBE742
:1075B0004B005B080343DBD00B031B0B1C436342F4
:1075C000234380244D0C24031B0B23406D042B43C9
:1075D00019004346DA000F4B9B181C685D680200D7
:1075E0000B002000290001F0BBFE009001910098E3
:1075F000019922002B0003F04BF842464B005B0838
:10760000D60733431900B3E701FCFFFFFFFF0F006C
:10761000EEFBFFFFA0D90000EDFBFFFFF8B5274A06
:107620004B005B0D9A180C000700132A10DC002A8F
:1076300036DB234B13410B423AD080242403144100
:10764000002064189C430600250030002900F8BD86
:10765000332A0EDD80230600DB000D009A42F4D1B0
:1076600002000B003800210001F07AFE06000D0038
:10767000EBE7144D0600AC46012563446D42DD4046
:10768000AC4663460D000342DFD033239A1A323BE7
:1076900093401818874200D94C1C63469843D2E7A0
:1076A000C90FCC070020531CCDD1074B1C43CAE7A0
:1076B00006000D000028C0D1C7E7C04601FCFFFF4F
:1076C000FFFF0F00EDFBFFFF0000F03F30B5214A48
:1076D0004B0087B05B0893421EDD1F4A934205DDD5
:1076E00002000B0002F0D4FF07B030BD02AA00F088
:1076F00095F803231840049A059B012813D002280B
:107700001DD0002814D00298039900F06FFB80234D
:107710001B069C466144E7E70023002200930023F8
:1077200001F0DEF8E0E70298039900F05FFBDBE789
:10773000012402980399009401F0D2F8D4E70124BF
:1077400002980399009401F0CBF880231B069C4615
:107750006144C9E7FB21E93FFFFFEF7FF0B54746F2
:10776000CE4680B58DB004000D0000F067FA294BBD
:1077700006001B780F005BB29846013310D0220040
:107780002B002000290003F0CBFA8146002807D106
:10779000002200232000290001F014FC002806D15B
:1077A000300039000DB00CBC90469946F0BD012365
:1077B0000293194B0694079503934B460A9343464D
:1077C00004940595002B15D0002300221900100009
:1077D00002F0E2F8434608900991022B0ED103F023
:1077E000B9FB212303600A9B0193002B0CD1089E57
:1077F000099FD5E7002300240893099402A801F00B
:10780000C1F90028EFD1EAE703F0A4FB0A9B01933A
:107810000360ECE77C000020B0D90000F0B54E46D4
:107820004546DE465746E0B5E14B4C008FB09046EA
:10783000894664089C4200DC87E0DE4B9C4222DCE7
:10784000DD4A002900DC92E0DC4B02F021FFDB4B3B
:1078500006000F009C4200D17EE1D94AD94B02F0CC
:1078600017FF02000B00414630000A604B603900F0
:1078700002F00EFFD34BD24A02F00AFF4346012525
:107880009860D9606BE0D04B9C4200DC8FE0CF4B1E
:107890009C4200DD55E1CE4A231592469A4451465A
:1078A0000905631A19001D00040003F055FA03F0DE
:1078B00089FA02000B00200029000892099302F0C7
:1078C000E7FE0022C34B02F071FC0F00060003F03C
:1078D00043FA03F077FA04000D0002000B003000B9
:1078E00039000A940B9502F0D3FE0022B94B02F046
:1078F0005DFC002200230C900D9101F05DFB00283F
:1079000000D192E1002300222000290001F054FB65
:10791000434243410133B04A41460192022208A842
:107920000092524600F07CFB4B460500002B16DA15
:10793000802243461206944642465B6845426344B1
:107940005360D3686344D36009E00B0002004146F2
:107950000A604B600022002300258A60CB6028006B
:107960000FB03CBC90469946A246AB46F0BD934B47
:1079700001F0F6FC914B06000F009C4200D13DE166
:107980008F4A904B01F0ECFC02000B0041463000A6
:107990000A604B60390002F07BFE894A894B01F096
:1079A000DFFC012543466D429860D960D7E701F0BE
:1079B00049F88A4A8A4B06000F0002F0F7FB0022C2
:1079C000884B01F0CDFC03F0C7F9050003F0FAF98C
:1079D000794A7A4B0490059102F0E8FB02000B0013
:1079E0003000390002F054FE754A06000F0004987A
:1079F0000599744B02F0DAFB029003911F2D00DC15
:107A0000C7E0029A039B3000390002F041FE834632
:107A10008A4653465B0024155B0DE31A102B6CDD80
:107A200004980599D322674B520502F0BFFB020070
:107A30000B00300039000292039302F029FE0A0085
:107A4000010013000691079202003900300002F095
:107A50001FFE029A039B02F01BFE06000F00049813
:107A60000599614A614B02F0A1FB32003B0002F034
:107A70000FFE069E079F0B000200390030000292A5
:107A8000039302F005FE4B005B0D83468A46E41A21
:107A9000312C32DD04980599B822544B920502F03E
:107AA00085FB03000C000200029303940B00069870
:107AB000079902F0EDFD02000B0006000F0006988A
:107AC000079902F0E5FD029A039B02F0E1FD484AA6
:107AD0000290039104980599464B02F067FB029AC5
:107AE000039B02F0D5FD02000B003000390002922A
:107AF000039302F0CDFD83468A465A4653464146DB
:107B000030000A604B60390002F0C2FD029A039B0C
:107B100002F0BEFD44460B000200A260E3604B464B
:107B2000002B00DB1BE75B46236080231B065344CE
:107B3000636080231B069C466144A060E1606D4247
:107B40000DE70B00020002F0A3FD434600259860FC
:107B5000D9601860596002E7D3221A4B520502F02F
:107B600097FD214A214B0D00040002F091FD020017
:107B70000B00414620000A604B60290002F088FD9E
:107B80001A4B194A02F084FD434601259860D960DA
:107B9000E5E602000B003000390002F079FD6B1EB3
:107BA000154A9B009B5883468A46A342A5D130E7DD
:107BB000FB21E93F7BD9024000004054FB21F93F03
:107BC0003163621A61B4D03DFB213941FFFFEF7F81
:107BD000EAFBFFFF0000704138DA000083C8C96D7E
:107BE000305FE43F0000E03F7370032E8A19A33B2F
:107BF000C14920259A837B39B8D90000D3220C4B88
:107C0000520501F0ADFB0B4A0B4B04000D0001F0D7
:107C1000A7FB02000B00414620000A604B602900D0
:107C200002F036FD034A044BB9E6032373E6C0466F
:107C300061B4D03D7370032E8A19A33BF8B5474653
:107C4000CE46674B80B50A000F0019000500394089
:107C5000994200D19BE004000100002F69DD3F152F
:107C600000D1B4E05F4B12039C468023120B5B03F0
:107C700013435B00CA0F67449B184A00F80703D5FB
:107C8000D20F5B009B188A0079108C46002180205F
:107C90001624894680030D189D4202DC29185B1BBF
:107CA0008144D50F5B00013C5B1952004008002C59
:107CB000F1D100208046802020250027000609E021
:107CC0008B425CD0D40F5B00013DE31852004008AA
:107CD000002D16D0C4198B42F2DD27180E00002C9F
:107CE00049DB5B1AA242894149425B1A121BD40F3D
:107CF0005B00013D80443100E31852004008002D34
:107D0000E8D113434ED143465B0837494A4688467B
:107D1000494652104244C90702D5802109060B4347
:107D200061460F05BD18180029000CBC9046994605
:107D3000F8BD7B005B0803433900002BF5D0002F12
:107D40003CD1E30A153A6405002BFAD080204003A9
:107D500003423FD1002700E00F005B00791C034283
:107D6000FAD0250020208D40401A2900D71B220080
:107D7000C2401A4376E7FE43F60F8E19B1E79442EC
:107D8000A0D82718002CF6DB1E000023AEE7020067
:107D90003B002800390002F009FA2A003B0001F0FC
:107DA000DFFAC2E74346013303D0434601335B08A1
:107DB000ABE7012398460023C144A6E73B0002003D
:107DC00002F066FC02000B0001F0E6FDADE71300D7
:107DD0000022BBE70127210020207F42C6E7C046E2
:107DE0000000F07F01FCFFFF0000E03FF0B54746D8
:107DF000CE4680B587B000920193754B4F00814607
:107E000088467F089F4263DC02F0A6FF002800D16D
:107E1000D4E04A4643464846414602F0C7F90400CA
:107E20000D006C4A6C4B02F0C1F96C4A6C4B01F0CE
:107E300097FA22002B0002F0B9F96A4A6A4B02F065
:107E400027FC22002B0002F0B1F9684A684B01F0D0
:107E500087FA22002B0002F0A9F9664A664B02F06D
:107E600017FC22002B0002F0A1F9644A644B01F0D8
:107E700077FA22002B0002F099F902900391002278
:107E8000604B2000290002F091F9029A039B060042
:107E90000F002000290002F089F9009A019B0400DC
:107EA0000D004846414602F081F902000B00200017
:107EB000290002F0EDFB02000B003000390002F057
:107EC000E7FB02000B0000204F4902F0E1FB70E0ED
:107ED00002000B0002F06AF904000D003D4A3E4B1F
:107EE00002F064F93D4A3E4B01F03AFA22002B00C1
:107EF00002F05CF93B4A3C4B02F0CAFB22002B002B
:107F000002F054F9394A3A4B01F02AFA22002B00C8
:107F100002F04CF9374A384B02F0BAFB22002B0032
:107F200002F044F9354A364B01F01AFA2B002200D0
:107F300002F03CF9354B029003919F429FDD344B98
:107F400000229F423DDC334900207B182E49160059
:107F50001F0002F09DFB049005910022294B200098
:107F6000290002F023F932003B0002F091FB029A53
:107F7000039B06000F002000290002F017F9009A69
:107F8000019B04000D004846414602F00FF9020033
:107F90000B002000290002F07BFB02000B003000E8
:107FA000390002F075FB02000B000498059902F0FD
:107FB0006FFB07B00CBC90469946F0BD00201249FB
:107FC000F7E7154B002604920593144FC5E7C0460A
:107FD000FFFF3F3ED43888BEE9FAA8BDC4B1B4BDA6
:107FE0009EEE213EAD529C804F7E923E9015CB1965
:107FF000A001FA3E7751C1166CC1563F4C555555FC
:108000005555A53F0000E03F0000F03F3233D33F1D
:108010000000E93F0000E0FF0000E73F0000D23F22
:10802000F0B5DE464E4645465746E0B5DC4CA54425
:108030000D9114001900A49A0993DA4B9200D658B6
:108040004D1E03901821E01E0696029500F0AAFE30
:10805000C3430100DB1719404B1C9A009B1ADB003D
:108060001B190B9105934C1B771918D4A59BA500E0
:108070009C463F1922AE6544013707E0286802F0AC
:10808000A1FE013403C60435BC4208D0002CF5DA49
:1080900000200021013403C60435BC42F6D1069B02
:1080A000002B01DA00F0FDFB069B03990133DB0096
:1080B0009A46099BDA00944600920022914672AAE1
:1080C0000492B94A6144934688469AAB63449B4400
:1080D000029B002B00DABCE15D4600260027039CD2
:1080E0004D442A686B6803CC02F060F802000B0074
:1080F0003000390001F034F9083D06000F00444516
:10810000EFD1049B4B441E605F6008239C46E14412
:10811000D145DDD10EA804218446494261448C46F4
:10812000069A93009C44614684460A910399083B51
:1081300063448C460C93009B009263449B46009AD8
:108140000498D10003008C46634408911E685F6860
:10815000002A33DD954980468C466244D30098441A
:1081600070AB9A460EAB99460022914B3000390015
:1081700002F01CF802F0F0FD02F024FE00228D4B0C
:1081800004000D0002F012F802000B00300039006C
:1081900002F07EFA02F0E0FD4B4601C399464346E9
:1081A00020001A685B68290001F0DAF808235B42B6
:1081B0009C46E04406000F00D045D5D1059B300019
:1081C0001A003900984600F0DFFCFF2300229B05CF
:1081D00004000D0001F0EAFF00F038FC0022764BAD
:1081E00001F0E4FF02000B002000290002F050FA29
:1081F0000D00040002F0B0FD814602F0E3FD020034
:108200000B002000290002F043FA060040460F0050
:10821000002800DCEEE0009B18215A1E92000EABF5
:108220009B58091A1D000D41A9448D405D1B0EABE2
:108230009D5017231B1A1D41002D2DDD01239C4647
:10824000009BE144002B00DC1CE20E9C0123002C6F
:1082500000D0B5E0009A012A09D099000EAA54581E
:108260000133002C00D0ACE0009A9A42F5D1059B76
:10827000002B0EDD012B00D1A8E1022B09D1009BC0
:108280000EA95A1E92000EAB9B5807939B029B0AA5
:108290008B50022D00D1C1E00023002230003900B4
:1082A00000F08AFE009B002800D194E2069A591E35
:1082B0008A4210DC414A0A9894460EAA63449446C6
:1082C00000229B0063441C68043B22438342FAD192
:1082D000002A00D0C0E0069B0EAA013B9B00D358A9
:1082E000002B00D0B3E001220C9B043B5968013203
:1082F0000029FAD0009B9C466244110007921A00A4
:1083000001338B4246DC0B9863468046A59C434470
:10831000A046099C9B00A1464A449844D30022AA47
:108320009146049A99449446089BA59A63448446CE
:10833000614494469A468B006344009343465868D0
:1083400002F040FD4B4618605960029B002B24DB75
:108350004D46039C0026002701E0286869680CCC84
:1083600001F024FF02000B003000390000F0F8FF9C
:10837000083D06000F005C45EFD153469E60DF606C
:1083800004239C460433E0449C46009BE144E244C1
:108390009845D3D1079B0093D1E600260027ECE750
:1083A00094FDFFFF80DB000018FEFFFFFFFFFF1FB3
:1083B0000000703E0000704100002040FFFFFF3FC2
:1083C000002180225204141B0EAA54500099994295
:1083D0000EDD0EA884469B000EAA8900D258614487
:1083E0006344CF4800E01A68821A04C38B42FAD172
:1083F00001243CE7059B002B06D1009B0EAA013B04
:108400009B00D558ED1517E70022C64B300000F051
:10841000F7FD002800D024E100253DE732003B00B5
:108420000020C14902F034F906000F00002C00D1F1
:1084300032E7059A0020BC4900F0A6FB02000B00C1
:108440003000390002F024F906000F0024E7012271
:1084500050E70026002754E64B46059A07938846C6
:108460008B000EA9CB58183A08950592002B0DD118
:108470008C464146AD4B43449B006344043B5868E3
:108480000139183A0028F9D088460592059A00204B
:10849000A54900F079FB434604000D00002B00DAEB
:1084A00005E29E000EAB9C464346DB0066449C46BC
:1084B000059370AB9946049F67440097306802F0BB
:1084C00081FC22002B0001F071FE002238607960EF
:1084D000974B2000290001F069FE083F04000D00C1
:1084E000043EB945EAD14AAB03939B4600239A4622
:1084F000069B4246994643460132029204934B46FC
:10850000002B00DAAAE080208A4B009D9846C00527
:10851000894900260027002408E008239C460835E6
:10852000E044544511DC4346186859682A686B6872
:1085300001F03CFE02000B003000390000F010FF9B
:10854000013406000F00A145E7DA5B46C0C39B4635
:1085500001239C46009BE244083B0093029B9A4502
:10856000CDD1049B9846A49B022B00DD8EE0002B0E
:1085700037DC1FD1059B00271D00039B00249C4670
:108580001E006544083E2A686B683800210000F030
:10859000E7FE083D07000C00AE42F4D1089B002B1B
:1085A00003D080231B069C4664443A0023000D99A7
:1085B0000A604B600720079B18409B239B009D444B
:1085C0003CBC90469946A246AB46F0BD009B0EA926
:1085D0005A1E92000EAB9B5807935B025B0A8B50AE
:1085E00057E64346002B00DA70E100200021DB0053
:1085F0004AAAD61848AF32687368083E00F0B0FE49
:10860000B742F8D1089B002B00D025E10B000200F7
:108610004A984B990D9C2260636002F039F84346FA
:1086200007000C00002B13DD01254CAEB1463800CD
:108630002E0021004C4601360CCC00F091FEA146E4
:10864000B045F7DA089B07000C00002B00D015E1BD
:108650003A0023000D998A60CB60ABE70026002723
:1086600073E701239C46009BE1440225002B00DDBB
:10867000EBE532003B0000202B4902F009F8060030
:108680000F0009E60024F2E54AAB0393A49B032BF9
:1086900000D08FE74346002B00DC14E1039ADB0097
:1086A0009B46130091465B441E685F68234B43441E
:1086B0000293DB00994448AB9A464B465C681B68C2
:1086C0001800210032003B000090019100F048FEAC
:1086D00004000D0002000B000098019901F0D8FF82
:1086E0003B00320000F03CFE4B469860D9601C60B5
:1086F0005D6008235B429C46E14426002F00CA458A
:10870000DBD14346012B00DCE3E0039A13005B441A
:108710001E685F68029BDB0099464A44904610E061
:10872000FFFFFF000000E03F0000F03FFFFFFF3FC2
:108730000000703E40DB0000FB21F93FFFFFFF1F00
:10874000984643465C681B681800210032003B00D5
:108750000090019100F004FE04000D0002000B00E7
:108760000098019901F094FF32003B0000F0F8FD01
:108770004346039A9860D9601C605D60083B260000
:108780002F009A42DCD14D469446002600244746ED
:10879000083565442A686B683000210000F0E0FD70
:1087A000083D06000C00AF42F4D1039B4A9F5D6870
:1087B0009968D868089B002B65D0802212069446E1
:1087C0000D9B6544604464441F605D609960D8609F
:1087D0001E615C61EEE69A464B460793059B3000AE
:1087E0005A423900089500F0CFF900223A4B0600B2
:1087F0000F0000F005FC002824D0384B0022300088
:10880000390001F0D3FC02F0A7FA524604009500AB
:1088100002F0D8FA0022304B01F0C8FC02000B0035
:108820003000390001F034FF02F096FA0EAA5051E0
:108830000122059B524418339046059393000EAADB
:10884000D45023E65346300039009C0002F084FAED
:108850000EAB1851D04619E680230D9A1B06CB1893
:10886000106053600B0002004A984B9901F010FF12
:10887000434607000C00002B00DDD5E680231B06D5
:108880009C466444E4E62B003A000D9D2A606B6030
:108890000A000300AA60EB60320023002A616B61CA
:1088A00088E6099BDB00009372AB049332E4A49B3F
:1088B000022B00DDE8E6002B00DD92E600D079E631
:1088C000002700246AE6002600246EE7002000212D
:1088D00098E60026340068E7000070410000703E12
:1088E000F0B5CE46474680B587B000920193474A1F
:1088F0004B00814688465B08934207DC4146484668
:1089000002F02AFA4146031E484666D04A464346CC
:108910004846414601F04AFC04000D0002000B00ED
:108920004846414601F042FC394A3A4B06000F00E6
:108930002000290001F03AFC374A384B01F0A8FE2C
:1089400022002B0001F032FC354A364B00F008FDC6
:1089500022002B0001F02AFC334A344B01F098FE30
:1089600022002B0001F022FC314B324A00F0F8FCCF
:108970000E9B02900391002B34D0009801990022A5
:108980002D4B01F013FC029A039B049005913000DB
:10899000390001F00BFC02000B000498059901F06E
:1089A00077FE22002B0001F001FC009A019B01F0F0
:1089B0006FFE224A04000D00214B3000390001F007
:1089C000F5FB02000B002000290000F0C9FC0200AA
:1089D0000B004846414601F05BFE07B00CBC9046D8
:1089E0009946F0BD02000B002000290001F0DEFBDB
:1089F000124A134B01F04CFE32003B0001F0D6FB53
:108A00004A46434600F0ACFCE7E7C046FFFF3F3E66
:108A10007CD5CF5A3AD9E53DEB9C2B8AE6E55A3E08
:108A20007DFEB157E31DC73ED561C119A0012A3FA4
:108A30001111813FA6F810110000E03F495555552E
:108A40005555C53F49004B0819007047474AF0B5D6
:108A50004F4691464B005B0D99444646D6464A46E2
:108A6000C0B505000C000E0088460700132A27DC5D
:108A7000002A4BDB3E4B13419A460B0052461340F3
:108A8000034318D03B4A3C4B2800210000F068FC0F
:108A90000022002300F0AAFA002847D0002C04DAB4
:108AA00080234A465B0313419844464653460027B9
:108AB0009E43380031001CBC90469946A246F0BD4A
:108AC000332A08DD8023DB009945F4D102000B0036
:108AD00000F046FCEFE7294A9446012263445242E3
:108AE000DA4092460242E6D0224A234B2800210077
:108AF00000F036FC0022002300F078FA002815D0A0
:108B0000002C1EDB534646469F430FE0194A1A4B82
:108B10002800210000F024FC0022002300F066FA67
:108B2000002803D0002C04DB002700263800310089
:108B3000C1E76400640825430027002DF6D0104EDD
:108B4000F4E74B46142B0BD03422D21A0123934066
:108B50005D19BD4208D201239C462F00E044D1E7B5
:108B6000133B9C46E044CDE72F00CBE701FCFFFF21
:108B7000FFFF0F009C7500883CE4377EEDFBFFFF94
:108B80000000F0BF002070474B0070B55B0D140073
:108B90000A00002B1AD14B005B08034315D0234B6E
:108BA000002201F003FB224B9C422DDB0A004B000C
:108BB0005B0D363B1F4DE318AB422ADC002B0DDD6D
:108BC0001D4C1B0522401A43110070BD1B4DAB42CA
:108BD000F0D102000B0000F0C3FBF6E71D003535B5
:108BE00019DA174B02009C4209DD0B0015481649A3
:108BF00000F032F8134A144B01F0D8FAE5E70B0005
:108C00001248134900F028F8104A114B01F0CEFA2F
:108C1000DBE70200E9E7084C363322401B0513432B
:108C2000190000220B4B01F0C1FACEE700005043BF
:108C3000B03CFFFFFE070000FFFF0F80FF070000B2
:108C400050C300009C7500883CE4377E59F3F8C29D
:108C50001F6EA5010000903C30B54A00DB0FDB071A
:108C600052081A43110030BD02B471464908490048
:108C7000095C49008E4402BC7047C04603B471468B
:108C8000490840004900095A49008E4403BC704716
:108C9000002243088B4274D303098B425FD3030A3B
:108CA0008B4244D3030B8B4228D3030C8B420DD34E
:108CB000FF22090212BA030C8B4202D312120902DC
:108CC00065D0030B8B4219D300E0090AC30B8B421A
:108CD00001D3CB03C01A5241830B8B4201D38B03C8
:108CE000C01A5241430B8B4201D34B03C01A52416D
:108CF000030B8B4201D30B03C01A5241C30A8B42B0
:108D000001D3CB02C01A5241830A8B4201D38B029A
:108D1000C01A5241430A8B4201D34B02C01A52413E
:108D2000030A8B4201D30B02C01A5241CDD2C309B0
:108D30008B4201D3CB01C01A524183098B4201D32C
:108D40008B01C01A524143098B4201D34B01C01A17
:108D5000524103098B4201D30B01C01A5241C3088F
:108D60008B4201D3CB00C01A524183088B4201D3FE
:108D70008B00C01A524143088B4201D34B00C01AEA
:108D80005241411A00D20146524110467047FFE756
:108D900001B5002000F0F0F802BDC0460029F7D070
:108DA00076E7704703460B437FD4002243088B428B
:108DB00074D303098B425FD3030A8B4244D3030B62
:108DC0008B4228D3030C8B420DD3FF22090212BA27
:108DD000030C8B4202D31212090265D0030B8B42A3
:108DE00019D300E0090AC30B8B4201D3CB03C01A8D
:108DF0005241830B8B4201D38B03C01A5241430B68
:108E00008B4201D34B03C01A5241030B8B4201D357
:108E10000B03C01A5241C30A8B4201D3CB02C01AC2
:108E20005241830A8B4201D38B02C01A5241430A3A
:108E30008B4201D34B02C01A5241030A8B4201D329
:108E40000B02C01A5241CDD2C3098B4201D3CB01D0
:108E5000C01A524183098B4201D38B01C01A52417F
:108E600043098B4201D34B01C01A524103098B4283
:108E700001D30B01C01A5241C3088B4201D3CB006E
:108E8000C01A524183088B4201D38B00C01A524151
:108E900043088B4201D34B00C01A5241411A00D201
:108EA00001465241104670475DE0CA0F00D049426A
:108EB000031000D34042534000229C4603098B42DA
:108EC0002DD3030A8B4212D3FC22890112BA030A62
:108ED0008B420CD3890192118B4208D389019211E4
:108EE0008B4204D389013AD0921100E08909C30969
:108EF0008B4201D3CB01C01A524183098B4201D36B
:108F00008B01C01A524143098B4201D34B01C01A55
:108F1000524103098B4201D30B01C01A5241C308CD
:108F20008B4201D3CB00C01A524183088B4201D33C
:108F30008B00C01A5241D9D243088B4201D34B0057
:108F4000C01A5241411A00D20146634652415B1099
:108F5000104601D34042002B00D54942704763467A
:108F60005B1000D3404201B5002000F005F802BDBF
:108F70000029F8D016E770477047C046D0400B1C58
:108F80001141203A03D49C46134118436346524290
:108F9000934018437047C0468446101C62468C4676
:108FA000191C634600E0C0461FB501F097F8002881
:108FB00001D40021C8421FBD10B500F0EFFF4042B0
:108FC000013010BD10B501F089F8002801DB002048
:108FD00010BD012010BDC04610B501F07FF800287B
:108FE00001DD002010BD012010BDC04610B501F00C
:108FF00011F8002801DC002010BD012010BDC04682
:1090000010B501F007F8002801DA002010BD01209A
:1090100010BDC046F0B5CE46474615042D0C2E00B7
:1090200080B50704140C3F0C9946030C7E435D4346
:10903000674363437F19340CE4199C46A54203D966
:1090400080235B029846C4444B4643435143250C5E
:1090500036046544360C2404A4195B195918200001
:109060000CBC90469946F0BDF0B54E465746454675
:10907000DE46E0B543025B0A450083B00F1C99460B
:109080002D0EC60F002D57D0FF2D24D08020DB00E1
:10909000C0041843002381469A469B467F3D7C02CC
:1090A0007A00FB0F640A120E984623D0FF2A4BD099
:1090B000E30080240020E4047F3A1C43AD186B1CBD
:1090C00047460193534677403A000F2B48D87D49D5
:1090D0009B00CB589F46002B00D085E008339A4672
:1090E000063B9B467C027A00FB0FFF25640A120EAA
:1090F0009846DBD1002C00D090E0524601231A4361
:1091000092460120DBE74C4658461700022824D03F
:10911000032800D1CFE00022002301284DD15802BE
:10912000D205400AFF071043384303B03CBC9046C9
:109130009946A246AB46F0BD002B5BD104239A466C
:10914000033B00259B46AAE7FF35002C60D1524621
:1091500002231A4392460220B1E7FF220023DEE7F2
:109160004B461B0C9C464B462604360C18046146A5
:109170003300220C6446000C43434E435043544397
:1091800080191A0C1218964203D9802149028C4684
:1091900064441B041B0C1004C01883015E1EB34101
:1091A000800E1843130C1B199B0103431C00230161
:1091B00079D5012362081C401443019A7F32002AAA
:1091C0004DDD630704D00F232340042B00D004346B
:1091D000230103D53C4B019A1C408032FE2ABCDCA3
:1091E000A3015B0AD2B29AE70C239A46093BFF25FA
:1091F0009B4654E7180001F071FE4A46431F76254E
:109200009A4000236D4291462D1A9A469B4646E7A6
:10921000524603231A439246032050E7200001F0F0
:109220005DFE431F2D1A9C40763D002047E78023BA
:109230000027DB03FF2272E7424666E74C46320016
:10924000584662E780234A46DB031A4222D01C427A
:1092500020D123435B025B0A4746FF225FE70123DD
:109260009A1A1B2A21DC23000199D3409E318C409D
:109270001A0023005C1EA34113435A0704D00F2297
:109280001A40042A00D004335A0111D49B015B0A0E
:10929000002244E780234A46DB0313435B025B0A58
:1092A0003700FF223BE7019587E70022002336E7DE
:1092B0000122002333E78023DB0323435B025B0AA5
:1092C000FF222CE790DB0000FFFFFFF770B50028BE
:1092D0003DD0C317C5185D40C40F280001F0FEFD46
:1092E0009E22121A962A07DCD2B2082833DD0838EB
:1092F00085406802400A23E0992A0BDD05232900F6
:109300001B1AD94003001B339D402B005D1EAB414F
:1093100019430D00052801DD431F9D402B000F4917
:109320000B406E0709D00F263540042D05D00433BD
:109330005D0102D59F220B40121A9B01580AD2B23E
:109340004002D205400AE4071043204370BD0024C8
:1093500000220020F4E76802400AF1E7FFFFFFFB6C
:10936000F0B54F464646D6460C000903C0B5490A3B
:10937000470F5E0039431F03DB0F9C4665007B0AE5
:10938000570F1F436D0DE40F760DA146C000B84680
:10939000D200AB1B64457BD0002B5FDD002E00D0DC
:1093A000A4E03E00164300D112E15E1E002E00D064
:1093B0009EE1871A4346B84280410125C91A4042BE
:1093C000091A0B0200D431E149024E0A002E00D1E5
:1093D0006EE1300001F082FD0300083B1F2B00DD31
:1093E00061E120223900D21A9E40D1409F400E43B5
:1093F0009D4200DD51E15D1B6B1C1F2B00DD7CE1FC
:109400002021C91A3D0030008F408840DD40791E80
:109410008F41310007222843D940002507433A40B5
:10942000002A09D00F233B40042B05D03B1DBB4233
:10943000BF417F42C9191F000B0200D426E26A1CFB
:10944000C64B55056D0D9A4200D106E1C44AFF088E
:109450000A40530752023B43120B8EE0002B00D010
:10946000B8E06B1C5B055B0D012B00DC30E1871A5B
:109470004346B842B641CB1A76429E1B330200D512
:109480004CE13B003343A1D100220024002570E0D1
:10949000002B00DCE5E0002E00D183E0AF4EB542AA
:1094A00060D0802636043743B846382B00DC3EE1D6
:1094B000434613431F007A1E97413F18874280415D
:1094C000404209180B0200D4B0E0A44B01359D4284
:1094D00000D1C3E0A24A7B080A4001210F401F438C
:1094E0005108D30707221F433A4099E79B4EB542E4
:1094F00038D0802636043743B846382B00DDDCE010
:109500001F2B00DC30E11E004746203EF740BC46E2
:10951000202B04D04026F31A46469E4032431700C3
:1095200063467A1E97411F43CCE0002B00D104E232
:109530004346134300D159E14B07C0081843802329
:10954000C9081B03194208D04546ED081D4204D145
:109550004346D008590708432900420FC9007F4DF0
:109560001143C0004B07CA087C49C00803438D4221
:1095700068D012036D05120B6D0D00211203180047
:10958000130B0A0D12051A43764B2D0513402B437E
:109590005B00E4075B08234319001CBC9046994616
:1095A000A246F0BD3E00164312D05E1E002E00D033
:1095B00000E1871887428041414440420918012553
:1095C0000B0233D5022585E764463300414610007F
:1095D0001D00C7E7002D00D0DAE00C000443F3D0F3
:1095E0005C1C00D19FE15D4CA64200D12FE1DB4322
:1095F000382B00DD66E11F2B00DD83E12024050010
:10960000E41A0F00DD40D940A0404346A7405B1A52
:10961000441EA04198462F433843171ABA4292413C
:1096200043465242991A64463500CAE607223A4038
:10963000002A00D0F6E64B07CA084849FF083B431A
:109640008D4296D11900114300D19EE1802109037A
:109650000A431203120B414D8FE71500002200232D
:109660008BE7002B00D0C7E06B1C5F057F0D012F3F
:1096700000DCF1E0394DAB4200D1B9E085180A00B9
:10968000854289414244494251180722CF076D085B
:109690002F4349083A401D00C2E607223049ED1A1F
:1096A00031403A40BCE63E002838864000279FE61D
:1096B000380001F013FC20308EE6434613431F00B0
:1096C0007A1E9741C71BB84280414042091A78E68A
:1096D0000E003B0006431343002D61D1002E00D045
:1096E000F4E0002B00D11BE164463900100039E79B
:1096F0001A4FBB427AD03300FFE630001F3DE840EE
:10970000202B03D04021CB1A9E4037437B1E9F4124
:10971000072207433A400021002589E7171A4346EC
:10972000BA42B641591A76428E1B64464EE61F2B4A
:1097300000DDADE020264746F61AB740B9461700CF
:10974000B246DF404E463E4337005646B240561EB4
:10975000B24117434246DA408918AEE6FF070000DF
:10976000FFFF7FFFFFFF0F8020264746F61AB74016
:10977000B9461700B246DF404E463E4337005646D4
:10978000B240561EB24117434246DA40891A99E761
:109790007F4CA6425BD0802424045B42214327E710
:1097A000002E0CD1002B00D1CBE064463900100014
:1097B000774DD7E6764FBB4218D0330075E6002BC5
:1097C00014D04B07C00818438023C9081B03194253
:1097D00007D0FC081C4204D17907D0080843E146B1
:1097E00021004C46420FC9001143C000684DB9E644
:1097F0001D0000220023C0E6002D5BD10D000543B3
:1098000000D1E2E65D1C00D1B0E0614DAE421FD058
:10981000DB43382B71DC1F2B00DD96E020250F0089
:10982000ED1AAF40B9460700AA46DF404D463D431A
:109830002F005546A840D940451EA84188440743FB
:10984000BF18974292415142414435003AE664467E
:1098500035004146100085E60B000343002D00D083
:1098600063E6002BF5D04346134300D17AE6871810
:109870008742804107224144404209183A400B0286
:1098800000D4D5E6434B01351940C9E5380069E6F7
:109890001E004746203EF740BC46202B04D0402601
:1098A000F31A46469E403243170063467A1E97419C
:1098B0001F4302E6364DAE42CAD080252D045B42DE
:1098C0002943A6E70843411E8841A6E6002B00D1A4
:1098D00048E6871A4346B842B641CB1A76429E1BE9
:1098E00033024BD5171A4346BA429241591A524293
:1098F000891A072264463A4092E501430F00791E17
:109900008F419DE71C000F00203CE740202B03D037
:109910004024E31A99400843411E884138437CE6BD
:109920000022002425E6171A4346BA429241591AEA
:109930005242891A6446350043E541461000144DF1
:1099400010E680220024120380E61D000F00203D57
:10995000EF40BC46202B03D04025EB1A994008432A
:1099600007006346781E87411F4369E787189742BF
:109970009B4141445B42C9183500A3E53B0033439A
:10998000CED0072231003A4052E600231A00F4E517
:10999000FF070000FFFF7FFFF0B55746DE464E464B
:1099A0004546E0B5834607000E03480085B0924661
:1099B0001C00360B400DCD0F002800D19DE0954BCB
:1099C000984239D08023F6001B041E43924A7B0F35
:1099D00033439946944603006344009300230026D2
:1099E000FF00029323031B0B98466300E40F5246CB
:1099F0005B0D019400D1B3E086498B4200D19EE01B
:109A00004246D100802212040A435146490F1143B5
:109A10008B46814952468C4600996344CB1A0021FB
:109A2000D20000932B0063409A460F2E00D905E127
:109A30007A4BB6009B599F465B463343994600D00C
:109A4000B8E002230826002700900293CAE7CB461D
:109A50003A0002990195019B9A46022927D00329D1
:109A600000D180E2012944D06D49009B8C466344BB
:109A70001C00002C38DD530700D013E2D2085B46EF
:109A8000DB0109D55946674B19408B468021C90037
:109A90008C46009B63441C00634B9C4207DC5B4686
:109AA00064055F075B0217431B0B620D02E0002396
:109AB0000027584A00211B031C0B0B0D1B052343D9
:109AC00014055A4A380013401C4353466400DB0710
:109AD00064081C43210005B03CBC90469946A24650
:109AE000AB46F0BD0122524201231B1B382B00DC88
:109AF000ADE1002200230027DCE75B4633439946B3
:109B00005ED0002E00D18AE1300001F0E7F90300B9
:109B10000B3B1C2B00DD7BE11D22D31A5A460100B2
:109B2000DA4008398E4013005F46334399468F4030
:109B30003F4B00261B1A00930023029352E7414635
:109B400053460B433B499B468C46009B6344009322
:109B50005B46002B3BD1022300221E43022161E71A
:109B6000434613439B4637D04346002B00D162E166
:109B7000404601F0B3F903000B3B1C2B00DD53E121
:109B800002004146083A914088461D21CB1A5146B1
:109B9000D9400B0041460B439B46534693401A0065
:109BA000009B25499C46604403008C466344009317
:109BB000002137E70323B14600900C26029311E7FA
:109BC0000023009301330426002702930AE70323AE
:109BD000C3461E43032125E701331E430022012112
:109BE00020E700239A46802300271B03094A61E7E8
:109BF000802349461B03194200D1E2E0594619422D
:109C000000D0DEE00B431B0317001B0BA246014AEA
:109C100050E7C046FF07000001FCFFFFD0DB00005B
:109C2000FF030000FFFFFFFEFE070000FFFF0F80A5
:109C30000DFCFFFF01F8FFFFF3030000D94500D939
:109C4000CBE000D1C6E03C0048460027009B013B2A
:109C500000935B46160E1B021E4313029846330404
:109C60001B0C9946310C0191FFF798F84A46424384
:109C70000B04210C050019438A4207D98919013DBB
:109C80008E4203D88A4201D9851E8919881A019902
:109C9000FFF784F809048C464A462104644642438F
:109CA000090C030021438A4204D98919013B8E42E1
:109CB00000D8F1E02D041D43AB464346891A4246C5
:109CC000280C12041D0C5B46140C22001B041B0CF8
:109CD0005A4303946B434443029568431B19150C84
:109CE000EB189C4203D980246402A44660441C0CF7
:109CF00015041B042D0C20185D19814277D373D0F5
:109D00000C1AA24A7D1BAF42BF419446009B7F4282
:109D10006344E01B1C00864200D1DBE00199FFF7A1
:109D20003DF84A4642430B04290C070019438A4276
:109D300007D98919013F8E4203D88A4201D9871E6B
:109D40008919881A0199FFF729F809044A468946B2
:109D500029044D464243090C030029438A4207D98E
:109D60008919013B8E4203D88A4201D9831E891981
:109D70003F04891A3A00039F1A43380013041B0C4E
:109D8000584381460298150C6F4343434543484668
:109D9000000C8446DB1963449F4203D980204002B3
:109DA0008446654448461F0C00041B04000C7D19C2
:109DB0001818A94200D284E000D17FE001231A43A1
:109DC00057E680234A461B0313431B031B0BAA467B
:109DD0006F4A6FE6BA4200D935E74B46DC075808B0
:109DE0007B081C43FF0734E70024AF4289D2474475
:109DF0004745A4415B466442A4196418013BA6424E
:109E00001ED2A0426DD800D1B6E0241A9B4678E756
:109E100003005A46283B9A400027914688E6584658
:109E200001F05CF8203072E603005246283B9A406D
:109E300093460022B4E6504601F050F820309AE6EE
:109E4000A642E2D1B845DCD9341A9B4659E71F2B0C
:109E500065DC504C0099A4465C46614408008C4087
:109E600011008240D940501E82410C4314435A468F
:109E7000DA401300620709D00F222240042A05D0DD
:109E80002200141D9442894149425B181A0262D58E
:109E90000122002300270DE68A4200D80AE7831E2C
:109EA000891907E70F231340042B00D1E6E5171D9E
:109EB0009742924153429B44FA08E0E5002800D1C2
:109EC000D7E57118531EB14227D3A94215D358D0F4
:109ED0001A0073E7002B00DC04E6012300229B44F8
:109EE000CDE502234744474589415B429C464942B0
:109EF00089190C19E344241A03E743465F004745D8
:109F00009B41B8465B429E19023A8919A94200D08A
:109F100054E7404500D051E7ABE51A00F6E71F21B2
:109F20005F4649420C1BE740202B07D01A49009B93
:109F30008C46634418005B4683401A43501E82419E
:109F40003A4307270023174009D00F21002311406F
:109F50001400042995D122005F075B021B0BD20875
:109F600017430022A6E5802359461B030B431B031E
:109F700017001B0B064A9DE5BD42B2D89B46002444
:109F8000BFE68045B9D31A00C3E7C046FF0300000F
:109F9000FF0700001E0400003E040000F0B54F461D
:109FA0004646D6468446C0B58046194E18030F0370
:109FB0004D00000B5C0082463F0B6D0DC90F9146B2
:109FC000640DDB0F0120B5420AD0B44203D0A54294
:109FD00001D157450CD01CBC90469946A246F0BD15
:109FE00066463E43F7D1AC42F5D154461443F2D114
:109FF0000120C845EFD1994207D0002DEBD163462F
:10A000001F433800471EB841E5E70020E3E7C0469C
:10A01000FF070000F0B54F464646D6464D00C0B596
:10A020000E03C90F8A462C491F035C008046360B7D
:10A030006D0D91463F0B640DDB0F8D421ED08C429F
:10A0400016D0002D1ED130438446002C01D13A4356
:10A0500023D06246002A1AD09A4529D051460220C0
:10A060000139084001381CBC90469946A246F0BD13
:10A0700039001143E5D002204042F4E73043FAD1E1
:10A08000AC420FD0002C0FD13A43E7D00CE00122B4
:10A09000013B934318000130E5E763460020002BA5
:10A0A000E1D0DBE73A43E6D19A45D7D1A542D5DCEA
:10A0B000A54205DBBE42D1D808D00020BE42D2D294
:10A0C00050460123013898430130CCE7C845C5D834
:10A0D0000020C845F4D3C6E7FF070000F0B54F469F
:10A0E0004646D6464D00C0B50E03C90F8A462E49D6
:10A0F0001F035C008046360B6D0D91463F0B640DCF
:10A10000DB0F8D4218D08C4211D0002D18D1304376
:10A110008446002C1ED13A431CD163460020002BFC
:10A1200030D0514602200139084001382AE0390078
:10A130001143EAD0022025E03043FBD1AC4226D0C7
:10A14000002C26D13A4324D151460220013908403F
:10A15000013817E06246002A0FD09A45E1D1A542A6
:10A1600005DBBE42DDD819D00020BE420AD25046DF
:10A17000012301389843013004E00122013B93435D
:10A18000180001301CBC90469946A246F0BD3A43E7
:10A19000D0D19A45C5D1A542C3DCE0E7C845C0D8B7
:10A1A0000020C845E3D3EDE7FF070000F0B55746B0
:10A1B000DE464E464546E0B5834606000F0348009E
:10A1C00087B092461D003F0B400DCC0F002800D1F8
:10A1D0006FE0DE4B984238D08023FF001B041F4302
:10A1E000730F3B430193DA4B0027994600239B46AC
:10A1F000F60081442B0369001B0B52469846490D1B
:10A20000ED0F002900D185E0D04B994200D173E0D9
:10A210004346DA0080231B0413435246CC48520FB6
:10A2200084461343524600206144D20089442100F1
:10A23000694000918C46012149448A460F2F00D97C
:10A2400090E0C449BF00CF59BF465B463B430193F2
:10A2500000D06AE102230827002681469B46C9E711
:10A2600032005846019B61460091022800D175E0FA
:10A27000032800D1FEE1012800D02CE100230027B3
:10A28000002600253F032A0D3F0BB34812053A4331
:10A2900002401B051343009A5B00D1075B080B4388
:10A2A0003000190007B03CBC90469946A246AB4628
:10A2B000F0BD5B463B43019300D12FE1002F00D15D
:10A2C000A5E1380000F00AFE03000B3B1C2B00DD6B
:10A2D00096E11D22D31A5A460100DA405E4608393B
:10A2E0008F4013008E403B4301939C4B00271B1A69
:10A2F000994600239B467DE7414653460B439349CD
:10A300008C46E144002B00D01AE1022202201743C0
:10A3100000228CE7134300D10DE14346002B00D10E
:10A3200081E1404600F0DAFD02000B3A1C2A00DD14
:10A3300072E10100434608398B4098461D239A1A62
:10A340005346D3401A004346134352468A40494677
:10A35000081A824989468144002068E77B4B002720
:10A3600000268EE7140C1204120C1100370C360470
:10A37000350C794328008C462E00604360448346A8
:10A3800056432100300C80465846794340440291A0
:10A39000844506D98846802149028C46E0444146DE
:10A3A00002913604010C360C00048B4681191E0CF8
:10A3B0001B041B0C0391190079438C46280075433C
:10A3C0006544A8465843050C45447743A94203D940
:10A3D000802149028C466744290C8C4639000004D0
:10A3E000000C2D042D186144AB440591594604918D
:10A3F00001990F043F0C080C390051434243904629
:10A4000002008C46090C8B4662437C4344445C4406
:10A41000A04503D98021490288464244210C884640
:10A4200061460904090C8C46390059434343704383
:10A430007E430F0CF6182404BE19644442448C4633
:10A44000B34203D980235B0298464044029B614695
:10A450009846049B370443449B46AB45AD416B4251
:10A460000D0405992D0C8C467F196744FD18A846EC
:10A470005D462D19A542A44193466442A446C344B7
:10A48000DC448F42BF4198459B4193459241A4458E
:10A49000A4415B427F421F43360C52426442BF19C3
:10A4A0002243BF18624638184302D20D0399134362
:10A4B0006A020A43501E82416146ED0D2A434E0254
:10A4C0003243D90100D4B3E00126500832400243A0
:10A4D000DE0732435B08224C5444002C62DD5107F6
:10A4E00009D00F201040042805D0101D9042924141
:10A4F00052429B180200D90104D580241948E40077
:10A50000034054441848844200DD27E75E075B029D
:10A51000D2081F0B630516435B0DB2E60023994674
:10A520000133042700269B4664E6032301978146F6
:10A530000C279B465EE6012201201743002276E6A7
:10A54000032303201F43434671E6C046FF07000074
:10A5500001FCFFFF10DC0000FFFF0F800DFCFFFF80
:10A56000FF030000FFFFFFFEFE070000002380271F
:10A5700000933F030026434B83E6019B3200A44631
:10A58000584670E6AC466EE6802701993F03394293
:10A590002DD03B422BD11F433F033F0B00951600AC
:10A5A000384B6EE601252D1B382D00DD66E61F2D8C
:10A5B00040DC35481C005044160082408440EE4088
:10A5C000501E824134431443EB40620709D00F22EE
:10A5D0002240042A05D02200141D944280414042AA
:10A5E0001B181A023ED501230027002649E68027C2
:10A5F000019B3F031F433F033F0B0094214B40E669
:10A6000003005A46283B9A40002601926DE65846C0
:10A6100000F064FC203057E603005246283B9A4085
:10A620001300002293E6504600F058FC20307BE6F1
:10A63000CA4650E71F201E004042041BE640202D62
:10A6400003D0124C5444A3401A43501E824132435B
:10A6500007260027164009D00F20002310401400C1
:10A660000428B9D122005E075B021F0BD2081643F3
:10A67000002306E680273F031F433F033F0B1600DE
:10A68000004BFEE5FF0700001E0400003E04000032
:10A69000F8B557464E464546DE460C000903E0B580
:10A6A000490A460F5F0031431E03DB0F760A9B46C3
:10A6B000530F3343C84E6500C000E40FD2006D0D48
:10A6C000A24681467F0D9C469046B74200D1B9E034
:10A6D0005B46012673409B46EE1BA34500D183E0F9
:10A6E000002E63DD002F00D0B1E06346134300D19C
:10A6F00023E1731E002B00D0BAE1861A6346B042F4
:10A7000080410125C91A4042091A0B0200D447E1D1
:10A7100049024B0A98464346002B00D189E1404646
:10A7200000F0DCFB0300083B1F2B00DD7CE1202256
:10A730003000D21A4146D040994002009E400A4360
:10A740009D4200DD6AE15D1B6B1C1F2B00DD94E167
:10A75000202110003500C91A8E40DA408840DD40C3
:10A76000711E8E4111000722284300250643324006
:10A77000002A09D00F233340042B05D0331DB342E8
:10A78000B641764289191E000B0200D43DE26A1CD4
:10A79000914B55056D0D9A4200D119E18F4AF6088B
:10A7A0000A40570752023743120B9BE0002E00D09D
:10A7B000C5E06E1C7605760D012E00DC48E167468B
:10A7C000861ACB1BB042BF417F42B8461F004346AA
:10A7D000FF1A3B00B8461B0200D55FE137439AD110
:10A7E00000220024002579E0002E00DCFAE0002F92
:10A7F00000D18DE0784B9D4267D0802367461B04D3
:10A800001F43BC46382E00DC52E1634613435A1EF8
:10A8100093411E1886428041404209180B0200D421
:10A82000BEE06D4B01359D4200D1D2E06B4A73080A
:10A830000A4001210E401E435108D30707221E4340
:10A84000324095E71E00164300D045E740E7624BD3
:10A850009D423AD0802367461B041F43BC46382ED6
:10A8600000DDEBE01F2E00DC3AE133006746203BC1
:10A87000DF403B00202E05D04027BF1B6646BE4070
:10A88000324390464646721E96413343DAE0002B2F
:10A8900000D114E26346134300D168E180234E07E0
:10A8A000C008C9081B030643194208D06046C00807
:10A8B000184204D163460100D2085E071643F30034
:10A8C0009946C900720F444D11434B46DE08424B76
:10A8D0004F073743CA089D4200D16EE012036D0551
:10A8E000120B6D0D00211203130B0A0D12051A43F2
:10A8F0003B4B2D0513402B435B00E4075B082343D0
:10A90000380019003CBC90469946A246AB46F8BDBB
:10A910006346134311D0731E002B00D007E1861845
:10A920008642804161444042091801250B0237D517
:10A9300002257BE73E00614691463500C5E75C464F
:10A94000002D00D0E1E00B000343F3D0731C00D1D5
:10A95000ACE1214B9F4200D13AE1F343382B00DDBB
:10A960006FE11F2B00DD8CE120250E00ED1AAE40BB
:10A97000B0460600AA46DE40454635432E00554601
:10A98000D940A8406346451EA8415B1A9C46304307
:10A99000161AB242924163465242991A3D00B4E6F9
:10A9A00007223240002A00D0E4E60B4BF6084F079E
:10A9B0003743CA089D4200D090E73B00134300D1C3
:10A9C000A6E180231B031A431203120B024D89E7F1
:10A9D00015000022002785E7FF070000FFFF7FFF2B
:10A9E000FFFF0F80002E00D0C7E06B1C5E05760DC8
:10A9F000012E00DCF0E0C84DAB4200D1B9E0851873
:10AA00000A00854289416244494251180722CE0713
:10AA10006D082E43490832401D00A9E6BF49ED1AD2
:10AA2000114007223240A3E6320028388240002637
:10AA300086E6300000F052FA203073E66346134396
:10AA40005A1E9341C61AB04280414042091A5CE640
:10AA50000E00674606431743002D5ED1002E00D03E
:10AA6000F3E0002F00D11EE15C46614691462CE7E1
:10AA7000A94FBE427BD01E00F1E610001F3DE8400A
:10AA8000202B03D04021CB1A9A401643731E9E41BF
:10AA90000722064332400021002583E7161A634649
:10AAA000B2428041591A40420B1A98465C4632E63F
:10AAB0001F2E00DDABE02027BB1B9A46634657469E
:10AAC000BB40994613004F46F3401F433B00574697
:10AAD000BA40571EBA4113436246F240891898E6BD
:10AAE0002027BB1B9A4663465746BB409946130036
:10AAF0004F46F3401F433B005746BA40571EBA41EA
:10AB000013436246F240891A9CE7834B9F425FD011
:10AB100080252D047342294320E7002E0CD1002FFD
:10AB200000D1D0E05C46614691467B4DCDE67A4F40
:10AB3000BE421CD01E0065E6002F18D0C0084E078C
:10AB400006438020C9080003014208D06346DC08A0
:10AB5000044204D12100DA46D2085E071643F3000E
:10AB6000994601245346C900720F11431C406A4D97
:10AB7000ABE61D0000220027B4E6002D59D10B00E2
:10AB8000034300D1D6E6731C00D1B2E0624B9F4272
:10AB90001ED0F343382B6FDC1F2B00DD97E0202500
:10ABA0000E00ED1AAE40B0460600AA46DE4045460D
:10ABB00035432E005546A840D940451EA8418C4437
:10ABC0000643B61896429241514261443D0025E643
:10ABD0003D006146914678E60B000343002D00D00E
:10ABE00055E6002BF5D06346134300D16DE6861879
:10ABF0008642804161444042091800220B0200D481
:10AC0000D0E6464B01351940B2E5B1465DE633006A
:10AC10006746203BDF403B00202E05D04027BF1B6E
:10AC20006646BE40324390464646721E96413343C6
:10AC3000EFE5394B9F42CBD080252D047342294349
:10AC4000A8E70843411E8841A2E6002F00D13CE658
:10AC50006346861ACF1AB0429B415B42FB1A984664
:10AC60001B024ED5161A6346B2429241591A5242FD
:10AC7000891A5C4600227BE501430E00711E8E415D
:10AC80009FE71D000E00203DEE40B046202B04D073
:10AC90004025EB1A99400843814648464346411EE9
:10ACA0008841184374E60022002417E6161A63460A
:10ACB000B2429241591A5242891A3D0025E5614635
:10ACC0009146154D01E680220024120379E61D000D
:10ACD0000E00203DEE40B046202B04D04025EB1A5C
:10ACE0009940084381464E464346711E8E411E439D
:10ACF00067E7861896429B4161445B42C9183D0054
:10AD00008CE547463743CED007224146324049E6DC
:10AD100000273A00E6E5C046FF070000FFFF7FFF7F
:10AD200070B50C4E0D031C0349005B002D0B490D43
:10AD3000240B5B0DB14208D0064900208B4203D1A1
:10AD400014432000441EA04170BD05430120002D86
:10AD5000FAD1F1E7FF07000030B5144D0A034B00AC
:10AD6000120B5B0DC90F0024AB4211DD104CA34246
:10AD700010DC8024640322430E4CE41A1F2C0CDDEB
:10AD80000D48C31ADA4013005C42002900D11C00B0
:10AD9000200030BD094BCC18FAE7094DE040AC4625
:10ADA00063449A4013000343EEE7C046FE030000ED
:10ADB0001D0400003304000013040000FFFFFF7FA8
:10ADC000EDFBFFFF70B500282DD0C317C5185D40FF
:10ADD000C40F280000F082F8154B1B1A5B055B0DB1
:10ADE0000A2815DD0B38854000222D032D0B00218C
:10ADF00010002D030A0D2D0B12052A430D4D1B05C6
:10AE00002A4013435B00E4075B082343190070BD2D
:10AE100002002900153291400A000B21081AC54092
:10AE20002D032D0BE3E70024002300250022DEE79D
:10AE30001E040000FFFF0F804100090E4B1C70B57F
:10AE4000DBB24602750AC40F012B14DDE0239B0020
:10AE50006D07360BCB1800210A0D280012051C4D7A
:10AE600032435B052A405B0813435B00E4075B0841
:10AE70002343190070BD002914D1002D1ED02800D5
:10AE800000F02CF80A281CDC0B232A001B1ADA40DD
:10AE9000030015339D400F4B12031B1A5B05160B65
:10AEA0005B0DD8E7002D06D0320B802636036D07E8
:10AEB0001643094BCFE7084B0026CCE700230026BA
:10AEC000C9E703002A000B3B9A400025E3E7C04690
:10AED000FFFF0F8089030000FF0700001C210123F2
:10AEE0001B04984201D3000C10391B0A984201D36D
:10AEF000000A08391B09984201D30009043902A24B
:10AF0000105C40187047C0460403020201010101B1
:10AF1000000000000000000030B51C00094B0500D7
:10AF20001B6885B0D868084B002A01D1074B1A006E
:10AF30000292019300912B002200054900F026F8AF
:10AF400000F0A6FD8000002050DC000033CA0000A5
:10AF50005DDC0000014B18687047C046800000208F
:10AF6000084B10B50400002B02D0002100E000BF08
:10AF7000054B1868836A002B00D09847200001F029
:10AF80005DFBC046000000008CDC00000EB403B581
:10AF9000010003AB044804CB0068019300F076F88D
:10AFA00002B008BC03B018478000002070B500262E
:10AFB0000C4D0D4C641BA410A64209D1002601F0D3
:10AFC0003FFB0A4D0A4C641BA410A64205D170BD7C
:10AFD000B300EB5898470136EEE7B300EB589847BB
:10AFE0000136F2E7500200205002002050020020FB
:10AFF00060020020002310B59A4200D110BDCC5C45
:10B00000C4540133F8E710B5884202D98B1898422E
:10B0100003D3002307E08B5C8354013AFBD210BDBD
:10B02000CC5CC45401339A42FAD1F8E703001218F9
:10B03000934200D1704719700133F9E7936810B556
:10B04000013B9360002B04DA9469A34207DB0A29D1
:10B0500005D01368581C10601970080010BD00F06E
:10B060004BFC0100F9E7F8B506000F001400D518F5
:10B07000AC4201D1002007E021783A003000FFF710
:10B08000DDFF0134431CF3D1F8BD0000F0B59FB0E3
:10B0900002900F0016000593002805D083690493E1
:10B0A000002B01D100F0F4FD7B4B9F425BD1029B52
:10B0B0005F68BB891B0762D53B69002B5FD000230B
:10B0C00006AC6361203363761033A37635002B78AA
:10B0D000002B01D0252B5CD1AB1B04930CD032008C
:10B0E00039000298FFF7BFFF431C00D1C4E062693A
:10B0F000049B9446634463612B78002B00D1BBE032
:10B10000012200235242626002A9543252186E1C7E
:10B110002360E360A3601370A365317805225F4864
:10B1200000F0D4FE751C002835D12268D30604D562
:10B13000532302A95B1820211970130704D5532348
:10B1400002A95B182B21197033782A2B2CD03500DB
:10B1500000210A20E3682A786E1C303A092A64D953
:10B1600000292ED026E04E4B9F4202D1029B9F68C1
:10B170009FE74C4B9F429CD1029BDF6899E73900C7
:10B18000029800F00FFC002899D0012040421FB027
:10B19000F0BD01359BE7414B2268C01A0123834073
:10B1A000134323602E00B8E7059B191D1B6805910A
:10B1B000002B01DB099304E05B42E36002231343AD
:10B1C00023602B782E2B0AD16B782A2B35D1059B47
:10B1D00002351A1D1B680592002B2BDB0793324E9C
:10B1E00029780322300000F071FE002806D04023A9
:10B1F000801B83402268013513432360297806228F
:10B200002A486E1C217600F061FE00283AD0284BB7
:10B21000002B25D10722059B073393430833059361
:10B220006369039A9B18636150E7434301219B18AC
:10B23000350090E701235B42D0E700230A201A0083
:10B240000135636029786E1C3039092903D9002B38
:10B25000C5D00792C3E74243012352183500F1E7F6
:10B2600005AB00933A00134B2100029800E000BFA9
:10B270000390039B0133D3D1BB895B0600D584E7E0
:10B280000B9884E705AB00933A000A4B2100029823
:10B2900000F080F8ECE7C046E4DC000090DC000041
:10B2A00004DD0000C4DC000096DC00009ADC000035
:10B2B0000000000067B00000F7B5150001938A6830
:10B2C0000B6900900C00934200DA130022002B60FF
:10B2D00043321278002A01D001332B6023689B0689
:10B2E00002D52B6802332B60062723681F4027D026
:10B2F000230043331B785A1E93412268920630D4B0
:10B300002200019943320098089EB047431C25D083
:10B31000062320682A68E16803400025042B03D136
:10B320008D1AEB43DB171D40A3682269934201DDB0
:10B330009B1AED180027BD4220D1002010E00137F4
:10B34000E3682A689B1ABB42D2DD2200012319322E
:10B3500001990098089EB047431CF0D1012040425B
:10B36000FEBD3020E1184331087021005A1C4531E0
:10B370000978A218433202331170C1E72200012379
:10B380001A3201990098089EB047431CE6D0013755
:10B39000D1E70000F0B589B004920A00433205936A
:10B3A000039002920A7E0C000E9B6E2A00D186E06A
:10B3B0001FD8632A33D008D8002A00D18CE0582A3D
:10B3C0004DD0250042352A7030E0642A01D0692A28
:10B3D000F7D1196825680A1D280629D508681A605A
:10B3E000002803DA2D23029A404213706B4E0A277D
:10B3F0004FE0732A74D008D86F2A1FD0702AE0D18A
:10B40000202209680A43226003E0752A16D0782AB0
:10B41000D7D12200782145321170614E22E02500FB
:10B420001A684235111D196013682B70012365E0FD
:10B4300008681A606906D3D500B2D1E71968256893
:10B44000081D186008682E0605D5544E08276F2A77
:10B450001BD00A2719E06D06F7D580B2F5E7453114
:10B460004E4E0A7018682268011D006819601506A2
:10B4700021D5D30702D520231A43226010270028A4
:10B4800003D1202322689A43226023000022433301
:10B490001A706368A360002B58DB04222168914373
:10B4A0002160002854D1029D002B5AD0250033780A
:10B4B00042352B7055E05506DBD580B2D9E71A68C6
:10B4C0000D68101D4969186013682E0601D51960B2
:10B4D00002E06D06FBD519800023029D23614FE039
:10B4E0001A68111D1960156800216268280000F0B3
:10B4F000EDFC002801D0401B6060636823610023DD
:10B50000029A13703CE023692A0004990398059D70
:10B51000A847431C3ED023689B0715D4079BE068CF
:10B52000984239DA180037E02200012319320499D1
:10B530000398059EB047431C2CD00135E368079A59
:10B540009B1AAB42F0DCE9E70025F7E70028ADD015
:10B55000029D3900FDF722FC735C013D2B70002831
:10B56000F7D1082F09D12368DB0706D56368226964
:10B57000934202DC3023013D2B70029B5B1B236155
:10B58000059B07AA00932100049B0398FFF794FEF4
:10B59000431CB8D10120404209B0F0BDA1DC00003D
:10B5A000B2DC00000D4B70B51C680500A36B002BCE
:10B5B0000FD1182000F06EFC094BA0630360094B0B
:10B5C00001224360084B83600B23838100230261C7
:10B5D00043610022A36B1D615A6170BD8000002091
:10B5E0000E33CDAB34126DE6ECDE0500124B10B518
:10B5F0001C68A36B002B0FD1182000F04BFC0F4BE5
:10B60000A06303600E4B012243600E4B83600B234B
:10B610008381002302614361A46B0B4A2069616945
:10B620000A4BFDF7F7FC01220023801859412061E5
:10B6300061614800400810BD800000200E33CDAB92
:10B6400034126DE6ECDE05002D7F954C2DF451583B
:10B650000CB430B5164B9DB00C1E1D6808DA8B2358
:10B6600001202B6040421DB030BC08BC02B018471E
:10B67000822302A99B008B810023029008619C42D7
:10B6800000D0631E8B604B6101235B42CB81209A0B
:10B6900021AB2800019300F055FD431C01DA8B23F8
:10B6A0002B60002CDFD00023029A1370DBE7C0462A
:10B6B000800000200EB400B50B499CB01DAB029079
:10B6C0000690079104910948094904CB0591006847
:10B6D00002A9019300F036FD0023029A13701CB0FA
:10B6E00008BC03B01847C046FFFFFF7F8000002062
:10B6F0000802FFFF020010B51378541C002B05D17F
:10B70000CC5CD4540133002CFAD110BD2200F3E7F5
:10B71000C9B20378002B04D08B4200D170470130AE
:10B72000F7E74B42594149420840F7E702780B7866
:10B73000002A03D0013001319A42F7D0D01A704765
:10B740000023C25C0133002AFBD1581E704700233E
:10B7500030B59A420AD0013AC45CCD5CAC4204D107
:10B76000934202D00133002CF6D1631B180030BD88
:10B7700030B50500002A00D130BD0C78013A6B1CB1
:10B780002C700131002C05D19A189A42F4D01C700B
:10B790000133FAE71D00EDE710B50378002B0FD158
:10B7A0000B785A4253415B42184010BD0023CA5CDB
:10B7B000002AFAD0C45C944201D10133F7E701308A
:10B7C0000378002BF2D11800EFE70000F0B51F005E
:10B7D0000E0087B00590019102920C98347800F029
:10B7E000EAFA082200194378751C134036D12D2C33
:10B7F00036D1B51C74780126002F62D0102F09D1E4
:10B80000302C07D120222B789343582B54D110276A
:10B810006C7802352D4B3900F31818000393FDF7AF
:10B82000BDFA049101210023494202008C46180010
:10B830002100303909291AD80C00A74223DD591CF0
:10B8400009D06346824206D302D10499A14202DBA9
:10B850000123784320182C780135E9E72E00BCE756
:10B860002B2C01D01E00C7E7B51C7478FAE7210025
:10B870004139192901D8373CDFE7210061391929FD
:10B8800001D8573CD9E75A1C08D1059A23331360D5
:10B89000029B0398002B09D107B0F0BD002E00D009
:10B8A0004042029A002AF7D0002B01D06B1E019370
:10B8B000029B019A1A60EFE73024002FAAD10827D3
:10B8C000A8E7302C9ED00A27A4E7C046FFFFFF7FE1
:10B8D00037B51300064A05001068046A002C00D131
:10B8E000044C0A0000942900FFF770FF3EBDC046DB
:10B8F00080000020E4000020F8B505000E001400D0
:10B90000002804D08369002B01D100F0C1F9224B3B
:10B910009C422DD16C68A369A360A3891B0731D514
:10B920002369002B2ED023682269F7B2981A636925
:10B93000F6B2834205DC2100280000F03BF9002824
:10B9400026D1A3680130013BA36023685A1C226002
:10B950001F706369834204D0A389DB071AD50A2EBE
:10B9600018D12100280000F025F9002812D00FE09E
:10B970000A4B9C4201D1AC68CDE7094B9C42CAD12D
:10B98000EC68C8E72100280000F00CF80028CAD0B5
:10B99000012676423000F8BDE4DC000004DD000042
:10B9A000C4DC0000364B70B51D6806000C00002D8D
:10B9B00005D0AB69002B02D1280000F069F9314BAA
:10B9C0009C420FD16C680C23E25E93B219072DD410
:10B9D000D90611D409230120336037331343A381DF
:10B9E000404270BD284B9C4201D1AC68EBE7274B2D
:10B9F0009C42E8D1EC68E6E75B0713D5616B002950
:10BA000008D023004433994202D0300000F06AFA93
:10BA1000002363632422A3899343A38100236360EB
:10BA2000236923600823A2891343A3812369002B80
:10BA30000BD1A0218022A389890092000B40934260
:10BA400003D02100300000F0E1F90123A289134066
:10BA500011D00023A36063695B42A36100202369C6
:10BA60008342BED10C23E25E1306BAD540231343B2
:10BA7000A3810138B5E7920700D46369A360EDE7BD
:10BA800080000020E4DC000004DD0000C4DC0000D5
:10BA900010B5062000F090FC012000F0CFFD000062
:10BAA000F7B58A8905000C00130760D44B68002B9A
:10BAB00004DC0B6C002B01DC0020FEBDE76A002FCC
:10BAC000FAD000232E682B6080235B01216A1A4084
:10BAD00034D0606DA3895B0706D56368C01A636BB9
:10BAE000002B01D0236CC01A0200216A0023280019
:10BAF000E76AB847A189431C06D12B681D2B30D8B3
:10BB00002B4ADA40D3072CD50023636023692360D6
:10BB1000CB0405D5431C02D12B68002B00D16065F6
:10BB2000616B2E600029C7D023004433994202D0B4
:10BB3000280000F0D7F900206063BEE70123280049
:10BB4000B847431CC6D12B68002BC3D01D2B01D096
:10BB5000162B01D12E60AFE74023A2891343A381A6
:10BB6000ABE740230B430120A3814042A5E70F69C7
:10BB7000002FA1D00B680F60DB1B019300239207FD
:10BB800000D14B69A360019B002B00DC94E7019B73
:10BB90003A00216A2800A66AB047002803DC402347
:10BBA000A2891343DFE7019B3F181B1A0193EAE7C1
:10BBB000010040200B6970B505000C00002B01D17D
:10BBC000002070BD002804D08369002B01D100F053
:10BBD0005FF80B4B9C4209D16C680C22A35E002BD2
:10BBE000EED021002800FFF75BFFEAE7054B9C42FF
:10BBF00001D1AC68F1E7044B9C42EED1EC68ECE774
:10BC0000E4DC000004DD0000C4DC0000002310B50B
:10BC1000040003604360836081814366C2810361E5
:10BC200043618361190008225C30FFF7FFF9054B7F
:10BC300024626362044BA362044BE362044B2363FC
:10BC400010BDC046F9C3000021C4000059C4000063
:10BC500085C4000010B5024900F08CF810BDC04644
:10BC6000B5BB000070B568254A1E55430E0029007B
:10BC7000743100F081F9041E08D000212A0001600F
:10BC800046600C30A0606832FFF7D0F9200070BD2C
:10BC9000836913B50400002B28D18364C364036552
:10BCA000134B144A1B6882620193984201D101230D
:10BCB0008361200000F020F86060200000F01CF894
:10BCC000A060200000F018F80022E0600421606805
:10BCD000FFF79CFF01220921A068FFF797FF0222CE
:10BCE0001221E068FFF792FF0123A36113BDC04654
:10BCF0008CDC000055BC0000F8B51C4B07001E682A
:10BD0000B369002B02D13000FFF7C2FF4836B46898
:10BD10007368013B04D53368002B07D03668F6E71B
:10BD20000C22A55E002D0DD06834F2E70421380006
:10BD3000FFF798FF30600028F0D10C2304003B602F
:10BD40002000F8BD20000A4B656625606560A5608F
:10BD5000E36025616561A561082229005C30FFF779
:10BD600065F96563A563A564E564E9E78CDC00001B
:10BD70000100FFFFF7B504000700002601914834D9
:10BD8000002C01D13000FEBD6368A5680093009BC4
:10BD9000013B009301D52468F2E7AB89012B08D958
:10BDA0000E22AB5E013304D029003800019B984776
:10BDB00006436835EBE7EC300068704770B50E005D
:10BDC0001D000E23C95E96B01400002907DA002377
:10BDD0002B60B3891B0611D48023DB000FE06A4679
:10BDE00000F088FB0028F2DBF022019B12021340D6
:10BDF000054A9B185A4253412B60EDE7402300202F
:10BE0000236016B070BDC04600E0FFFFF7B5022604
:10BE10008B8905000C00334206D023004733236092
:10BE2000236101236361F7BD01AB6A46FFF7C6FFDB
:10BE300000990700280000F09FF8002808D10C2284
:10BE4000A35E9A05EFD4032293431E43A681E4E741
:10BE50000F4BAB628023A28920601343A381009B18
:10BE600020616361019B002B0DD00E23E15E280051
:10BE700000F052FB002806D00322A38993431A0046
:10BE800001231343A381A0893843A081CBE7C04697
:10BE900055BC000010B5034B0100186800F06CF8A9
:10BEA00010BDC0468000002082B0002900D101A949
:10BEB000101E06D0002B06D013780B601078431E9E
:10BEC000984102B0704702204042FAE7C9B2821896
:10BED000904201D10020704703788B42FBD00130A3
:10BEE000F6E7000070B50500002910D00C1F23688C
:10BEF000002B00DAE418280000F034FB1D4A136818
:10BF0000002B05D163601460280000F02CFB70BD8D
:10BF1000A34209D9216860188342F3D118685B688D
:10BF200041182160EEE713005A68002A01D0A242AE
:10BF3000F9D919685818A0420BD120680918581867
:10BF400019608242E0D110685268411819605A6045
:10BF5000DAE7A04202D90C232B60D5E721686018EC
:10BF6000824203D1106852684118216062605C60AF
:10BF7000CAE7C0461C1C0020032370B5CD1C9D439E
:10BF8000083506000C2D1ED20C25A9421DD8300004
:10BF900000F0E8FA254A14682100002919D1244C40
:10BFA0002368002B03D1300000F0CAF9206029007B
:10BFB000300000F0C5F9431C2BD10C233000336056
:10BFC00000F0D1FA03E0002DDFDA0C23336000200B
:10BFD00070BD0B685B1B19D40B2B03D90B60CC18FD
:10BFE000256003E04B688C420DD11360300000F0F7
:10BFF000BAFA200007220B30231D9043C31AE7D062
:10C000005A42E250E4E763600C00EFE70C00496835
:10C01000C3E70323C41C9C43A042E1D0211A300093
:10C0200000F08EF9431CDBD1C7E7C0461C1C002082
:10C03000201C0020F8B507000D001600002905D1CE
:10C040001100FFF799FF04002000F8BD002A03D17A
:10C05000FFF748FF3400F7E700F086FA2C00B04203
:10C06000F2D231003800FFF787FF041EECD0290020
:10C070003200FEF7BFFF29003800FFF733FFE3E788
:10C08000F0B58E6885B007000C00039201939E42C4
:10C090003CD890238A89DB001A4234D003250969F1
:10C0A00023685B1A0293636902985D43EB0F5D1985
:10C0B000019B6D1001331B18AB4200D91D005305C5
:10C0C00032D529003800FFF757FF061E09D10C238F
:10C0D0003B6040230120A28940421343A38105B065
:10C0E000F0BD029A2169FEF785FFA389144A1A4020
:10C0F00080231343A381029B2661F61826606561A5
:10C10000019EED1AA560019B9E4200D9019E32005E
:10C1100003992068FEF777FFA36800209B1BA360AC
:10C1200023689E192660DAE72A003800FFF782FFAD
:10C13000061EE0D121693800FFF7D4FEC7E7C046EC
:10C140007FFBFFFFF0B59FB0029005938B890F0036
:10C1500016001B0611D50B69002B0ED14021FFF7ED
:10C160000BFF38603861002805D10C23029A013892
:10C1700013601FB0F0BD40237B61002306AC6361F8
:10C18000203363761033A37635002B78002B01D053
:10C19000252B46D1AB1B04930CD0320039000298FA
:10C1A000FFF76EFF431C00D1AEE06269049B94462A
:10C1B000634463612B78002B00D1A5E001220023AA
:10C1C0005242626002A9543252186E1C2360E3602E
:10C1D000A3601370A365317805225448FFF776FEFB
:10C1E000751C00281FD12268D30604D5532302A949
:10C1F0005B1820211970130704D5532302A95B187B
:10C200002B21197033782A2B16D0350000210A20F3
:10C21000E3682A786E1C303A092A4ED9002918D0D2
:10C2200010E00135B1E7414B2268C01A0123834079
:10C23000134323602E00CEE7059B191D1B68059153
:10C24000002B01DB099304E05B42E360022313430C
:10C2500023602B782E2B0AD16B782A2B35D1059BA6
:10C2600002351A1D1B680592002B2BDB0793304EFD
:10C27000297803223000FFF729FE002806D040234A
:10C28000801B8340226801351343236029780622EE
:10C2900028486E1C2176FFF719FE00283CD0264B5B
:10C2A000002B25D10722059B0733934308330593C1
:10C2B0006369039A9B18636166E7434301219B18F6
:10C2C0003500A6E701235B42D0E700230A201A00CD
:10C2D0000135636029786E1C3039092903D9002B98
:10C2E000C5D00792C3E74243012352183500F1E756
:10C2F00005AB00933A00114B2100029800E000BF0B
:10C300000390039B0133D3D1BB890B985B0600D408
:10C310002FE7012040422CE705AB00933A00074B82
:10C3200021000298FFF736F8EAE7C04690DC0000EB
:10C3300096DC00009ADC00000000000081C00000D4
:10C34000002370B5064C05000800236000F060F97A
:10C35000431C03D12368002B00D02B6070BDC04666
:10C36000982F002070B504000D001F2904D9162352
:10C3700003600120404270BD436C002B04D08A0052
:10C380009B181A68002A08D1200000F031F82A0012
:10C390000100200000F01AF8EDE70020012AEAD0A1
:10C3A000511C03D1162301302360E4E70024280048
:10C3B0001C6090472000DEE710B5034B01001868B1
:10C3C000FFF7D0FF10BDC04680000020002370B5ED
:10C3D000064C050008001100236000F001F9431C21
:10C3E00003D12368002B00D02B6070BD982F002054
:10C3F00010B500F0E5F810BD70B50C000E25495FD2
:10C4000000F0BAF8002803DB636D1B18636570BD8C
:10C41000A389024A1340A381F9E7C046FFEFFFFF5B
:10C42000F8B51F008B8905000C001600DB0505D54B
:10C430000E23C95E0022022300F080F8A389054A7A
:10C4400028001340A38132000E23E15E3B0000F080
:10C450002BF8F8BDFFEFFFFF70B50C000E25495F0C
:10C4600000F06CF8A389421C03D1054A1340A38154
:10C4700070BD802252011343A3816065F8E7C04676
:10C48000FFEFFFFF10B50E23C95E00F021F810BDCD
:10C490000B1E04D0FF2A04D98A2303608B3B1800AB
:10C4A00070470A700123FAE770B505000800110013
:10C4B0000022064C22601A0000F0B8F8431C03D199
:10C4C0002368002B00D02B6070BDC046982F002041
:10C4D000002370B5064C05000800236000F060F8EA
:10C4E000431C03D12368002B00D02B6070BDC046D5
:10C4F000982F0020002370B5064C0500080011009D
:10C50000236000F055F8431C03D12368002B00D0B2
:10C510002B6070BD982F0020002370B5064C0500DD
:10C520000800236000F054F8431C03D12368002B5B
:10C5300000D02B6070BDC046982F002070B505005C
:10C54000080011000022064C22601A0000F050F88A
:10C55000431C03D12368002B00D02B6070BDC04664
:10C56000982F0020704770470B1F1B68181F002B67
:10C5700001DA0B58C018704770B5050008001100AB
:10C580000022064C22601A0000F03AF8431C03D146
:10C590002368002B00D02B6070BDC046982F002070
:10C5A00058220120014B40421A607047982F00200A
:10C5B00058220120014B40421A607047982F0020FA
:10C5C00058220120014B40421A607047982F0020EA
:10C5D0005822024B00201A607047C046982F002056
:10C5E00058220120014B40421A607047982F0020CA
:10C5F00058220120014B40421A607047982F0020BA
:10C6000058220120014B40421A607047982F0020A9
:10C61000044A1368002B00D1034B1818106018004F
:10C620007047C046241C0020A02F00205822012063
:10C63000014B40421A607047982F0020FEE7C04629
:10C64000F8B5C046F8BC08BC9E467047F8B5C04671
:10C65000F8BC08BC9E46704764617461000000002D
:10C66000D4C60000EB010000DDC600001704000086
:10C67000E5C6000029070000ECC6000039080000EC
:10C68000F1C60000DF020000FCC6000083040000C9
:10C6900001C70000B10900000DC700001B02000027
:10C6A00017C700003106000025C700009F050000E5
:10C6B00072616E646F6D00616C6C006C617374000C
:10C6C00066616C7365007472756500252E31357373
:10C6D0002E2E2E006D616B654C697374006164646D
:10C6E0004C6173740064656C657465006A6F696E93
:10C6F00000636F707946726F6D546F0066696E6487
:10C70000006A6F696E537472696E677300756E6943
:10C71000636F6465417400756E69636F646553741B
:10C7200072696E6700667265654D656D6F7279003E
:10C73000E80F0000F80F0000121000009010000039
:10C74000C8100000FE100000361100005C1100004F
:10C7500098110000DA11000030120000741200007D
:10C76000E0120000281300004E13000086130000A2
:10C77000CC130000F213000020140000521400003B
:10C780008A1400000E150000D61500004C1600009B
:10C79000B816000004170000241700004617000018
:10C7A000F81700003E180000B6180000E80F00005F
:10C7B000E80F0000E41800004C190000D019000038
:10C7C000161A00005E1A0000D41A00004A1B00006E
:10C7D000921B0000D81B00000E1C0000541C00001F
:10C7E0009A1C0000E21C0000361D0000941D000091
:10C7F000D21D00003C1E0000721E0000BA1E000088
:10C80000021F00004A1F0000841F0000CC1F000010
:10C810001420000080210000E80F0000E80F000055
:10C820007C200000E80F0000B2200000DE200000A5
:10C830001421000040210000E80F0000E80F000074
:10C84000E80F0000E80F0000F62100003822000089
:10C85000E80F0000E80F00007E220000CE2200005A
:10C86000F4220000E80F0000E80F0000E80F0000CD
:10C87000222300005223000082230000B82300007E
:10C88000E223000018240000422400006A24000073
:10C8900092240000C2240000F22400001C250000A5
:10C8A00046250000A0250000CA250000E80F000072
:10C8B000E80F0000E80F0000E80F0000E80F00009C
:10C8C000FA25000026260000522600007E260000E1
:10C8D000AA260000E0260000162700004C270000D2
:10C8E00082270000AE270000DA2700001028000091
:10C8F000E80F0000E80F0000E80F0000E80F00005C
:10C90000E80F0000E80F0000E80F0000E80F00004B
:10C91000E80F0000E80F0000E80F0000E80F00003B
:10C92000E80F0000E80F00003C280000722800001B
:10C93000282564206974656D206C6973742900284A
:10C940006F626A65637420747970653A2025642982
:10C9500000537461636B20756E646572666C6F77EB
:10C9600000626F6F6C65616E006E756D626572005E
:10C97000737472696E67006C69737400070000005D
:10C9800003000000C6C9000095290000CEC90000C0
:10C99000452A0000D7C90000DD2A0000E0C90000D8
:10C9A00099290000000000000100000002000000C2
:10C9B00003000000040000000A0000006D696372BB
:10C9C0006F3A62697400686173546F6E6500706CD1
:10C9D0006179546F6E6500686173536572766F009C
:10C9E000736574536572766F00474320746F6F6B85
:10C9F0002025642075736563733B2066726565202E
:10CA0000256420776F726473003C496E74656765B6
:10CA1000723E003C4F626A6563743E003C4C697331
:10CA2000743E000D0A564D2050616E69633A202510
:10CA3000730D0A006D6973630000000081CA000075
:10CA4000B13700008ACA0000F93600008ECA000023
:10CA50004D36000096CA0000F3350000A0CA000061
:10CA600089350000ACCA00008B340000B6CA000053
:10CA700005380000C0CA0000613700006E756C6C9C
:10CA800000686578546F496E740073696E006A734C
:10CA90006F6E476574006A736F6E436F756E7400D6
:10CAA0006A736F6E56616C75654174006A736F6E60
:10CAB0004B657941740062797465436F756E7400DB
:10CAC00062797465417400003CCB00004D38000071
:10CAD00044CB0000513800004ECB00006F380000FE
:10CAE00057CB00007938000062CB0000833800008B
:10CAF0006ECB00008D3800007ECB00009738000020
:10CB00008ECB0000A1380000A3CB0000AB380000A2
:10CB1000B8CB0000B5380000C4CB0000BF3800001F
:10CB2000D4CB0000C9380000E0CB00005B38000027
:10CB3000EDCB0000653800006E65740068617357C6
:10CB40006946690073746172745769466900737449
:10CB50006F705769466900776966695374617475C7
:10CB600073006D7949504164647265737300737426
:10CB70006172744874747053657276657200737470
:10CB80006F7074487474705365727665720068745F
:10CB90007470536572766572476574526571756518
:10CBA000737400726573706F6E64546F4874747040
:10CBB000526571756573740068747470436F6E6E3E
:10CBC00065637400687474704973436F6E6E656357
:10CBD000746564006874747052657175657374006F
:10CBE00068747470526573706F6E736500687474E6
:10CBF00070436C6F7365001A1B1C03040607090A57
:10CC0000171819000000000008080800080A4A4028
:10CC100000000A5FEA5FEA0ED92ED36E193244890A
:10CC2000330C924C924D0808000000048808080458
:10CC30000804848488000A448A4000048EC480006A
:10CC40000000048800000EC000000000080001225F
:10CC50004488100C9252524C048C84848E1C824C5A
:10CC6000901E1EC244924C06CA525FE21FF01EC1C3
:10CC70003E02448ED12E1FE24488100ED12ED12EBA
:10CC80000ED12EC488000800080000048004880229
:10CC900044880482000EC00EC008048244880ED16D
:10CCA00026C0040ED135B36C0C925ED2521C925C3D
:10CCB000925C0ED010100E1C9252525C1ED01C9032
:10CCC0001E1ED01C90100ED013712E12525ED25226
:10CCD0001C8808081C1FE242524C125498149210EF
:10CCE0001010101E113B75B131113935B3710C9212
:10CCF00052524C1C925C90100C92524C861C925CCE
:10CD000092510ED00C825C1FE484848412525252E1
:10CD10004C1131312A44113135BB7112524C9252AF
:10CD2000112A4484841EC488101E0EC808080E10E0
:10CD3000080482410EC242424E048A4000000000B4
:10CD400000001F0804800000000ED2524F10101C7B
:10CD5000925C000ED0100E02424ED24E0C925C90AD
:10CD60000E06C81C88080ED24EC24C10101C9252DF
:10CD70000800080808024002424C10149814920857
:10CD800008080806001B75B131001C925252000CB5
:10CD900092524C001C925C90000ED24EC2000ED0FB
:10CDA00010100006C8049808080EC8070012525256
:10CDB0004F0011312A4400113135BB00124C8C92C6
:10CDC00000112A4498001EC4881E06C48C8486085C
:10CDD0000808080818080C881800000C8360000078
:10CDE000000000000100000002000000030000003D
:10CDF000040000000500000006000000070000001D
:10CE000008000000090000000A0000000B000000FC
:10CE10000C0000000D0000000E0000000F000000DC
:10CE200010000000120000001400000016000000B6
:10CE3000180000001A0000001C0000001E00000086
:10CE40002000000023000000260000002900000050
:10CE50002C0000002F00000032000000360000000F
:10CE60003A0000003E0000004200000046000000C2
:10CE70004B00000050000000550000005A00000068
:10CE800061000000680000006F00000076000000F4
:10CE90007D000000840000008B0000009200000074
:10CEA00099000000A0000000A7000000AE000000F4
:10CEB000B5000000BC000000C3000000CA00000074
:10CEC000D1000000D8000000DF000000E6000000F4
:10CED000ED000000F4000000FB000000FF00000077
:10CEE00030CF0000ED3800003BCF0000313E0000A5
:10CEF00045CF0000A93A000052CF0000A13C00003D
:10CF000059CF0000F13C000062CF0000413D00001D
:10CF10006ECF00003D3C00007FCF0000193B0000B9
:10CF20008CCF0000D53B0000646973706C617900A0
:10CF30006C696768744C6576656C006D62446973F2
:10CF4000706C6179006D62446973706C61794F66D1
:10CF500066006D62506C6F74006D62556E706C6F20
:10CF600074006D62447261775368617065006D6230
:10CF70005368617065466F724C6574746572006EBB
:10CF8000656F506978656C53656E64006E656F50AF
:10CF90006978656C53657450696E004E6F742065D6
:10CFA0006E6F75676820726F6F6D206576656E2095
:10CFB000616674657220636F6D70616374696F6E12
:10CFC00000436F6D70616374656420466C617368C3
:10CFD00020636F64652073746F72650A2564206234
:10CFE0007974657320757365642028256425252967
:10CFF000206F6620256400426164207265636F7251
:10D000006420666F756E6420647572696E6720694E
:10D010006E697469616C697A6174696F6E00256408
:10D020002025642025642028256420776F7264738E
:10D0300029002564207265636F7264732C20256457
:10D0400020776F7264732C206D61784944202564C9
:10D050002C20636F6D70616374696F6E20637963F8
:10D060006C657320256400526573746F726564206B
:10D0700025642073637269707473005374617274F1
:10D08000656400726164696F000000001CD10000DB
:10D09000F947000029D10000954A000039D100006D
:10D0A000154A000047D10000294C000052D1000071
:10D0B0002148000062D10000A948000076D100009C
:10D0C0009148000085D100000B4E000091D1000076
:10D0D000894D00009AD100002D4D0000A5D100001F
:10D0E000754C0000B0D10000B14C0000B9D1000077
:10D0F000E54C0000C2D1000031480000D1D1000051
:10D1000011480000DAD10000414800006E6F6E65E2
:10D11000006F7468657200706169720064697361A0
:10D12000626C65526164696F006D657373616765F8
:10D130005265636569766564007061636B657452FE
:10D14000656365697665007061636B657453656ED0
:10D1500064007265636569766564496E74656765C8
:10D16000720072656365697665644D6573736167A6
:10D17000655479706500726563656976656453749A
:10D1800072696E670073656E64496E746567657277
:10D190000073656E64506169720073656E645374E8
:10D1A00072696E67007365744368616E6E656C00CA
:10D1B00073657447726F757000736574506F77652F
:10D1C00072007369676E616C537472656E67746820
:10D1D000006465766963654944006C6173744D65EC
:10D1E000737361676549440000000000963007775B
:10D1F0002C610EEEBA51099919C46D078FF46A704B
:10D2000035A563E9A395649E3288DB0EA4B8DC796A
:10D210001EE9D5E088D9D2972B4CB609BD7CB17EEA
:10D22000072DB8E7911DBF906410B71DF220B06ABA
:10D230004871B9F3DE41BE847DD4DA1AEBE4DD6DCA
:10D2400051B5D4F4C785D38356986C13C0A86B64CA
:10D250007AF962FDECC9658A4F5C0114D96C0663EA
:10D26000633D0FFAF50D088DC8206E3B5E10694CCA
:10D27000E44160D5727167A2D1E4033C47D4044B0A
:10D28000FD850DD26BB50AA5FAA8B5356C98B242EA
:10D29000D6C9BBDB40F9BCACE36CD832755CDF456A
:10D2A000CF0DD6DC593DD1ABAC30D9263A00DE519A
:10D2B0008051D7C81661D0BFB5F4B42123C4B3568A
:10D2C0009995BACF0FA5BDB89EB802280888055F0A
:10D2D000B2D90CC624E90BB1877C6F2F114C68586A
:10D2E000AB1D61C13D2D66B69041DC760671DB0158
:10D2F000BC20D2982A10D5EF8985B1711FB5B6062A
:10D30000A5E4BF9F33D4B8E8A2C9077834F9000F69
:10D310008EA8099618980EE1BB0D6A7F2D3D6D0809
:10D32000976C6491015C63E6F4516B6B62616C1CF9
:10D33000D83065854E0062F2ED95066C7BA5011B29
:10D34000C1F4088257C40FF5C6D9B06550E9B712C9
:10D35000EAB8BE8B7C88B9FCDF1DDD62492DDA1589
:10D36000F37CD38C654CD4FB5861B24DCE51B53AA9
:10D370007400BCA3E230BBD441A5DF4AD795D83DA9
:10D380006DC4D1A4FBF4D6D36AE96943FCD96E34E9
:10D39000468867ADD0B860DA732D0444E51D0333C9
:10D3A0005F4C0AAAC97C0DDD3C710550AA410227D9
:10D3B00010100BBE86200CC925B56857B3856F20A9
:10D3C00009D466B99FE461CE0EF9DE5E98C9D92909
:10D3D0002298D0B0B4A8D7C7173DB359810DB42E49
:10D3E0003B5CBDB7AD6CBAC02083B8EDB6B3BF9A95
:10D3F0000CE2B6039AD2B1743947D5EAAF77D29D21
:10D400001526DB048316DC73120B63E3843B649400
:10D410003E6A6D0DA85A6A7A0BCF0EE49DFF099300
:10D4200027AE000AB19E077D44930FF0D2A3088770
:10D4300068F2011EFEC206695D5762F7CB67658020
:10D4400071366C19E7066B6E761BD4FEE02BD38920
:10D450005A7ADA10CC4ADD676FDFB9F9F9EFBE8E80
:10D4600043BEB717D58EB060E8A3D6D67E93D1A1C0
:10D47000C4C2D83852F2DF4FF167BBD16757BCA6A0
:10D48000DD06B53F4B36B248DA2B0DD84C1B0AAF40
:10D49000F64A0336607A0441C3EF60DF55DF67A8C0
:10D4A000EF8E6E3179BE69468CB361CB1A8366BC50
:10D4B000A0D26F2536E2685295770CCC03470BBBA0
:10D4C000B91602222F260555BE3BBAC5280BBDB2A0
:10D4D000925AB42B046AB35CA7FFD7C231CFD0B540
:10D4E0008B9ED92C1DAEDE5BB0C2649B26F263EC32
:10D4F0009CA36A750A936D02A906099C3F360EEB40
:10D500008567077213570005824ABF95147AB8E2FF
:10D51000AE2BB17B381BB60C9B8ED2920DBED5E5DF
:10D52000B7EFDC7C21DFDB0BD4D2D38642E2D4F12F
:10D53000F8B3DD686E83DA1FCD16BE815B26B9F6BF
:10D54000E177B06F7747B718E65A0888706A0FFF1F
:10D55000CA3B06665C0B0111FF9E658F69AE62F8DF
:10D56000D3FF6B6145CF6C1678E20AA0EED20DD7DF
:10D570005483044EC2B30339612667A7F71660D0FF
:10D580004D476949DB776E3E4A6AD1AEDC5AD6D93F
:10D59000660BDF40F03BD83753AEBCA9C59EBBDE5F
:10D5A0007FCFB247E9FFB5301CF2BDBD8AC2BACA0F
:10D5B0003093B353A6A3B4240536D0BA9306D7CD7F
:10D5C0002957DE54BF67D9232E7A66B3B84A61C49F
:10D5D000021B685D942B6F2A37BE0BB4A18E0CC35F
:10D5E0001BDF055A8DEF022D416C6C207461736B4B
:10D5F000732073746F707065640076303739002063
:10D600002573202573004D656D6F727920636C65FD
:10D6100061726564004E6F20667265652074617387
:10D620006B20656E747269657300000074D600002B
:10D63000C960000081D60000555D00008DD6000055
:10D64000FF60000093D600000F61000099D6000033
:10D650001F6100009FD60000895D0000A9D6000070
:10D6600031610000B1D60000C95E000073656E73C1
:10D670006F727300616363656C65726174696F6E6C
:10D680000074656D70657261747572650074696CA3
:10D6900074580074696C74590074696C745A00741D
:10D6A0006F756368526561640069326352656164D5
:10D6B00000693263577269746500000030D700005A
:10D6C000B96100003ED70000BD61000047D70000EF
:10D6D000C961000051D70000CD6100005AD7000099
:10D6E000D16100005FD70000D561000064D7000061
:10D6F000D961000070D70000DD61000077D700001D
:10D70000E161000080D70000E561000085D70000DE
:10D71000E961000090D70000ED6100009AD7000099
:10D72000C1610000A4D70000C561000074667400E8
:10D73000656E61626C65446973706C6179006765E0
:10D7400074576964746800676574486569676874CC
:10D7500000736574506978656C006C696E65007261
:10D7600065637400726F756E6465645265637400FE
:10D77000636972636C6500747269616E676C6500E1
:10D780007465787400746674546F756368656400BA
:10D79000746674546F7563685800746674546F755A
:10D7A00063685900746674546F756368507265736A
:10D7B000737572650076617273000000DCD700003B
:10D7C0007D660000E6D700005D660000EFD7000030
:10D7D00039660000FBD70000C56500007661724520
:10D7E0007869737473007661724E616D656400735D
:10D7F00065745661724E616D6564007661724E614A
:10D800006D65466F72496E6465780057656C636F2D
:10D810006D6520746F204D6963726F426C6F636B2E
:10D82000732100705F73706920213D204E554C4C70
:10D83000002F686F6D652F62726F6D61676F736126
:10D840002F2E706C6174666F726D696F2F706163DB
:10D850006B616765732F6672616D65776F726B2D93
:10D8600061726475696E6F6E6F726469636E726601
:10D87000352F6C69627261726965732F5350492F3D
:10D880005350492E63707000535049436C61737359
:10D890003A3A535049436C617373284E52465F5372
:10D8A00050495F547970652A2C2075696E74385F11
:10D8B000742C2075696E74385F742C2075696E74D1
:10D8C000385F742900000000000000000000000024
:10D8D00089680000456800006B68000075680000FA
:10D8E0007F6800006968000003000000020000007B
:10D8F000010000000400000005000000110000000D
:10D900000C0000000B000000120000000A000000E4
:10D91000060000001A0000001400000017000000BC
:10D92000160000001500000010000000FFFFFFFFC0
:10D93000FFFFFFFF000000001E00000019000000B4
:10D9400018000000070000000800000009000000A7
:10D950000D0000000E0000000F0000001C00000081
:10D960001B0000001D00000013000000000000006C
:10D9700000000000396D000069740000B96D0000FE
:10D98000CD6D0000C36D0000356D0000296D0000F5
:10D99000D96D0000556D0000256D000000000000ED
:10D9A000000000000000304300000000000030C311
:10D9B0007371727400000000FB21F93FFB210940E4
:10D9C0007CD91240FB2119407A6A1F407CD9224041
:10D9D000BBFD2540FB2129403A462C407A6A2F4066
:10D9E0005C4731407CD932409C6B3440BBFD3540B4
:10D9F000DB8F3740FB2139401BB43A403A463C406C
:10DA00005AD83D407A6A3F404C7E40405C47414096
:10DA10006C1042407CD942408CA243409C6B4440F5
:10DA2000AC344540BBFD4540CBC64640DB8F47404C
:10DA3000EB584840FB21494083F9A200444E6E0058
:10DA4000FC291500D1572700DD34F50062DBC0004A
:10DA50003C999500419043006351FE00BBDEAB0052
:10DA6000B761C5003A6E2400D24D42004906E0007D
:10DA700009EA2E001C92D100EB1DFE0029B11C000A
:10DA8000E83EA700F535820044BB2E009CE98400E7
:10DA9000B4267000417E5F00D6913900538339006F
:10DAA0009CF439008B5F840028F9BD00F81F3B000F
:10DAB000DEFF97000F980500112FEF000A5A8B0028
:10DAC0006D1F6D00CF7E360009CB2700464FB70093
:10DAD0009E663F002DEA5F00BA277500E5EBC700A0
:10DAE0003D7BF100F739070092528A00FB6BEA0098
:10DAF0001FB15F00085D8D00300356007BFC4600BF
:10DB0000F0AB6B0020BCCF0036F49A00E3A91D00F7
:10DB10005E619100081BE60085996500A0145F0016
:10DB20008D40680080D8FF0027734D000606310045
:10DB3000CA561500C9A873007BE260006B8CC00058
:10DB400000000040FB21F93F000000002D44743E1E
:10DB5000000000809846F83C0000006051CC783B03
:10DB600000000080831BF0390000004020257A3837
:10DB7000000000802282E336000000001DF36935BA
:10DB80000200000003000000040000000600000086
:10DB9000609100000A9100000A9100003892000094
:10DBA00006910000069100002E92000038920000BD
:10DBB000069100002E9200000691000038920000AD
:10DBC0003C9200003C9200003C9200004492000015
:10DBD0003C9C0000AE9A0000F29A0000569A0000A9
:10DBE000F29A0000E29B0000F29A0000569A0000B0
:10DBF000AE9A0000AE9A0000E29B0000569A000028
:10DC00004E9A00004E9A00004E9A0000F09B0000D1
:10DC100064A3000066A2000066A2000084A50000C4
:10DC200060A2000060A200006CA5000084A50000B6
:10DC300060A200006CA5000060A2000084A50000A6
:10DC40007AA500007AA500007AA5000088A500004A
:10DC50002C2066756E6374696F6E3A200061737371
:10DC6000657274696F6E2022257322206661696C6B
:10DC700065643A2066696C6520222573222C206C2D
:10DC8000696E65202564257325730A0084000020D1
:10DC9000232D302B2000686C4C0065666745464795
:10DCA0000030313233343536373839414243444518
:10DCB0004600303132333435363738396162636487
:10DCC0006566000000000000000000000000000089
:10DCD0000000000000000000000000000000000044
:10DCE0000000000000000000000000000000000034
:10DCF0000000000000000000000000000000000024
:10DD00000000000000000000000000000000000013
:10DD10000000000000000000000000000000000003
:10DD2000000000004300504F5349580000202020BD
:10DD300020202020202028282828282020202020BB
:10DD4000202020202020202020202020208810108B
:10DD500010101010101010101010101010040404E7
:10DD600004040404040404101010101010104141A5
:10DD70004141414101010101010101010101010193
:10DD800001010101010101011010101010104242A7
:10DD90004242424202020202020202020202020263
:10DDA0000202020202020202101010102000000003
:10DDB0000000000000000000000000000000000063
:10DDC0000000000000000000000000000000000053
:10DDD0000000000000000000000000000000000043
:10DDE0000000000000000000000000000000000033
:10DDF0000000000000000000000000000000000023
:10DE00000000000000000000000000000000000012
:10DE10000000000000000000000000000000000002
:10DE200000000000000000000000000000000000F2
:04DE300000000000EE
:08DE3400D422FF7F0100000071
:10DE3C00FFFFFFFF4006000001000000E803DC05C7
:10DE4C00DC05DC05DC050000FFFFFFFFFFFFFFFF2B
:10DE5C001800000019FCFFFFFFFFFFFFFF00000090
:10DE6C000200000003000000FFFFFFFF00000000A5
:10DE7C00010000000000020001000000FFFFFFFF96
:10DE8C00000000000200000000000400020000007E
:10DE9C00FFFFFFFF0000000003000000000008006F
:10DEAC00030000000A000000080000000100000050
:10DEBC008400002000000000E4DC000004DD000011
:10DECC00C4DC0000000000000000000000000000A6
:10DEDC000000000000000000000000000000000036
:10DEEC000000000000000000000000000000000026
:10DEFC000000000000000000000000000000000016
:10DF0C000000000000000000000000000000000005
:10DF1C0000000000430000000000000000000000B2
:10DF2C0000000000000000000000000000000000E5
:10DF3C000000000043000000000000000000000092
:10DF4C0000000000000000000000000000000000C5
:10DF5C000000000043000000000000000000000072
:10DF6C0000000000000000000000000000000000A5
:10DF7C000000000043000000000000000000000052
:10DF8C000000000000000000000000000000000085
:10DF9C000000000043000000000000000000000032
:10DFAC000000000000000000000000000000000065
:10DFBC000000000043000000000000000000000012
:10DFCC000000000000000000000000000000000045
:10DFDC0000000000430000000000000000000000F2
:10DFEC000000000000000000000000000000000025
:10DFFC000000000091C40000A9BE00000000000059
:10E00C002CDD0000D2C6000033CA000033CA000069
:10E01C0033CA000033CA000033CA000033CA000000
:10E02C0033CA000033CA000033CA0000FFFFFFFFF1
:10E03C00FFFFFFFFFFFFFFFFFFFF00000100415349
:10E04C0043494900000000000000000000000000EF
:10E05C000000000000000000000000000000415320
:10E06C0043494900000000000000000000000000CF
:10E07C000000000000000000000000000000000094
:10E08C00E9000000156800005D6B00008570000061
:04E09C00C1000000BF
:0400000300006BF995
:00000001FF
